Microchip Technology Inc, v1.25 (A)

Tool Name:
  c:\program files (x86)\microchip\xc16\v1.25\bin\bin\..\bin/elf-ld.exe

Command:
  -p24FJ128GA406 \
  -o \
  dist/default/production/O5DaughterDbg.production.elf \
  -Lc:/program files (x86)/microchip/xc16/v1.25/bin/bin/.. \
  -Lc:/program files (x86)/microchip/xc16/v1.25/bin/bin/../../lib \
  -Lc:/program files (x86)/microchip/xc16/v1.25/bin/bin/../../support/PIC24E/gld \
  -Lc:/program files (x86)/microchip/xc16/v1.25/bin/bin/../../support/PIC24F/gld \
  -Lc:/program files (x86)/microchip/xc16/v1.25/bin/bin/../../support/PIC24H/gld \
  -Lc:/program files (x86)/microchip/xc16/v1.25/bin/bin/../../support/dsPIC30F/gld \
  -Lc:/program files (x86)/microchip/xc16/v1.25/bin/bin/../../support/dsPIC33E/gld \
  -Lc:/program files (x86)/microchip/xc16/v1.25/bin/bin/../../support/dsPIC33F/gld \
  build/default/production/_ext/1470100448/mbascii.o \
  build/default/production/_ext/833655638/mbfunccoils.o \
  build/default/production/_ext/833655638/mbfuncdiag.o \
  build/default/production/_ext/833655638/mbfuncdisc.o \
  build/default/production/_ext/833655638/mbfuncholding.o \
  build/default/production/_ext/833655638/mbfuncinput.o \
  build/default/production/_ext/833655638/mbfuncother.o \
  build/default/production/_ext/833655638/mbutils.o \
  build/default/production/_ext/1433339410/portevent.o \
  build/default/production/_ext/1433339410/portserial.o \
  build/default/production/_ext/1433339410/porttimer.o \
  build/default/production/_ext/1477781822/mbcrc.o \
  build/default/production/_ext/1477781822/mbrtu.o \
  build/default/production/_ext/1043210786/debug.o \
  build/default/production/_ext/1043210786/mb.o \
  build/default/production/_ext/1472/main.o \
  build/default/production/_ext/1472/mcc.o \
  build/default/production/_ext/1472/periph.o \
  build/default/production/_ext/1472/sys_timer.o \
  build/default/production/_ext/1472/misc.o \
  build/default/production/_ext/1472/buffer.o \
  build/default/production/_ext/1472/serial.o \
  build/default/production/_ext/1472/config.o \
  build/default/production/_ext/1472/flash_mem.o \
  build/default/production/_ext/1472/inst_port.o \
  build/default/production/_ext/1472/dig_io.o \
  --local-stack \
  --defsym=__MPLAB_BUILD=1 \
  -Tp24FJ128GA406.gld.00 \
  --stack=1024 \
  --check-sections \
  --data-init \
  --pack-data \
  --handles \
  --isr \
  --no-gc-sections \
  --fill-upper=0 \
  --stackguard=16 \
  --no-force-link \
  --smart-io \
  -Map=dist/default/production/O5DaughterDbg.production.map \
  --report-mem \
  --cref \
  --memorysummary \
  dist/default/production/memoryfile.xml \
  -start-group \
  --library=pic30-elf \
  --library=m-elf \
  --library=c-elf \
  -end-group \


Optional library libpPIC24Fxxx.a not found
Archive member included because of file (symbol)

c:/program files (x86)/microchip/xc16/v1.25/bin/bin/../../lib\libpic30-elf.a(crt0_extended.o)
                              (__resetPRI)
c:/program files (x86)/microchip/xc16/v1.25/bin/bin/../../lib\libpic30-elf.a(data_init_extended.o)
                              c:/program files (x86)/microchip/xc16/v1.25/bin/bin/../../lib\libpic30-elf.a(crt0_extended.o) (__data_init_extended)
c:/program files (x86)/microchip/xc16/v1.25/bin/bin/../../lib\libm-elf.a(divsi3.eo)
                              build/default/production/_ext/1472/sys_timer.o (___divsi3)
c:/program files (x86)/microchip/xc16/v1.25/bin/bin/../../lib\libm-elf.a(udivsi3.eo)
                              build/default/production/_ext/1477781822/mbrtu.o (___udivsi3)
c:/program files (x86)/microchip/xc16/v1.25/bin/bin/../../lib\libc-elf.a(atoi.eo)
                              build/default/production/_ext/1472/main.o (_atoi)
c:/program files (x86)/microchip/xc16/v1.25/bin/bin/../../lib\libc-elf.a(atol.eo)
                              build/default/production/_ext/1472/main.o (_atol)
c:/program files (x86)/microchip/xc16/v1.25/bin/bin/../../lib\libc-elf.a(fassert.eo)
                              build/default/production/_ext/1470100448/mbascii.o (__fassert)
c:/program files (x86)/microchip/xc16/v1.25/bin/bin/../../lib\libc-elf.a(fprintf.eo)
                              c:/program files (x86)/microchip/xc16/v1.25/bin/bin/../../lib\libc-elf.a(fassert.eo) (_fprintf)
c:/program files (x86)/microchip/xc16/v1.25/bin/bin/../../lib\libc-elf.a(memcpy.eo)
                              build/default/production/_ext/833655638/mbfuncother.o (_memcpy)
c:/program files (x86)/microchip/xc16/v1.25/bin/bin/../../lib\libc-elf.a(memset.eo)
                              build/default/production/_ext/1472/main.o (_memset)
c:/program files (x86)/microchip/xc16/v1.25/bin/bin/../../lib\libc-elf.a(strtol.eo)
                              build/default/production/_ext/1472/main.o (_strtol)
c:/program files (x86)/microchip/xc16/v1.25/bin/bin/../../lib\libc-elf.a(signal.eo)
                              c:/program files (x86)/microchip/xc16/v1.25/bin/bin/../../lib\libc-elf.a(fassert.eo) (_abort)
c:/program files (x86)/microchip/xc16/v1.25/bin/bin/../../lib\libc-elf.a(_iob.eo)
                              c:/program files (x86)/microchip/xc16/v1.25/bin/bin/../../lib\libc-elf.a(fassert.eo) (__iob)
c:/program files (x86)/microchip/xc16/v1.25/bin/bin/../../lib\libc-elf.a(errno.elo)
                              c:/program files (x86)/microchip/xc16/v1.25/bin/bin/../../lib\libc-elf.a(strtol.eo) (_errno)
c:/program files (x86)/microchip/xc16/v1.25/bin/bin/../../lib\libc-elf.a(exit.elo)
                              c:/program files (x86)/microchip/xc16/v1.25/bin/bin/../../lib\libc-elf.a(signal.eo) (_exit)
c:/program files (x86)/microchip/xc16/v1.25/bin/bin/../../lib\libc-elf.a(stdclean.elo)
                              c:/program files (x86)/microchip/xc16/v1.25/bin/bin/../../lib\libc-elf.a(exit.elo) (__cleanup)
c:/program files (x86)/microchip/xc16/v1.25/bin/bin/../../lib\libc-elf.a(sprintf_cdnopsuxX.XXeo)
                              build/default/production/_ext/1472/main.o (__sprintf_cdnopsuxX)
c:/program files (x86)/microchip/xc16/v1.25/bin/bin/../../lib\libc-elf.a(doprnt_cdnopsuxX.XXeo)
                              c:/program files (x86)/microchip/xc16/v1.25/bin/bin/../../lib\libc-elf.a(sprintf_cdnopsuxX.XXeo) (__vfprintf_cdnopsuxX)
c:/program files (x86)/microchip/xc16/v1.25/bin/bin/../../lib\libc-elf.a(isalpha.eso)
                              c:/program files (x86)/microchip/xc16/v1.25/bin/bin/../../lib\libc-elf.a(strtol.eo) (_isalpha)
c:/program files (x86)/microchip/xc16/v1.25/bin/bin/../../lib\libc-elf.a(isspace.eso)
                              c:/program files (x86)/microchip/xc16/v1.25/bin/bin/../../lib\libc-elf.a(strtol.eo) (_isspace)
c:/program files (x86)/microchip/xc16/v1.25/bin/bin/../../lib\libc-elf.a(toupper.eso)
                              build/default/production/_ext/1472/main.o (_toupper)
c:/program files (x86)/microchip/xc16/v1.25/bin/bin/../../lib\libc-elf.a(doprnt.eo)
                              c:/program files (x86)/microchip/xc16/v1.25/bin/bin/../../lib\libc-elf.a(fprintf.eo) (_vfprintf)
c:/program files (x86)/microchip/xc16/v1.25/bin/bin/../../lib\libc-elf.a(fputc.eo)
                              c:/program files (x86)/microchip/xc16/v1.25/bin/bin/../../lib\libc-elf.a(doprnt_cdnopsuxX.XXeo) (_fputc)
c:/program files (x86)/microchip/xc16/v1.25/bin/bin/../../lib\libc-elf.a(powers.eo)
                              c:/program files (x86)/microchip/xc16/v1.25/bin/bin/../../lib\libc-elf.a(doprnt.eo) (__powers_)
c:/program files (x86)/microchip/xc16/v1.25/bin/bin/../../lib\libc-elf.a(flsbuf.eo)
                              c:/program files (x86)/microchip/xc16/v1.25/bin/bin/../../lib\libc-elf.a(fputc.eo) (__flsbuf)
c:/program files (x86)/microchip/xc16/v1.25/bin/bin/../../lib\libpic30-elf.a(_exit.eo)
                              c:/program files (x86)/microchip/xc16/v1.25/bin/bin/../../lib\libc-elf.a(exit.elo) (__exit)
c:/program files (x86)/microchip/xc16/v1.25/bin/bin/../../lib\libpic30-elf.a(write.eo)
                              c:/program files (x86)/microchip/xc16/v1.25/bin/bin/../../lib\libc-elf.a(fputc.eo) (_write)
c:/program files (x86)/microchip/xc16/v1.25/bin/bin/../../lib\libpic30-elf.a(c30_uart.eo)
                              c:/program files (x86)/microchip/xc16/v1.25/bin/bin/../../lib\libpic30-elf.a(write.eo) (___C30_UART)
c:/program files (x86)/microchip/xc16/v1.25/bin/bin/../../lib\libm-elf.a(adddf3.eo)
                              c:/program files (x86)/microchip/xc16/v1.25/bin/bin/../../lib\libc-elf.a(doprnt.eo) (___adddf3)
c:/program files (x86)/microchip/xc16/v1.25/bin/bin/../../lib\libm-elf.a(deqltle.eo)
                              c:/program files (x86)/microchip/xc16/v1.25/bin/bin/../../lib\libc-elf.a(doprnt.eo) (___ltdf2)
c:/program files (x86)/microchip/xc16/v1.25/bin/bin/../../lib\libm-elf.a(dgtge.eo)
                              c:/program files (x86)/microchip/xc16/v1.25/bin/bin/../../lib\libc-elf.a(doprnt.eo) (___gedf2)
c:/program files (x86)/microchip/xc16/v1.25/bin/bin/../../lib\libm-elf.a(divdf3.eo)
                              c:/program files (x86)/microchip/xc16/v1.25/bin/bin/../../lib\libc-elf.a(doprnt.eo) (___divdf3)
c:/program files (x86)/microchip/xc16/v1.25/bin/bin/../../lib\libm-elf.a(dne.eo)
                              c:/program files (x86)/microchip/xc16/v1.25/bin/bin/../../lib\libc-elf.a(doprnt.eo) (___nedf2)
c:/program files (x86)/microchip/xc16/v1.25/bin/bin/../../lib\libm-elf.a(dpack.eo)
                              c:/program files (x86)/microchip/xc16/v1.25/bin/bin/../../lib\libm-elf.a(adddf3.eo) (__dpack)
c:/program files (x86)/microchip/xc16/v1.25/bin/bin/../../lib\libm-elf.a(dunpack2.eo)
                              c:/program files (x86)/microchip/xc16/v1.25/bin/bin/../../lib\libm-elf.a(adddf3.eo) (__dunpack2)
c:/program files (x86)/microchip/xc16/v1.25/bin/bin/../../lib\libm-elf.a(extendsfdf.eo)
                              c:/program files (x86)/microchip/xc16/v1.25/bin/bin/../../lib\libc-elf.a(doprnt.eo) (___extendsfdf2)
c:/program files (x86)/microchip/xc16/v1.25/bin/bin/../../lib\libm-elf.a(fixunsdfdi.eo)
                              c:/program files (x86)/microchip/xc16/v1.25/bin/bin/../../lib\libc-elf.a(doprnt.eo) (___fixunsdfdi)
c:/program files (x86)/microchip/xc16/v1.25/bin/bin/../../lib\libm-elf.a(fixunsdfsi.eo)
                              c:/program files (x86)/microchip/xc16/v1.25/bin/bin/../../lib\libc-elf.a(doprnt.eo) (___fixunsdfsi)
c:/program files (x86)/microchip/xc16/v1.25/bin/bin/../../lib\libm-elf.a(floatundidf.eo)
                              c:/program files (x86)/microchip/xc16/v1.25/bin/bin/../../lib\libc-elf.a(doprnt.eo) (___floatundidf)
c:/program files (x86)/microchip/xc16/v1.25/bin/bin/../../lib\libm-elf.a(floatunsidf.eo)
                              c:/program files (x86)/microchip/xc16/v1.25/bin/bin/../../lib\libc-elf.a(doprnt.eo) (___floatunsidf)
c:/program files (x86)/microchip/xc16/v1.25/bin/bin/../../lib\libm-elf.a(frexp.eo)
                              c:/program files (x86)/microchip/xc16/v1.25/bin/bin/../../lib\libc-elf.a(doprnt.eo) (_frexpl)
c:/program files (x86)/microchip/xc16/v1.25/bin/bin/../../lib\libm-elf.a(funpack.eo)
                              c:/program files (x86)/microchip/xc16/v1.25/bin/bin/../../lib\libm-elf.a(extendsfdf.eo) (__funpack)
c:/program files (x86)/microchip/xc16/v1.25/bin/bin/../../lib\libm-elf.a(muldf3.eo)
                              c:/program files (x86)/microchip/xc16/v1.25/bin/bin/../../lib\libc-elf.a(doprnt.eo) (___muldf3)
c:/program files (x86)/microchip/xc16/v1.25/bin/bin/../../lib\libm-elf.a(subdf3.eo)
                              c:/program files (x86)/microchip/xc16/v1.25/bin/bin/../../lib\libc-elf.a(doprnt.eo) (___subdf3)
c:/program files (x86)/microchip/xc16/v1.25/bin/bin/../../lib\libm-elf.a(mulsi3.eo)
                              c:/program files (x86)/microchip/xc16/v1.25/bin/bin/../../lib\libc-elf.a(atol.eo) (___mulsi3)
c:/program files (x86)/microchip/xc16/v1.25/bin/bin/../../lib\libm-elf.a(divmoddi3.eo)
                              c:/program files (x86)/microchip/xc16/v1.25/bin/bin/../../lib\libc-elf.a(doprnt_cdnopsuxX.XXeo) (___udivdi3)
c:/program files (x86)/microchip/xc16/v1.25/bin/bin/../../lib\libm-elf.a(muldi3.eo)
                              c:/program files (x86)/microchip/xc16/v1.25/bin/bin/../../lib\libc-elf.a(doprnt_cdnopsuxX.XXeo) (___muldi3)
c:/program files (x86)/microchip/xc16/v1.25/bin/bin/../../lib\libm-elf.a(dcompare.eo)
                              c:/program files (x86)/microchip/xc16/v1.25/bin/bin/../../lib\libm-elf.a(deqltle.eo) (__dcompare)
c:/program files (x86)/microchip/xc16/v1.25/bin/bin/../../lib\libm-elf.a(dpropagateNaN.eo)
                              c:/program files (x86)/microchip/xc16/v1.25/bin/bin/../../lib\libm-elf.a(dunpack2.eo) (__dPropagateNaN)
c:/program files (x86)/microchip/xc16/v1.25/bin/bin/../../lib\libm-elf.a(dtype.eo)
                              c:/program files (x86)/microchip/xc16/v1.25/bin/bin/../../lib\libm-elf.a(dcompare.eo) (__dtype)
c:/program files (x86)/microchip/xc16/v1.25/bin/bin/../../lib\libm-elf.a(dunpack.eo)
                              c:/program files (x86)/microchip/xc16/v1.25/bin/bin/../../lib\libm-elf.a(dunpack2.eo) (__dunpack)
c:/program files (x86)/microchip/xc16/v1.25/bin/bin/../../lib\libm-elf.a(umuldi3.eo)
                              c:/program files (x86)/microchip/xc16/v1.25/bin/bin/../../lib\libm-elf.a(muldi3.eo) (___umuldi3)


xc16-ld 1.25 (A)

Program Memory  [Origin = 0x100, Length = 0x15680]

section                    address   length (PC units)   length (bytes) (dec)
-------                    -------   -----------------   --------------------
.const                       0x100               0x828           0xc3c  (3132)
.text                        0x928               0x38c           0x552  (1362)
.text                        0xcb4               0x346           0x4e9  (1257)
.params                     0x1000               0x400           0x600  (1536)
.text                       0x1400              0x2a22          0x3f33  (16179)
.text                       0x3e22              0x1dce          0x2cb5  (11445)
.dinit                      0x5bf0               0x358           0x504  (1284)
.text                       0x5f48              0x19ac          0x2682  (9858)

                     Total program memory used (bytes):         0xb3e5  (46053) 35%


Data Memory  [Origin = 0x800, Length = 0x4000]

section                    address      alignment gaps    total length  (dec)
-------                    -------      --------------    -------------------
.nbss                        0x800                   0            0x64  (100)
.ndata                       0x864                   0             0x4  (4)
.nbss                        0x868                   0             0x4  (4)
.ndata                       0x86c                   0             0x2  (2)
.nbss                        0x86e                   0             0x2  (2)
.ndata                       0x870                   0             0x4  (4)
.nbss                        0x874                   0             0x2  (2)
.bss                         0x876                   0          0x2db8  (11704)
.data                       0x362e                   0           0x160  (352)
.bss                        0x378e                   0           0x230  (560)
.data                       0x39be                   0           0x238  (568)
.bss                        0x3bf6                   0            0x20  (32)
.data                       0x3c16                   0            0x24  (36)
.bss                        0x3c3a                   0            0x16  (22)
.data                       0x3c50                   0             0x2  (2)

                        Total data memory used (bytes):         0x3452  (13394) 81%


Dynamic Memory Usage

region                     address                      maximum length  (dec)
------                     -------                      ---------------------
heap                             0                                   0  (0)
stack                       0x3c52                               0xbae  (2990)

                        Maximum dynamic memory (bytes):          0xbae  (2990)


External Symbols in Data Memory (by address):

                    0x080e                  _pxMBFrameCBByteReceived
                    0x0810                  _pxMBFrameCBTransmitterEmpty
                    0x0812                  _pxMBPortCBTimerExpired
                    0x0814                  _pxMBFrameCBReceiveFSMCur
                    0x0816                  _pxMBFrameCBTransmitFSMCur
                    0x0864                  _mbTimeout
                    0x362e                  __powers_
                    0x36de                  __npowers_
                    0x38be                  _ucRTUBuf
                    0x3bd0                  __iob
                    0x3bf4                  __Files
                    0x3c16                  _UxSTARegs
                    0x3c22                  _UxBRGRegs
                    0x3c46                  __outdone
                    0x3c47                  __sibuf
                    0x3c49                  __sobuf
                    0x3c4c                  _errno
                    0x3c4e                  __atexitptr
                    0x3c50                  ___C30_UART

External Symbols in Data Memory (by name):

                    0x3c22                  _UxBRGRegs
                    0x3c16                  _UxSTARegs
                    0x3bf4                  __Files
                    0x3c50                  ___C30_UART
                    0x3c4e                  __atexitptr
                    0x3bd0                  __iob
                    0x36de                  __npowers_
                    0x3c46                  __outdone
                    0x362e                  __powers_
                    0x3c47                  __sibuf
                    0x3c49                  __sobuf
                    0x3c4c                  _errno
                    0x0864                  _mbTimeout
                    0x080e                  _pxMBFrameCBByteReceived
                    0x0814                  _pxMBFrameCBReceiveFSMCur
                    0x0816                  _pxMBFrameCBTransmitFSMCur
                    0x0810                  _pxMBFrameCBTransmitterEmpty
                    0x0812                  _pxMBPortCBTimerExpired
                    0x38be                  _ucRTUBuf

External Symbols in Program Memory (by address):

                  0x0008a6                  _serEnblBits
                  0x0008be                  _pwrBits
                  0x000928                  _eMBASCIIInit
                  0x000968                  _eMBASCIIStart
                  0x00097e                  _eMBASCIIStop
                  0x000990                  _eMBASCIIReceive
                  0x0009e6                  _eMBASCIISend
                  0x000a40                  _xMBASCIIReceiveFSM
                  0x000b20                  _xMBASCIITransmitFSM
                  0x000be2                  _xMBASCIITimerT1SExpired
                  0x000cb4                  _digInit
                  0x000cfe                  _digSerEnable
                  0x000d32                  _digSerDisable
                  0x000d68                  _digSetSerEnable
                  0x000dce                  _digGetSerEnable
                  0x000e02                  _digPwrSet
                  0x000ee8                  _digPwrVecSet
                  0x000fcc                  _digPwrIsOn
                  0x000ff2                  _digPwrGet
                  0x001000                  _paramBuff
                  0x001400                  __resetPRI
                  0x00142c                  __psv_init
                  0x001438                  __data_init_extended
                  0x001438                  __data_init
                  0x001532                  __DefaultInterrupt
                  0x001536                  _isalpha
                  0x00154a                  _isspace
                  0x00155a                  _toupper
                  0x0015d4                  ___divsi3
                  0x0015f2                  ___udivsi3
                  0x001612                  _atoi
                  0x001650                  _atol
                  0x0016a6                  __fassert
                  0x0016c4                  _fprintf
                  0x0016d0                  _memcpy
                  0x0016de                  _memset
                  0x0016ec                  _strtoul
                  0x0017f0                  _strtol
                  0x001880                  _signal
                  0x001892                  _raise
                  0x0018c0                  _abort
                  0x0018c8                  _exit
                  0x0018d2                  __sprintf_cdnopsuxX
                  0x001910                  __vfprintf_cdnopsuxX
                  0x002154                  _vfprintf
                  0x0035ae                  ___adddf3
                  0x0036a8                  ___ltdf2
                  0x0036a8                  ___ledf2
                  0x0036a8                  ___eqdf2
                  0x0036b2                  ___gedf2
                  0x0036b2                  ___gtdf2
                  0x0036bc                  ___divdf3
                  0x003770                  ___nedf2
                  0x00377a                  __dpack
                  0x0037d2                  __dunpack2
                  0x0037f4                  __dreturnNaN
                  0x0037fa                  __dunpack2exit
                  0x003804                  ___extendsfdf2
                  0x003842                  ___fixunsdfdi
                  0x0038a4                  ___fixunsdfsi
                  0x0038f0                  ___floatundidf
                  0x003946                  ___floatunsidf
                  0x00394a                  _frexpl
                  0x00394a                  _frexp
                  0x003984                  __funpack
                  0x0039ae                  ___muldf3
                  0x003a98                  ___subdf3
                  0x003a9c                  ___mulp32eds3
                  0x003a9c                  ___mulp32peds3
                  0x003a9c                  ___mulsi3
                  0x003af4                  ___udivmoddi3
                  0x003bda                  ___udivdi3
                  0x003be8                  ___umoddi3
                  0x003bf0                  ___divdi3
                  0x003c50                  ___moddi3
                  0x003cac                  ___muldi3
                  0x003cfe                  __dcompare
                  0x003d50                  __dPropagateNaN
                  0x003d6c                  __dtype
                  0x003d90                  __dunpack
                  0x003dde                  ___umuldi3
                  0x003e22                  _modBusTask
                  0x003e6a                  _main
                  0x003f18                  _eMBRegInputCB
                  0x003f92                  _eMBRegHoldingCB
                  0x0040c6                  _isBitSet
                  0x0040f8                  _bitSet
                  0x00415a                  _eMBRegCoilsCB
                  0x00437a                  _eMBRegDiscreteCB
                  0x00438c                  _getLine
                  0x00442c                  _signon
                  0x004448                  _checkMenuSeq
                  0x00448e                  _menuTask
                  0x0045cc                  _menuBanner
                  0x0045f8                  _menuConfig
                  0x004694                  _menuHelp
                  0x0046c2                  _menuOpt0
                  0x0046e4                  _menuOpt1
                  0x004700                  _menuOpt2
                  0x004766                  _menuOpt3
                  0x004820                  _menuOpt4
                  0x0048b2                  _menuOpt5
                  0x0048f0                  _menuOpt6
                  0x004974                  _menuOpt7
                  0x0049b4                  _menuOpt8
                  0x0049be                  _menuOpt9
                  0x0049c8                  _serInit
                  0x004ac4                  _serSetBaud
                  0x004b12                  _serGetBaud
                  0x004b34                  _serSetConfig
                  0x004c24                  _serGetConfig
                  0x004cda                  _serGetByte
                  0x004d12                  _serPutByte
                  0x004da0                  _serPutString
                  0x004e1a                  _serPutStringBool
                  0x004e44                  _serRxFlush
                  0x004ee0                  _serTxFlush
                  0x004f30                  _serSetBreak
                  0x005088                  _serGetBreak
                  0x0050aa                  _serIsRxFull
                  0x0050f0                  _serRxAvailable
                  0x00511c                  _serIsTxFull
                  0x005146                  _serIsTxEmpty
                  0x005170                  _serGetErrFlag
                  0x005198                  _serClrXERR
                  0x0051c4                  _serGetXERR
                  0x0051f4                  _serClrOERR
                  0x00523c                  _serGetOERR
                  0x00526a                  _serClrFERR
                  0x005296                  _serGetFERR
                  0x0052c4                  _serClrPERR
                  0x0052f0                  _serGetPERR
                  0x00531e                  _EnterAppCriticalSection
                  0x00532c                  _ExitAppCriticalSection
                  0x005340                  __U1TXInterrupt
                  0x005348                  __U1RXInterrupt
                  0x00539c                  __U2TXInterrupt
                  0x0053a4                  __U2RXInterrupt
                  0x0053f8                  __U3TXInterrupt
                  0x005400                  __U3RXInterrupt
                  0x005454                  __U4TXInterrupt
                  0x00545c                  __U4RXInterrupt
                  0x0054b0                  __U5TXInterrupt
                  0x0054b8                  __U5RXInterrupt
                  0x00550c                  _instPortInit
                  0x00554c                  _instPortTxTask
                  0x005590                  _instPortClearWriteReq
                  0x0055ac                  _instSnapshotRxAvail
                  0x0055d0                  _instPortReadReg
                  0x0058bc                  _instPortWriteReg
                  0x005f48                  _eMBFuncWriteHoldingRegister
                  0x005fa0                  _eMBFuncWriteMultipleHoldingRegister
                  0x006044                  _eMBFuncReadHoldingRegister
                  0x006110                  _eMBFuncReadWriteMultipleHoldingRegister
                  0x006250                  _miscInit
                  0x006266                  _miscRegRead
                  0x006306                  _miscRegWrite
                  0x0063c2                  _setBlinkyDebug
                  0x0063ee                  _getBlinkyDebug
                  0x0063f6                  _blinkyTask
                  0x006532                  _eMBInit
                  0x0065ee                  _eMBRegisterCB
                  0x0066ac                  _eMBClose
                  0x0066ce                  _eMBEnable
                  0x0066ec                  _eMBDisable
                  0x006718                  _eMBPoll
                  0x00680c                  _eMBRTUInit
                  0x006874                  _eMBRTUStart
                  0x006888                  _eMBRTUStop
                  0x00689a                  _eMBRTUReceive
                  0x0068f8                  _eMBRTUSend
                  0x006962                  _xMBRTUReceiveFSM
                  0x0069d2                  _xMBRTUTransmitFSM
                  0x006a2c                  _xMBRTUTimerT35Expired
                  0x006a7a                  _eMBFuncReadCoils
                  0x006b58                  _eMBFuncWriteCoil
                  0x006bea                  _eMBFuncWriteMultipleCoils
                  0x006ca0                  _vMBPortSerialEnable
                  0x006cc8                  _xMBPortSerialInit
                  0x006d78                  _xMBPortSerialPutByte
                  0x006d86                  _xMBPortSerialGetByte
                  0x006d98                  __U6TXInterrupt
                  0x006db8                  __U6RXInterrupt
                  0x006e28                  _EnterCriticalSection
                  0x006e3e                  _ExitCriticalSection
                  0x006e5a                  _memRead
                  0x006ee0                  _memWrite
                  0x006fca                  _memErase
                  0x007000                  _tmrInit
                  0x007020                  _tmrTask
                  0x007028                  _tmrDelayTicks
                  0x007046                  _tmrDelayMs
                  0x0070ac                  _tmrDelayUs
                  0x00710e                  _tmrGetTicks
                  0x00713a                  __T2Interrupt
                  0x00714e                  _xMBUtilSetBits
                  0x0071ec                  _xMBUtilGetBits
                  0x007244                  _prveMBError2Exception
                  0x007276                  _periphInit
                  0x00739a                  _cfgCheck
                  0x007406                  _cfgRead
                  0x007434                  _cfgWrite
                  0x007462                  _cfgSetBootFlag
                  0x007486                  _calcCheckSum
                  0x0074b6                  _bufInit
                  0x0074ea                  _bufPut
                  0x007532                  _bufGet
                  0x007588                  _bufClear
                  0x0075a6                  _eMBFuncReadDiscreteInputs
                  0x007682                  _eMBFuncReadInputRegister
                  0x007750                  _eMBSetSlaveID
                  0x0077b0                  _eMBFuncReportSlaveID
                  0x0077ce                  _xMBPortTimersInit
                  0x0077fe                  _vMBPortTimersEnable
                  0x007808                  _vMBPortTimersDisable
                  0x007816                  __T1Interrupt
                  0x007836                  _usMBCRC16
                  0x007890                  _xMBPortEventInit
                  0x00789a                  _xMBPortEventPost
                  0x0078ac                  _xMBPortEventGet
                  0x0078cc                  _SYSTEM_Initialize
                  0x0078d4                  _OSCILLATOR_Initialize

External Symbols in Program Memory (by name):

                  0x00531e                  _EnterAppCriticalSection
                  0x006e28                  _EnterCriticalSection
                  0x00532c                  _ExitAppCriticalSection
                  0x006e3e                  _ExitCriticalSection
                  0x0078d4                  _OSCILLATOR_Initialize
                  0x0078cc                  _SYSTEM_Initialize
                  0x001532                  __DefaultInterrupt
                  0x007816                  __T1Interrupt
                  0x00713a                  __T2Interrupt
                  0x005348                  __U1RXInterrupt
                  0x005340                  __U1TXInterrupt
                  0x0053a4                  __U2RXInterrupt
                  0x00539c                  __U2TXInterrupt
                  0x005400                  __U3RXInterrupt
                  0x0053f8                  __U3TXInterrupt
                  0x00545c                  __U4RXInterrupt
                  0x005454                  __U4TXInterrupt
                  0x0054b8                  __U5RXInterrupt
                  0x0054b0                  __U5TXInterrupt
                  0x006db8                  __U6RXInterrupt
                  0x006d98                  __U6TXInterrupt
                  0x0035ae                  ___adddf3
                  0x0036bc                  ___divdf3
                  0x003bf0                  ___divdi3
                  0x0015d4                  ___divsi3
                  0x0036a8                  ___eqdf2
                  0x003804                  ___extendsfdf2
                  0x003842                  ___fixunsdfdi
                  0x0038a4                  ___fixunsdfsi
                  0x0038f0                  ___floatundidf
                  0x003946                  ___floatunsidf
                  0x0036b2                  ___gedf2
                  0x0036b2                  ___gtdf2
                  0x0036a8                  ___ledf2
                  0x0036a8                  ___ltdf2
                  0x003c50                  ___moddi3
                  0x0039ae                  ___muldf3
                  0x003cac                  ___muldi3
                  0x003a9c                  ___mulp32eds3
                  0x003a9c                  ___mulp32peds3
                  0x003a9c                  ___mulsi3
                  0x003770                  ___nedf2
                  0x003a98                  ___subdf3
                  0x003bda                  ___udivdi3
                  0x003af4                  ___udivmoddi3
                  0x0015f2                  ___udivsi3
                  0x003be8                  ___umoddi3
                  0x003dde                  ___umuldi3
                  0x003d50                  __dPropagateNaN
                  0x001438                  __data_init
                  0x001438                  __data_init_extended
                  0x003cfe                  __dcompare
                  0x00377a                  __dpack
                  0x0037f4                  __dreturnNaN
                  0x003d6c                  __dtype
                  0x003d90                  __dunpack
                  0x0037d2                  __dunpack2
                  0x0037fa                  __dunpack2exit
                  0x0016a6                  __fassert
                  0x003984                  __funpack
                  0x00142c                  __psv_init
                  0x001400                  __resetPRI
                  0x0018d2                  __sprintf_cdnopsuxX
                  0x001910                  __vfprintf_cdnopsuxX
                  0x0018c0                  _abort
                  0x001612                  _atoi
                  0x001650                  _atol
                  0x0040f8                  _bitSet
                  0x0063f6                  _blinkyTask
                  0x007588                  _bufClear
                  0x007532                  _bufGet
                  0x0074b6                  _bufInit
                  0x0074ea                  _bufPut
                  0x007486                  _calcCheckSum
                  0x00739a                  _cfgCheck
                  0x007406                  _cfgRead
                  0x007462                  _cfgSetBootFlag
                  0x007434                  _cfgWrite
                  0x004448                  _checkMenuSeq
                  0x000dce                  _digGetSerEnable
                  0x000cb4                  _digInit
                  0x000ff2                  _digPwrGet
                  0x000fcc                  _digPwrIsOn
                  0x000e02                  _digPwrSet
                  0x000ee8                  _digPwrVecSet
                  0x000d32                  _digSerDisable
                  0x000cfe                  _digSerEnable
                  0x000d68                  _digSetSerEnable
                  0x000928                  _eMBASCIIInit
                  0x000990                  _eMBASCIIReceive
                  0x0009e6                  _eMBASCIISend
                  0x000968                  _eMBASCIIStart
                  0x00097e                  _eMBASCIIStop
                  0x0066ac                  _eMBClose
                  0x0066ec                  _eMBDisable
                  0x0066ce                  _eMBEnable
                  0x006a7a                  _eMBFuncReadCoils
                  0x0075a6                  _eMBFuncReadDiscreteInputs
                  0x006044                  _eMBFuncReadHoldingRegister
                  0x007682                  _eMBFuncReadInputRegister
                  0x006110                  _eMBFuncReadWriteMultipleHoldingRegister
                  0x0077b0                  _eMBFuncReportSlaveID
                  0x006b58                  _eMBFuncWriteCoil
                  0x005f48                  _eMBFuncWriteHoldingRegister
                  0x006bea                  _eMBFuncWriteMultipleCoils
                  0x005fa0                  _eMBFuncWriteMultipleHoldingRegister
                  0x006532                  _eMBInit
                  0x006718                  _eMBPoll
                  0x00680c                  _eMBRTUInit
                  0x00689a                  _eMBRTUReceive
                  0x0068f8                  _eMBRTUSend
                  0x006874                  _eMBRTUStart
                  0x006888                  _eMBRTUStop
                  0x00415a                  _eMBRegCoilsCB
                  0x00437a                  _eMBRegDiscreteCB
                  0x003f92                  _eMBRegHoldingCB
                  0x003f18                  _eMBRegInputCB
                  0x0065ee                  _eMBRegisterCB
                  0x007750                  _eMBSetSlaveID
                  0x0018c8                  _exit
                  0x0016c4                  _fprintf
                  0x00394a                  _frexp
                  0x00394a                  _frexpl
                  0x0063ee                  _getBlinkyDebug
                  0x00438c                  _getLine
                  0x005590                  _instPortClearWriteReq
                  0x00550c                  _instPortInit
                  0x0055d0                  _instPortReadReg
                  0x00554c                  _instPortTxTask
                  0x0058bc                  _instPortWriteReg
                  0x0055ac                  _instSnapshotRxAvail
                  0x0040c6                  _isBitSet
                  0x001536                  _isalpha
                  0x00154a                  _isspace
                  0x003e6a                  _main
                  0x006fca                  _memErase
                  0x006e5a                  _memRead
                  0x006ee0                  _memWrite
                  0x0016d0                  _memcpy
                  0x0016de                  _memset
                  0x0045cc                  _menuBanner
                  0x0045f8                  _menuConfig
                  0x004694                  _menuHelp
                  0x0046c2                  _menuOpt0
                  0x0046e4                  _menuOpt1
                  0x004700                  _menuOpt2
                  0x004766                  _menuOpt3
                  0x004820                  _menuOpt4
                  0x0048b2                  _menuOpt5
                  0x0048f0                  _menuOpt6
                  0x004974                  _menuOpt7
                  0x0049b4                  _menuOpt8
                  0x0049be                  _menuOpt9
                  0x00448e                  _menuTask
                  0x006250                  _miscInit
                  0x006266                  _miscRegRead
                  0x006306                  _miscRegWrite
                  0x003e22                  _modBusTask
                  0x001000                  _paramBuff
                  0x007276                  _periphInit
                  0x007244                  _prveMBError2Exception
                  0x0008be                  _pwrBits
                  0x001892                  _raise
                  0x00526a                  _serClrFERR
                  0x0051f4                  _serClrOERR
                  0x0052c4                  _serClrPERR
                  0x005198                  _serClrXERR
                  0x0008a6                  _serEnblBits
                  0x004b12                  _serGetBaud
                  0x005088                  _serGetBreak
                  0x004cda                  _serGetByte
                  0x004c24                  _serGetConfig
                  0x005170                  _serGetErrFlag
                  0x005296                  _serGetFERR
                  0x00523c                  _serGetOERR
                  0x0052f0                  _serGetPERR
                  0x0051c4                  _serGetXERR
                  0x0049c8                  _serInit
                  0x0050aa                  _serIsRxFull
                  0x005146                  _serIsTxEmpty
                  0x00511c                  _serIsTxFull
                  0x004d12                  _serPutByte
                  0x004da0                  _serPutString
                  0x004e1a                  _serPutStringBool
                  0x0050f0                  _serRxAvailable
                  0x004e44                  _serRxFlush
                  0x004ac4                  _serSetBaud
                  0x004f30                  _serSetBreak
                  0x004b34                  _serSetConfig
                  0x004ee0                  _serTxFlush
                  0x0063c2                  _setBlinkyDebug
                  0x001880                  _signal
                  0x00442c                  _signon
                  0x0017f0                  _strtol
                  0x0016ec                  _strtoul
                  0x007046                  _tmrDelayMs
                  0x007028                  _tmrDelayTicks
                  0x0070ac                  _tmrDelayUs
                  0x00710e                  _tmrGetTicks
                  0x007000                  _tmrInit
                  0x007020                  _tmrTask
                  0x00155a                  _toupper
                  0x007836                  _usMBCRC16
                  0x006ca0                  _vMBPortSerialEnable
                  0x007808                  _vMBPortTimersDisable
                  0x0077fe                  _vMBPortTimersEnable
                  0x002154                  _vfprintf
                  0x000a40                  _xMBASCIIReceiveFSM
                  0x000be2                  _xMBASCIITimerT1SExpired
                  0x000b20                  _xMBASCIITransmitFSM
                  0x0078ac                  _xMBPortEventGet
                  0x007890                  _xMBPortEventInit
                  0x00789a                  _xMBPortEventPost
                  0x006d86                  _xMBPortSerialGetByte
                  0x006cc8                  _xMBPortSerialInit
                  0x006d78                  _xMBPortSerialPutByte
                  0x0077ce                  _xMBPortTimersInit
                  0x006962                  _xMBRTUReceiveFSM
                  0x006a2c                  _xMBRTUTimerT35Expired
                  0x0069d2                  _xMBRTUTransmitFSM
                  0x0071ec                  _xMBUtilGetBits
                  0x00714e                  _xMBUtilSetBits

Memory Configuration

Name             Origin             Length             Attributes
data             0x000800           0x004000           a !xr
FBOOT            0x801800           0x000002  
reset            0x000000           0x000004  
ivt              0x000004           0x0000fc  
program          0x000100           0x015680           xr
FSEC             0x015780           0x000002  
FBSLIM           0x015790           0x000002  
FSIGN            0x015794           0x000002  
FOSCSEL          0x015798           0x000002  
FOSC             0x01579c           0x000002  
FWDT             0x0157a0           0x000002  
FPOR             0x0157a4           0x000002  
FICD             0x0157a8           0x000002  
FDS              0x0157ac           0x000002  
FDEVOPT1         0x0157b0           0x000002  
*default*        0x000000           0xffffffff  

Linker script and memory map

LOAD build/default/production/_ext/1470100448/mbascii.o
LOAD build/default/production/_ext/833655638/mbfunccoils.o
LOAD build/default/production/_ext/833655638/mbfuncdiag.o
LOAD build/default/production/_ext/833655638/mbfuncdisc.o
LOAD build/default/production/_ext/833655638/mbfuncholding.o
LOAD build/default/production/_ext/833655638/mbfuncinput.o
LOAD build/default/production/_ext/833655638/mbfuncother.o
LOAD build/default/production/_ext/833655638/mbutils.o
LOAD build/default/production/_ext/1433339410/portevent.o
LOAD build/default/production/_ext/1433339410/portserial.o
LOAD build/default/production/_ext/1433339410/porttimer.o
LOAD build/default/production/_ext/1477781822/mbcrc.o
LOAD build/default/production/_ext/1477781822/mbrtu.o
LOAD build/default/production/_ext/1043210786/debug.o
LOAD build/default/production/_ext/1043210786/mb.o
LOAD build/default/production/_ext/1472/main.o
LOAD build/default/production/_ext/1472/mcc.o
LOAD build/default/production/_ext/1472/periph.o
LOAD build/default/production/_ext/1472/sys_timer.o
LOAD build/default/production/_ext/1472/misc.o
LOAD build/default/production/_ext/1472/buffer.o
LOAD build/default/production/_ext/1472/serial.o
LOAD build/default/production/_ext/1472/config.o
LOAD build/default/production/_ext/1472/flash_mem.o
LOAD build/default/production/_ext/1472/inst_port.o
LOAD build/default/production/_ext/1472/dig_io.o
                    0x0001                  __MPLAB_BUILD = 0x1
LOAD pPIC24Fxxx
LOAD c:/program files (x86)/microchip/xc16/v1.25/bin/bin/../../lib\libfx-elf.a
                    0x801800                  __FBOOT = 0x801800
                    0x15780                  __FSEC = 0x15780
                    0x15790                  __FBSLIM = 0x15790
                    0x15794                  __FSIGN = 0x15794
                    0x15798                  __FOSCSEL = 0x15798
                    0x1579c                  __FOSC = 0x1579c
                    0x157a0                  __FWDT = 0x157a0
                    0x157a4                  __FPOR = 0x157a4
                    0x157a8                  __FICD = 0x157a8
                    0x157ac                  __FDS = 0x157ac
                    0x157b0                  __FDEVOPT1 = 0x157b0
                    0x0100                  __CODE_BASE = 0x100
                    0x15680                  __CODE_LENGTH = 0x15680
                    0x0004                  __IVT_BASE = 0x4
                    0x0800                  __DATA_BASE = 0x800
                    0x4000                  __DATA_LENGTH = 0x4000

.reset            0x000000          0x4
                  0x000000          0x2 SHORT 0x1400 ABSOLUTE (__reset)
                  0x000001          0x2 SHORT 0x4
                  0x000002          0x2 SHORT 0x0 ((ABSOLUTE (__reset) >> 0x10) & 0x7f)
                  0x000003          0x2 SHORT 0x0

.text             0x001400       0x2a22
 *(.init)
 .init            0x001400         0x38 c:/program files (x86)/microchip/xc16/v1.25/bin/bin/../../lib\libpic30-elf.a(crt0_extended.o)
                  0x001400                  __resetPRI
                  0x001400                  __reset
                  0x00142c                  __psv_init
 .init            0x001438         0x9a c:/program files (x86)/microchip/xc16/v1.25/bin/bin/../../lib\libpic30-elf.a(data_init_extended.o)
                  0x001438                  __data_init
                  0x001438                  __data_init_extended
 *(.user_init)
 *(.handle)
 .handle          0x0014d2         0x60 jump_table
 *(.isr*)
 .isr             0x001532          0x4 default_isr
                  0x001532                  __DefaultInterrupt
 *(.libc)
 .libc            0x001536         0x14 c:/program files (x86)/microchip/xc16/v1.25/bin/bin/../../lib\libc-elf.a(isalpha.eso)
                  0x001536                  _isalpha
 .libc            0x00154a         0x10 c:/program files (x86)/microchip/xc16/v1.25/bin/bin/../../lib\libc-elf.a(isspace.eso)
                  0x00154a                  _isspace
 .libc            0x00155a          0xe c:/program files (x86)/microchip/xc16/v1.25/bin/bin/../../lib\libc-elf.a(toupper.eso)
                  0x00155a                  _toupper
 .libc            0x001568         0x10 c:/program files (x86)/microchip/xc16/v1.25/bin/bin/../../lib\libpic30-elf.a(_exit.eo)
                  0x001568                  __exit
 .libc            0x001578         0x5c c:/program files (x86)/microchip/xc16/v1.25/bin/bin/../../lib\libpic30-elf.a(write.eo)
                  0x001578                  _write
 *(.libm)
 *(.libdsp)
 *(.lib*)
 .libm.divsi3     0x0015d4         0x1e c:/program files (x86)/microchip/xc16/v1.25/bin/bin/../../lib\libm-elf.a(divsi3.eo)
                  0x0015d4                  ___divsi3
 .libm.udivsi3    0x0015f2         0x20 c:/program files (x86)/microchip/xc16/v1.25/bin/bin/../../lib\libm-elf.a(udivsi3.eo)
                  0x0015f2                  ___udivsi3
 .libc.atoi       0x001612         0x3e c:/program files (x86)/microchip/xc16/v1.25/bin/bin/../../lib\libc-elf.a(atoi.eo)
                  0x001612                  _atoi
 .libc.atol       0x001650         0x56 c:/program files (x86)/microchip/xc16/v1.25/bin/bin/../../lib\libc-elf.a(atol.eo)
                  0x001650                  _atol
 .libc._fassert
                  0x0016a6         0x1e c:/program files (x86)/microchip/xc16/v1.25/bin/bin/../../lib\libc-elf.a(fassert.eo)
                  0x0016a6                  __fassert
 .libc.fprintf    0x0016c4          0xc c:/program files (x86)/microchip/xc16/v1.25/bin/bin/../../lib\libc-elf.a(fprintf.eo)
                  0x0016c4                  _fprintf
 .libc.memcpy     0x0016d0          0xe c:/program files (x86)/microchip/xc16/v1.25/bin/bin/../../lib\libc-elf.a(memcpy.eo)
                  0x0016d0                  _memcpy
 .libc.memset     0x0016de          0xe c:/program files (x86)/microchip/xc16/v1.25/bin/bin/../../lib\libc-elf.a(memset.eo)
                  0x0016de                  _memset
 .libc.strtoul    0x0016ec        0x104 c:/program files (x86)/microchip/xc16/v1.25/bin/bin/../../lib\libc-elf.a(strtol.eo)
                  0x0016ec                  _strtoul
 .libc.strtol     0x0017f0         0x90 c:/program files (x86)/microchip/xc16/v1.25/bin/bin/../../lib\libc-elf.a(strtol.eo)
                  0x0017f0                  _strtol
 .libc.signal     0x001880         0x12 c:/program files (x86)/microchip/xc16/v1.25/bin/bin/../../lib\libc-elf.a(signal.eo)
                  0x001880                  _signal
 .libc.raise      0x001892         0x2e c:/program files (x86)/microchip/xc16/v1.25/bin/bin/../../lib\libc-elf.a(signal.eo)
                  0x001892                  _raise
 .libc.abort      0x0018c0          0x8 c:/program files (x86)/microchip/xc16/v1.25/bin/bin/../../lib\libc-elf.a(signal.eo)
                  0x0018c0                  _abort
 .libc.exit       0x0018c8          0x8 c:/program files (x86)/microchip/xc16/v1.25/bin/bin/../../lib\libc-elf.a(exit.elo)
                  0x0018c8                  _exit
 .libc._cleanup
                  0x0018d0          0x2 c:/program files (x86)/microchip/xc16/v1.25/bin/bin/../../lib\libc-elf.a(stdclean.elo)
                  0x0018d0                  __cleanup
 .libc._sprintf_cdnopsuxX
                  0x0018d2         0x2c c:/program files (x86)/microchip/xc16/v1.25/bin/bin/../../lib\libc-elf.a(sprintf_cdnopsuxX.XXeo)
                  0x0018d2                  __sprintf_cdnopsuxX
 .libc.sputc      0x0018fe         0x12 c:/program files (x86)/microchip/xc16/v1.25/bin/bin/../../lib\libc-elf.a(doprnt_cdnopsuxX.XXeo)
 .libc._vfprintf_cdnopsuxX
                  0x001910        0x6b4 c:/program files (x86)/microchip/xc16/v1.25/bin/bin/../../lib\libc-elf.a(doprnt_cdnopsuxX.XXeo)
                  0x001910                  __vfprintf_cdnopsuxX
 .libc.fround     0x001fc4         0xba c:/program files (x86)/microchip/xc16/v1.25/bin/bin/../../lib\libc-elf.a(doprnt.eo)
 .libc.scale      0x00207e         0xc4 c:/program files (x86)/microchip/xc16/v1.25/bin/bin/../../lib\libc-elf.a(doprnt.eo)
 .libc.sputc      0x002142         0x12 c:/program files (x86)/microchip/xc16/v1.25/bin/bin/../../lib\libc-elf.a(doprnt.eo)
 .libc.vfprintf
                  0x002154       0x1352 c:/program files (x86)/microchip/xc16/v1.25/bin/bin/../../lib\libc-elf.a(doprnt.eo)
                  0x002154                  _vfprintf
 .libc.fputc      0x0034a6         0x86 c:/program files (x86)/microchip/xc16/v1.25/bin/bin/../../lib\libc-elf.a(fputc.eo)
                  0x0034a6                  _fputc
 .libc._flsbuf    0x00352c         0x7e c:/program files (x86)/microchip/xc16/v1.25/bin/bin/../../lib\libc-elf.a(flsbuf.eo)
                  0x00352c                  __flsbuf
 .libc.dowrite    0x0035aa          0x4 c:/program files (x86)/microchip/xc16/v1.25/bin/bin/../../lib\libpic30-elf.a(write.eo)
 .libm.adddf3     0x0035ae         0xfa c:/program files (x86)/microchip/xc16/v1.25/bin/bin/../../lib\libm-elf.a(adddf3.eo)
                  0x0035ae                  ___adddf3
 .libm.eqdf2      0x0036a8          0xa c:/program files (x86)/microchip/xc16/v1.25/bin/bin/../../lib\libm-elf.a(deqltle.eo)
                  0x0036a8                  ___eqdf2
                  0x0036a8                  ___ltdf2
                  0x0036a8                  ___ledf2
 .libm.gtdf2      0x0036b2          0xa c:/program files (x86)/microchip/xc16/v1.25/bin/bin/../../lib\libm-elf.a(dgtge.eo)
                  0x0036b2                  ___gtdf2
                  0x0036b2                  ___gedf2
 .libm.divdf3     0x0036bc         0xb4 c:/program files (x86)/microchip/xc16/v1.25/bin/bin/../../lib\libm-elf.a(divdf3.eo)
                  0x0036bc                  ___divdf3
 .libm.nedf2      0x003770          0xa c:/program files (x86)/microchip/xc16/v1.25/bin/bin/../../lib\libm-elf.a(dne.eo)
                  0x003770                  ___nedf2
 .libm.dpack      0x00377a         0x58 c:/program files (x86)/microchip/xc16/v1.25/bin/bin/../../lib\libm-elf.a(dpack.eo)
                  0x00377a                  __dpack
 .libm.dunpack2
                  0x0037d2         0x32 c:/program files (x86)/microchip/xc16/v1.25/bin/bin/../../lib\libm-elf.a(dunpack2.eo)
                  0x0037d2                  __dunpack2
                  0x0037f4                  __dreturnNaN
                  0x0037fa                  __dunpack2exit
 .libm.extendsfdf2
                  0x003804         0x3e c:/program files (x86)/microchip/xc16/v1.25/bin/bin/../../lib\libm-elf.a(extendsfdf.eo)
                  0x003804                  ___extendsfdf2
 .libm.fixunsdfdi
                  0x003842         0x62 c:/program files (x86)/microchip/xc16/v1.25/bin/bin/../../lib\libm-elf.a(fixunsdfdi.eo)
                  0x003842                  ___fixunsdfdi
 .libm.fixunsdfsi
                  0x0038a4         0x4c c:/program files (x86)/microchip/xc16/v1.25/bin/bin/../../lib\libm-elf.a(fixunsdfsi.eo)
                  0x0038a4                  ___fixunsdfsi
 .libm.floatundidf
                  0x0038f0         0x56 c:/program files (x86)/microchip/xc16/v1.25/bin/bin/../../lib\libm-elf.a(floatundidf.eo)
                  0x0038f0                  ___floatundidf
 .libm.floatunsidf
                  0x003946          0x4 c:/program files (x86)/microchip/xc16/v1.25/bin/bin/../../lib\libm-elf.a(floatunsidf.eo)
                  0x003946                  ___floatunsidf
 .libm.frexp      0x00394a         0x3a c:/program files (x86)/microchip/xc16/v1.25/bin/bin/../../lib\libm-elf.a(frexp.eo)
                  0x00394a                  _frexp
                  0x00394a                  _frexpl
 .libm.funpack    0x003984         0x2a c:/program files (x86)/microchip/xc16/v1.25/bin/bin/../../lib\libm-elf.a(funpack.eo)
                  0x003984                  __funpack
 .libm.muldf3     0x0039ae         0xea c:/program files (x86)/microchip/xc16/v1.25/bin/bin/../../lib\libm-elf.a(muldf3.eo)
                  0x0039ae                  ___muldf3
 .libm.subdf3     0x003a98          0x4 c:/program files (x86)/microchip/xc16/v1.25/bin/bin/../../lib\libm-elf.a(subdf3.eo)
                  0x003a98                  ___subdf3
 .libm.mulsi3     0x003a9c          0xc c:/program files (x86)/microchip/xc16/v1.25/bin/bin/../../lib\libm-elf.a(mulsi3.eo)
                  0x003a9c                  ___mulp32peds3
                  0x003a9c                  ___mulsi3
                  0x003a9c                  ___mulp32eds3
 .libm.__PplusBdi
                  0x003aa8         0x26 c:/program files (x86)/microchip/xc16/v1.25/bin/bin/../../lib\libm-elf.a(divmoddi3.eo)
 .libm.__PminusBdi
                  0x003ace         0x26 c:/program files (x86)/microchip/xc16/v1.25/bin/bin/../../lib\libm-elf.a(divmoddi3.eo)
 .libm.__udivmoddi3
                  0x003af4         0xe6 c:/program files (x86)/microchip/xc16/v1.25/bin/bin/../../lib\libm-elf.a(divmoddi3.eo)
                  0x003af4                  ___udivmoddi3
 .libm.__udivdi3
                  0x003bda          0xe c:/program files (x86)/microchip/xc16/v1.25/bin/bin/../../lib\libm-elf.a(divmoddi3.eo)
                  0x003bda                  ___udivdi3
 .libm.__umoddi3
                  0x003be8          0x8 c:/program files (x86)/microchip/xc16/v1.25/bin/bin/../../lib\libm-elf.a(divmoddi3.eo)
                  0x003be8                  ___umoddi3
 .libm.__divdi3
                  0x003bf0         0x60 c:/program files (x86)/microchip/xc16/v1.25/bin/bin/../../lib\libm-elf.a(divmoddi3.eo)
                  0x003bf0                  ___divdi3
 .libm.__moddi3
                  0x003c50         0x5c c:/program files (x86)/microchip/xc16/v1.25/bin/bin/../../lib\libm-elf.a(divmoddi3.eo)
                  0x003c50                  ___moddi3
 .libm.__muldi3
                  0x003cac         0x52 c:/program files (x86)/microchip/xc16/v1.25/bin/bin/../../lib\libm-elf.a(muldi3.eo)
                  0x003cac                  ___muldi3
 .libm.dcompare
                  0x003cfe         0x52 c:/program files (x86)/microchip/xc16/v1.25/bin/bin/../../lib\libm-elf.a(dcompare.eo)
                  0x003cfe                  __dcompare
 .libm.dPropagateNaN
                  0x003d50         0x1c c:/program files (x86)/microchip/xc16/v1.25/bin/bin/../../lib\libm-elf.a(dpropagateNaN.eo)
                  0x003d50                  __dPropagateNaN
 .libm.dtype      0x003d6c         0x24 c:/program files (x86)/microchip/xc16/v1.25/bin/bin/../../lib\libm-elf.a(dtype.eo)
                  0x003d6c                  __dtype
 .libm.dunpack    0x003d90         0x4e c:/program files (x86)/microchip/xc16/v1.25/bin/bin/../../lib\libm-elf.a(dunpack.eo)
                  0x003d90                  __dunpack
 .libm.umuldi3    0x003dde         0x44 c:/program files (x86)/microchip/xc16/v1.25/bin/bin/../../lib\libm-elf.a(umuldi3.eo)
                  0x003dde                  ___umuldi3

usercode
 *(usercode)

__FBOOT
 *(__FBOOT.sec*)

__FSEC
 *(__FSEC.sec*)

__FBSLIM
 *(__FBSLIM.sec*)

__FSIGN
 *(__FSIGN.sec*)

__FOSCSEL
 *(__FOSCSEL.sec*)

__FOSC
 *(__FOSC.sec*)

__FWDT
 *(__FWDT.sec*)

__FPOR
 *(__FPOR.sec*)

__FICD
 *(__FICD.sec*)

__FDS
 *(__FDS.sec*)

__FDEVOPT1
 *(__FDEVOPT1.sec*)

.comment
 *(.comment)

.debug_info       0x000000       0xe987
 *(.debug_info)
 .debug_info      0x000000        0x845 build/default/production/_ext/1470100448/mbascii.o
 .debug_info      0x000845        0x549 build/default/production/_ext/833655638/mbfunccoils.o
 .debug_info      0x000d8e        0x3f5 build/default/production/_ext/833655638/mbfuncdisc.o
 .debug_info      0x001183        0x610 build/default/production/_ext/833655638/mbfuncholding.o
 .debug_info      0x001793        0x3df build/default/production/_ext/833655638/mbfuncinput.o
 .debug_info      0x001b72        0x491 build/default/production/_ext/833655638/mbfuncother.o
 .debug_info      0x002003        0x4bb build/default/production/_ext/833655638/mbutils.o
 .debug_info      0x0024be        0x2cb build/default/production/_ext/1433339410/portevent.o
 .debug_info      0x002789        0xd24 build/default/production/_ext/1433339410/portserial.o
 .debug_info      0x0034ad        0x99b build/default/production/_ext/1433339410/porttimer.o
 .debug_info      0x003e48        0x240 build/default/production/_ext/1477781822/mbcrc.o
 .debug_info      0x004088        0x6df build/default/production/_ext/1477781822/mbrtu.o
 .debug_info      0x004767        0x15b build/default/production/_ext/1043210786/debug.o
 .debug_info      0x0048c2        0x9a7 build/default/production/_ext/1043210786/mb.o
 .debug_info      0x005269       0x1182 build/default/production/_ext/1472/main.o
 .debug_info      0x0063eb        0x21e build/default/production/_ext/1472/mcc.o
 .debug_info      0x006609       0x1c91 build/default/production/_ext/1472/periph.o
 .debug_info      0x00829a        0xbb8 build/default/production/_ext/1472/sys_timer.o
 .debug_info      0x008e52        0x6ae build/default/production/_ext/1472/misc.o
 .debug_info      0x009500        0x2dd build/default/production/_ext/1472/buffer.o
 .debug_info      0x0097dd       0x388b build/default/production/_ext/1472/serial.o
 .debug_info      0x00d068        0x312 build/default/production/_ext/1472/config.o
 .debug_info      0x00d37a        0x7f1 build/default/production/_ext/1472/flash_mem.o
 .debug_info      0x00db6b        0x589 build/default/production/_ext/1472/inst_port.o
 .debug_info      0x00e0f4        0x893 build/default/production/_ext/1472/dig_io.o
 *(.gnu.linkonce.wi.*)

.debug_abbrev     0x000000       0x1a76
 *(.debug_abbrev)
 .debug_abbrev    0x000000        0x174 build/default/production/_ext/1470100448/mbascii.o
 .debug_abbrev    0x000174         0xc9 build/default/production/_ext/833655638/mbfunccoils.o
 .debug_abbrev    0x00023d          0x1 build/default/production/_ext/833655638/mbfuncdiag.o
 .debug_abbrev    0x00023e         0x80 build/default/production/_ext/833655638/mbfuncdisc.o
 .debug_abbrev    0x0002be         0xa8 build/default/production/_ext/833655638/mbfuncholding.o
 .debug_abbrev    0x000366         0x80 build/default/production/_ext/833655638/mbfuncinput.o
 .debug_abbrev    0x0003e6         0xaa build/default/production/_ext/833655638/mbfuncother.o
 .debug_abbrev    0x000490         0xce build/default/production/_ext/833655638/mbutils.o
 .debug_abbrev    0x00055e         0xa8 build/default/production/_ext/1433339410/portevent.o
 .debug_abbrev    0x000606        0x1aa build/default/production/_ext/1433339410/portserial.o
 .debug_abbrev    0x0007b0        0x14c build/default/production/_ext/1433339410/porttimer.o
 .debug_abbrev    0x0008fc         0x85 build/default/production/_ext/1477781822/mbcrc.o
 .debug_abbrev    0x000981        0x12e build/default/production/_ext/1477781822/mbrtu.o
 .debug_abbrev    0x000aaf         0x1f build/default/production/_ext/1043210786/debug.o
 .debug_abbrev    0x000ace        0x170 build/default/production/_ext/1043210786/mb.o
 .debug_abbrev    0x000c3e        0x251 build/default/production/_ext/1472/main.o
 .debug_abbrev    0x000e8f         0x6a build/default/production/_ext/1472/mcc.o
 .debug_abbrev    0x000ef9         0xb6 build/default/production/_ext/1472/periph.o
 .debug_abbrev    0x000faf        0x16a build/default/production/_ext/1472/sys_timer.o
 .debug_abbrev    0x001119        0x168 build/default/production/_ext/1472/misc.o
 .debug_abbrev    0x001281         0xbd build/default/production/_ext/1472/buffer.o
 .debug_abbrev    0x00133e        0x22f build/default/production/_ext/1472/serial.o
 .debug_abbrev    0x00156d         0xbd build/default/production/_ext/1472/config.o
 .debug_abbrev    0x00162a        0x19e build/default/production/_ext/1472/flash_mem.o
 .debug_abbrev    0x0017c8        0x12e build/default/production/_ext/1472/inst_port.o
 .debug_abbrev    0x0018f6        0x180 build/default/production/_ext/1472/dig_io.o

.debug_line       0x000000       0x5a5a
 *(.debug_line)
 .debug_line      0x000000        0x65b build/default/production/_ext/1470100448/mbascii.o
 .debug_line      0x00065b        0x306 build/default/production/_ext/833655638/mbfunccoils.o
 .debug_line      0x000961         0x24 build/default/production/_ext/833655638/mbfuncdiag.o
 .debug_line      0x000985        0x169 build/default/production/_ext/833655638/mbfuncdisc.o
 .debug_line      0x000aee        0x3a5 build/default/production/_ext/833655638/mbfuncholding.o
 .debug_line      0x000e93        0x15a build/default/production/_ext/833655638/mbfuncinput.o
 .debug_line      0x000fed        0x177 build/default/production/_ext/833655638/mbfuncother.o
 .debug_line      0x001164        0x208 build/default/production/_ext/833655638/mbutils.o
 .debug_line      0x00136c        0x119 build/default/production/_ext/1433339410/portevent.o
 .debug_line      0x001485        0x399 build/default/production/_ext/1433339410/portserial.o
 .debug_line      0x00181e        0x1cb build/default/production/_ext/1433339410/porttimer.o
 .debug_line      0x0019e9         0xb9 build/default/production/_ext/1477781822/mbcrc.o
 .debug_line      0x001aa2        0x441 build/default/production/_ext/1477781822/mbrtu.o
 .debug_line      0x001ee3         0x24 build/default/production/_ext/1043210786/debug.o
 .debug_line      0x001f07        0x48f build/default/production/_ext/1043210786/mb.o
 .debug_line      0x002396        0xe8b build/default/production/_ext/1472/main.o
 .debug_line      0x003221        0x148 build/default/production/_ext/1472/mcc.o
 .debug_line      0x003369        0x303 build/default/production/_ext/1472/periph.o
 .debug_line      0x00366c        0x2b1 build/default/production/_ext/1472/sys_timer.o
 .debug_line      0x00391d        0x413 build/default/production/_ext/1472/misc.o
 .debug_line      0x003d30        0x17c build/default/production/_ext/1472/buffer.o
 .debug_line      0x003eac        0xe39 build/default/production/_ext/1472/serial.o
 .debug_line      0x004ce5        0x1c9 build/default/production/_ext/1472/config.o
 .debug_line      0x004eae        0x28d build/default/production/_ext/1472/flash_mem.o
 .debug_line      0x00513b        0x56d build/default/production/_ext/1472/inst_port.o
 .debug_line      0x0056a8        0x3b2 build/default/production/_ext/1472/dig_io.o

.debug_frame      0x000000        0xdac
 *(.debug_frame)
 .debug_frame     0x000000         0xc4 build/default/production/_ext/1470100448/mbascii.o
 .debug_frame     0x0000c4         0x44 build/default/production/_ext/833655638/mbfunccoils.o
 .debug_frame     0x000108         0x24 build/default/production/_ext/833655638/mbfuncdisc.o
 .debug_frame     0x00012c         0x54 build/default/production/_ext/833655638/mbfuncholding.o
 .debug_frame     0x000180         0x24 build/default/production/_ext/833655638/mbfuncinput.o
 .debug_frame     0x0001a4         0x34 build/default/production/_ext/833655638/mbfuncother.o
 .debug_frame     0x0001d8         0x44 build/default/production/_ext/833655638/mbutils.o
 .debug_frame     0x00021c         0x44 build/default/production/_ext/1433339410/portevent.o
 .debug_frame     0x000260         0x94 build/default/production/_ext/1433339410/portserial.o
 .debug_frame     0x0002f4         0x54 build/default/production/_ext/1433339410/porttimer.o
 .debug_frame     0x000348         0x24 build/default/production/_ext/1477781822/mbcrc.o
 .debug_frame     0x00036c         0x94 build/default/production/_ext/1477781822/mbrtu.o
 .debug_frame     0x000400         0x74 build/default/production/_ext/1043210786/mb.o
 .debug_frame     0x000474        0x330 build/default/production/_ext/1472/main.o
 .debug_frame     0x0007a4         0x34 build/default/production/_ext/1472/mcc.o
 .debug_frame     0x0007d8         0x24 build/default/production/_ext/1472/periph.o
 .debug_frame     0x0007fc         0x94 build/default/production/_ext/1472/sys_timer.o
 .debug_frame     0x000890         0x74 build/default/production/_ext/1472/misc.o
 .debug_frame     0x000904         0x54 build/default/production/_ext/1472/buffer.o
 .debug_frame     0x000958        0x274 build/default/production/_ext/1472/serial.o
 .debug_frame     0x000bcc         0x64 build/default/production/_ext/1472/config.o
 .debug_frame     0x000c30         0x44 build/default/production/_ext/1472/flash_mem.o
 .debug_frame     0x000c74         0x94 build/default/production/_ext/1472/inst_port.o
 .debug_frame     0x000d08         0xa4 build/default/production/_ext/1472/dig_io.o

.debug_str        0x000000        0x5c5
 *(.debug_str)
 .debug_str       0x000000         0x3a build/default/production/_ext/1470100448/mbascii.o
 .debug_str       0x00003a         0x29 build/default/production/_ext/833655638/mbfunccoils.o
 .debug_str       0x000063         0x46 build/default/production/_ext/833655638/mbfuncholding.o
 .debug_str       0x0000a9         0x38 build/default/production/_ext/833655638/mbutils.o
 .debug_str       0x0000e1         0x65 build/default/production/_ext/1433339410/portserial.o
 .debug_str       0x000146         0x3c build/default/production/_ext/1433339410/porttimer.o
 .debug_str       0x000182         0x33 build/default/production/_ext/1477781822/mbrtu.o
 .debug_str       0x0001b5         0x6c build/default/production/_ext/1043210786/mb.o
 .debug_str       0x000221         0x4d build/default/production/_ext/1472/main.o
 .debug_str       0x00026e         0x1c build/default/production/_ext/1472/mcc.o
 .debug_str       0x00028a         0xd6 build/default/production/_ext/1472/periph.o
 .debug_str       0x000360         0x2f build/default/production/_ext/1472/sys_timer.o
 .debug_str       0x00038f         0x28 build/default/production/_ext/1472/misc.o
 .debug_str       0x0003b7        0x1cd build/default/production/_ext/1472/serial.o
 .debug_str       0x000584          0x7 build/default/production/_ext/1472/config.o
 .debug_str       0x00058b         0x15 build/default/production/_ext/1472/flash_mem.o
 .debug_str       0x0005a0         0x10 build/default/production/_ext/1472/inst_port.o
 .debug_str       0x0005b0         0x15 build/default/production/_ext/1472/dig_io.o

.debug_loc
 *(.debug_loc)

.debug_macinfo
 *(.debug_macinfo)

.debug_pubnames
                  0x000000        0xdb7
 *(.debug_pubnames)
 .debug_pubnames
                  0x000000         0xb6 build/default/production/_ext/1470100448/mbascii.o
 .debug_pubnames
                  0x0000b6         0x5a build/default/production/_ext/833655638/mbfunccoils.o
 .debug_pubnames
                  0x000110         0x30 build/default/production/_ext/833655638/mbfuncdisc.o
 .debug_pubnames
                  0x000140         0xa5 build/default/production/_ext/833655638/mbfuncholding.o
 .debug_pubnames
                  0x0001e5         0x2f build/default/production/_ext/833655638/mbfuncinput.o
 .debug_pubnames
                  0x000214         0x3d build/default/production/_ext/833655638/mbfuncother.o
 .debug_pubnames
                  0x000251         0x52 build/default/production/_ext/833655638/mbutils.o
 .debug_pubnames
                  0x0002a3         0x50 build/default/production/_ext/1433339410/portevent.o
 .debug_pubnames
                  0x0002f3         0xc9 build/default/production/_ext/1433339410/portserial.o
 .debug_pubnames
                  0x0003bc         0x6a build/default/production/_ext/1433339410/porttimer.o
 .debug_pubnames
                  0x000426         0x20 build/default/production/_ext/1477781822/mbcrc.o
 .debug_pubnames
                  0x000446         0xb3 build/default/production/_ext/1477781822/mbrtu.o
 .debug_pubnames
                  0x0004f9         0xf8 build/default/production/_ext/1043210786/mb.o
 .debug_pubnames
                  0x0005f1        0x17f build/default/production/_ext/1472/main.o
 .debug_pubnames
                  0x000770         0x42 build/default/production/_ext/1472/mcc.o
 .debug_pubnames
                  0x0007b2         0x21 build/default/production/_ext/1472/periph.o
 .debug_pubnames
                  0x0007d3         0x7b build/default/production/_ext/1472/sys_timer.o
 .debug_pubnames
                  0x00084e         0x75 build/default/production/_ext/1472/misc.o
 .debug_pubnames
                  0x0008c3         0x41 build/default/production/_ext/1472/buffer.o
 .debug_pubnames
                  0x000904        0x2bf build/default/production/_ext/1472/serial.o
 .debug_pubnames
                  0x000bc3         0x5c build/default/production/_ext/1472/config.o
 .debug_pubnames
                  0x000c1f         0x46 build/default/production/_ext/1472/flash_mem.o
 .debug_pubnames
                  0x000c65         0x91 build/default/production/_ext/1472/inst_port.o
 .debug_pubnames
                  0x000cf6         0xc1 build/default/production/_ext/1472/dig_io.o

.debug_ranges
 *(.debug_ranges)

.debug_aranges    0x000000        0x240
 *(.debug_aranges)
 .debug_aranges
                  0x000000         0x18 build/default/production/_ext/1470100448/mbascii.o
 .debug_aranges
                  0x000018         0x18 build/default/production/_ext/833655638/mbfunccoils.o
 .debug_aranges
                  0x000030         0x18 build/default/production/_ext/833655638/mbfuncdisc.o
 .debug_aranges
                  0x000048         0x18 build/default/production/_ext/833655638/mbfuncholding.o
 .debug_aranges
                  0x000060         0x18 build/default/production/_ext/833655638/mbfuncinput.o
 .debug_aranges
                  0x000078         0x18 build/default/production/_ext/833655638/mbfuncother.o
 .debug_aranges
                  0x000090         0x18 build/default/production/_ext/833655638/mbutils.o
 .debug_aranges
                  0x0000a8         0x18 build/default/production/_ext/1433339410/portevent.o
 .debug_aranges
                  0x0000c0         0x18 build/default/production/_ext/1433339410/portserial.o
 .debug_aranges
                  0x0000d8         0x18 build/default/production/_ext/1433339410/porttimer.o
 .debug_aranges
                  0x0000f0         0x18 build/default/production/_ext/1477781822/mbcrc.o
 .debug_aranges
                  0x000108         0x18 build/default/production/_ext/1477781822/mbrtu.o
 .debug_aranges
                  0x000120         0x18 build/default/production/_ext/1043210786/mb.o
 .debug_aranges
                  0x000138         0x18 build/default/production/_ext/1472/main.o
 .debug_aranges
                  0x000150         0x18 build/default/production/_ext/1472/mcc.o
 .debug_aranges
                  0x000168         0x18 build/default/production/_ext/1472/periph.o
 .debug_aranges
                  0x000180         0x18 build/default/production/_ext/1472/sys_timer.o
 .debug_aranges
                  0x000198         0x18 build/default/production/_ext/1472/misc.o
 .debug_aranges
                  0x0001b0         0x18 build/default/production/_ext/1472/buffer.o
 .debug_aranges
                  0x0001c8         0x18 build/default/production/_ext/1472/serial.o
 .debug_aranges
                  0x0001e0         0x18 build/default/production/_ext/1472/config.o
 .debug_aranges
                  0x0001f8         0x18 build/default/production/_ext/1472/flash_mem.o
 .debug_aranges
                  0x000210         0x18 build/default/production/_ext/1472/inst_port.o
 .debug_aranges
                  0x000228         0x18 build/default/production/_ext/1472/dig_io.o

.ivt              0x000004         0xfc
                  0x000004          0x4 LONG 0x1532 DEFINED (__OscillatorFail)?ABSOLUTE (__OscillatorFail):ABSOLUTE (__DefaultInterrupt)
                  0x000006          0x4 LONG 0x1532 DEFINED (__AddressError)?ABSOLUTE (__AddressError):ABSOLUTE (__DefaultInterrupt)
                  0x000008          0x4 LONG 0x1532 DEFINED (__GeneralHardError)?ABSOLUTE (__GeneralHardError):ABSOLUTE (__DefaultInterrupt)
                  0x00000a          0x4 LONG 0x1532 DEFINED (__StackError)?ABSOLUTE (__StackError):ABSOLUTE (__DefaultInterrupt)
                  0x00000c          0x4 LONG 0x1532 DEFINED (__MathError)?ABSOLUTE (__MathError):ABSOLUTE (__DefaultInterrupt)
                  0x00000e          0x4 LONG 0x1532 DEFINED (__ReservedTrap5)?ABSOLUTE (__ReservedTrap5):ABSOLUTE (__DefaultInterrupt)
                  0x000010          0x4 LONG 0x1532 DEFINED (__GeneralSoftError)?ABSOLUTE (__GeneralSoftError):ABSOLUTE (__DefaultInterrupt)
                  0x000012          0x4 LONG 0x1532 DEFINED (__ReservedTrap7)?ABSOLUTE (__ReservedTrap7):ABSOLUTE (__DefaultInterrupt)
                  0x000014          0x4 LONG 0x1532 DEFINED (__INT0Interrupt)?ABSOLUTE (__INT0Interrupt):ABSOLUTE (__DefaultInterrupt)
                  0x000016          0x4 LONG 0x1532 DEFINED (__IC1Interrupt)?ABSOLUTE (__IC1Interrupt):ABSOLUTE (__DefaultInterrupt)
                  0x000018          0x4 LONG 0x1532 DEFINED (__OC1Interrupt)?ABSOLUTE (__OC1Interrupt):ABSOLUTE (__DefaultInterrupt)
                  0x00001a          0x4 LONG 0x7816 DEFINED (__T1Interrupt)?ABSOLUTE (__T1Interrupt):ABSOLUTE (__DefaultInterrupt)
                  0x00001c          0x4 LONG 0x1532 DEFINED (__DMA0Interrupt)?ABSOLUTE (__DMA0Interrupt):ABSOLUTE (__DefaultInterrupt)
                  0x00001e          0x4 LONG 0x1532 DEFINED (__IC2Interrupt)?ABSOLUTE (__IC2Interrupt):ABSOLUTE (__DefaultInterrupt)
                  0x000020          0x4 LONG 0x1532 DEFINED (__OC2Interrupt)?ABSOLUTE (__OC2Interrupt):ABSOLUTE (__DefaultInterrupt)
                  0x000022          0x4 LONG 0x713a DEFINED (__T2Interrupt)?ABSOLUTE (__T2Interrupt):ABSOLUTE (__DefaultInterrupt)
                  0x000024          0x4 LONG 0x1532 DEFINED (__T3Interrupt)?ABSOLUTE (__T3Interrupt):ABSOLUTE (__DefaultInterrupt)
                  0x000026          0x4 LONG 0x1532 DEFINED (__SPI1Interrupt)?ABSOLUTE (__SPI1Interrupt):ABSOLUTE (__DefaultInterrupt)
                  0x000028          0x4 LONG 0x1532 DEFINED (__SPI1TXInterrupt)?ABSOLUTE (__SPI1TXInterrupt):ABSOLUTE (__DefaultInterrupt)
                  0x00002a          0x4 LONG 0x5348 DEFINED (__U1RXInterrupt)?ABSOLUTE (__U1RXInterrupt):ABSOLUTE (__DefaultInterrupt)
                  0x00002c          0x4 LONG 0x5340 DEFINED (__U1TXInterrupt)?ABSOLUTE (__U1TXInterrupt):ABSOLUTE (__DefaultInterrupt)
                  0x00002e          0x4 LONG 0x1532 DEFINED (__ADC1Interrupt)?ABSOLUTE (__ADC1Interrupt):ABSOLUTE (__DefaultInterrupt)
                  0x000030          0x4 LONG 0x1532 DEFINED (__DMA1Interrupt)?ABSOLUTE (__DMA1Interrupt):ABSOLUTE (__DefaultInterrupt)
                  0x000032          0x4 LONG 0x1532 DEFINED (__NVMInterrupt)?ABSOLUTE (__NVMInterrupt):ABSOLUTE (__DefaultInterrupt)
                  0x000034          0x4 LONG 0x1532 DEFINED (__SI2C1Interrupt)?ABSOLUTE (__SI2C1Interrupt):ABSOLUTE (__DefaultInterrupt)
                  0x000036          0x4 LONG 0x1532 DEFINED (__MI2C1Interrupt)?ABSOLUTE (__MI2C1Interrupt):ABSOLUTE (__DefaultInterrupt)
                  0x000038          0x4 LONG 0x1532 DEFINED (__CompInterrupt)?ABSOLUTE (__CompInterrupt):ABSOLUTE (__DefaultInterrupt)
                  0x00003a          0x4 LONG 0x1532 DEFINED (__CNInterrupt)?ABSOLUTE (__CNInterrupt):ABSOLUTE (__DefaultInterrupt)
                  0x00003c          0x4 LONG 0x1532 DEFINED (__INT1Interrupt)?ABSOLUTE (__INT1Interrupt):ABSOLUTE (__DefaultInterrupt)
                  0x00003e          0x4 LONG 0x1532 DEFINED (__Interrupt21)?ABSOLUTE (__Interrupt21):ABSOLUTE (__DefaultInterrupt)
                  0x000040          0x4 LONG 0x1532 DEFINED (__Interrupt22)?ABSOLUTE (__Interrupt22):ABSOLUTE (__DefaultInterrupt)
                  0x000042          0x4 LONG 0x1532 DEFINED (__Interrupt23)?ABSOLUTE (__Interrupt23):ABSOLUTE (__DefaultInterrupt)
                  0x000044          0x4 LONG 0x1532 DEFINED (__DMA2Interrupt)?ABSOLUTE (__DMA2Interrupt):ABSOLUTE (__DefaultInterrupt)
                  0x000046          0x4 LONG 0x1532 DEFINED (__OC3Interrupt)?ABSOLUTE (__OC3Interrupt):ABSOLUTE (__DefaultInterrupt)
                  0x000048          0x4 LONG 0x1532 DEFINED (__OC4Interrupt)?ABSOLUTE (__OC4Interrupt):ABSOLUTE (__DefaultInterrupt)
                  0x00004a          0x4 LONG 0x1532 DEFINED (__T4Interrupt)?ABSOLUTE (__T4Interrupt):ABSOLUTE (__DefaultInterrupt)
                  0x00004c          0x4 LONG 0x1532 DEFINED (__T5Interrupt)?ABSOLUTE (__T5Interrupt):ABSOLUTE (__DefaultInterrupt)
                  0x00004e          0x4 LONG 0x1532 DEFINED (__INT2Interrupt)?ABSOLUTE (__INT2Interrupt):ABSOLUTE (__DefaultInterrupt)
                  0x000050          0x4 LONG 0x53a4 DEFINED (__U2RXInterrupt)?ABSOLUTE (__U2RXInterrupt):ABSOLUTE (__DefaultInterrupt)
                  0x000052          0x4 LONG 0x539c DEFINED (__U2TXInterrupt)?ABSOLUTE (__U2TXInterrupt):ABSOLUTE (__DefaultInterrupt)
                  0x000054          0x4 LONG 0x1532 DEFINED (__SPI2Interrupt)?ABSOLUTE (__SPI2Interrupt):ABSOLUTE (__DefaultInterrupt)
                  0x000056          0x4 LONG 0x1532 DEFINED (__SPI2TXInterrupt)?ABSOLUTE (__SPI2TXInterrupt):ABSOLUTE (__DefaultInterrupt)
                  0x000058          0x4 LONG 0x1532 DEFINED (__CRYPTOBufferReadyInterrupt)?ABSOLUTE (__CRYPTOBufferReadyInterrupt):ABSOLUTE (__DefaultInterrupt)
                  0x00005a          0x4 LONG 0x1532 DEFINED (__CRYPTORolloverInterrupt)?ABSOLUTE (__CRYPTORolloverInterrupt):ABSOLUTE (__DefaultInterrupt)
                  0x00005c          0x4 LONG 0x1532 DEFINED (__DMA3Interrupt)?ABSOLUTE (__DMA3Interrupt):ABSOLUTE (__DefaultInterrupt)
                  0x00005e          0x4 LONG 0x1532 DEFINED (__IC3Interrupt)?ABSOLUTE (__IC3Interrupt):ABSOLUTE (__DefaultInterrupt)
                  0x000060          0x4 LONG 0x1532 DEFINED (__IC4Interrupt)?ABSOLUTE (__IC4Interrupt):ABSOLUTE (__DefaultInterrupt)
                  0x000062          0x4 LONG 0x1532 DEFINED (__IC5Interrupt)?ABSOLUTE (__IC5Interrupt):ABSOLUTE (__DefaultInterrupt)
                  0x000064          0x4 LONG 0x1532 DEFINED (__IC6Interrupt)?ABSOLUTE (__IC6Interrupt):ABSOLUTE (__DefaultInterrupt)
                  0x000066          0x4 LONG 0x1532 DEFINED (__OC5Interrupt)?ABSOLUTE (__OC5Interrupt):ABSOLUTE (__DefaultInterrupt)
                  0x000068          0x4 LONG 0x1532 DEFINED (__OC6Interrupt)?ABSOLUTE (__OC6Interrupt):ABSOLUTE (__DefaultInterrupt)
                  0x00006a          0x4 LONG 0x1532 DEFINED (__CCT3Interrupt)?ABSOLUTE (__CCT3Interrupt):ABSOLUTE (__DefaultInterrupt)
                  0x00006c          0x4 LONG 0x1532 DEFINED (__CCT4Interrupt)?ABSOLUTE (__CCT4Interrupt):ABSOLUTE (__DefaultInterrupt)
                  0x00006e          0x4 LONG 0x1532 DEFINED (__PMPInterrupt)?ABSOLUTE (__PMPInterrupt):ABSOLUTE (__DefaultInterrupt)
                  0x000070          0x4 LONG 0x1532 DEFINED (__DMA4Interrupt)?ABSOLUTE (__DMA4Interrupt):ABSOLUTE (__DefaultInterrupt)
                  0x000072          0x4 LONG 0x1532 DEFINED (__CCT5Interrupt)?ABSOLUTE (__CCT5Interrupt):ABSOLUTE (__DefaultInterrupt)
                  0x000074          0x4 LONG 0x1532 DEFINED (__CCT6Interrupt)?ABSOLUTE (__CCT6Interrupt):ABSOLUTE (__DefaultInterrupt)
                  0x000076          0x4 LONG 0x1532 DEFINED (__SI2C2Interrupt)?ABSOLUTE (__SI2C2Interrupt):ABSOLUTE (__DefaultInterrupt)
                  0x000078          0x4 LONG 0x1532 DEFINED (__MI2C2Interrupt)?ABSOLUTE (__MI2C2Interrupt):ABSOLUTE (__DefaultInterrupt)
                  0x00007a          0x4 LONG 0x1532 DEFINED (__CCT7Interrupt)?ABSOLUTE (__CCT7Interrupt):ABSOLUTE (__DefaultInterrupt)
                  0x00007c          0x4 LONG 0x1532 DEFINED (__Interrupt52)?ABSOLUTE (__Interrupt52):ABSOLUTE (__DefaultInterrupt)
                  0x00007e          0x4 LONG 0x1532 DEFINED (__INT3Interrupt)?ABSOLUTE (__INT3Interrupt):ABSOLUTE (__DefaultInterrupt)
                  0x000080          0x4 LONG 0x1532 DEFINED (__INT4Interrupt)?ABSOLUTE (__INT4Interrupt):ABSOLUTE (__DefaultInterrupt)
                  0x000082          0x4 LONG 0x1532 DEFINED (__CRYPTOInterrupt)?ABSOLUTE (__CRYPTOInterrupt):ABSOLUTE (__DefaultInterrupt)
                  0x000084          0x4 LONG 0x1532 DEFINED (__CRYPTOKeyInterrupt)?ABSOLUTE (__CRYPTOKeyInterrupt):ABSOLUTE (__DefaultInterrupt)
                  0x000086          0x4 LONG 0x1532 DEFINED (__SPI4RXInterrupt)?ABSOLUTE (__SPI4RXInterrupt):ABSOLUTE (__DefaultInterrupt)
                  0x000088          0x4 LONG 0x1532 DEFINED (__SPI1RXInterrupt)?ABSOLUTE (__SPI1RXInterrupt):ABSOLUTE (__DefaultInterrupt)
                  0x00008a          0x4 LONG 0x1532 DEFINED (__SPI2RXInterrupt)?ABSOLUTE (__SPI2RXInterrupt):ABSOLUTE (__DefaultInterrupt)
                  0x00008c          0x4 LONG 0x1532 DEFINED (__SPI3RXInterrupt)?ABSOLUTE (__SPI3RXInterrupt):ABSOLUTE (__DefaultInterrupt)
                  0x00008e          0x4 LONG 0x1532 DEFINED (__DMA5Interrupt)?ABSOLUTE (__DMA5Interrupt):ABSOLUTE (__DefaultInterrupt)
                  0x000090          0x4 LONG 0x1532 DEFINED (__RTCCInterrupt)?ABSOLUTE (__RTCCInterrupt):ABSOLUTE (__DefaultInterrupt)
                  0x000092          0x4 LONG 0x1532 DEFINED (__CCP1Interrupt)?ABSOLUTE (__CCP1Interrupt):ABSOLUTE (__DefaultInterrupt)
                  0x000094          0x4 LONG 0x1532 DEFINED (__CCP2Interrupt)?ABSOLUTE (__CCP2Interrupt):ABSOLUTE (__DefaultInterrupt)
                  0x000096          0x4 LONG 0x1532 DEFINED (__U1ErrInterrupt)?ABSOLUTE (__U1ErrInterrupt):ABSOLUTE (__DefaultInterrupt)
                  0x000098          0x4 LONG 0x1532 DEFINED (__U2ErrInterrupt)?ABSOLUTE (__U2ErrInterrupt):ABSOLUTE (__DefaultInterrupt)
                  0x00009a          0x4 LONG 0x1532 DEFINED (__CRCInterrupt)?ABSOLUTE (__CRCInterrupt):ABSOLUTE (__DefaultInterrupt)
                  0x00009c          0x4 LONG 0x1532 DEFINED (__DMA6Interrupt)?ABSOLUTE (__DMA6Interrupt):ABSOLUTE (__DefaultInterrupt)
                  0x00009e          0x4 LONG 0x1532 DEFINED (__DMA7Interrupt)?ABSOLUTE (__DMA7Interrupt):ABSOLUTE (__DefaultInterrupt)
                  0x0000a0          0x4 LONG 0x1532 DEFINED (__SI2C3Interrupt)?ABSOLUTE (__SI2C3Interrupt):ABSOLUTE (__DefaultInterrupt)
                  0x0000a2          0x4 LONG 0x1532 DEFINED (__MI2C3Interrupt)?ABSOLUTE (__MI2C3Interrupt):ABSOLUTE (__DefaultInterrupt)
                  0x0000a4          0x4 LONG 0x1532 DEFINED (__LVDInterrupt)?ABSOLUTE (__LVDInterrupt):ABSOLUTE (__DefaultInterrupt)
                  0x0000a6          0x4 LONG 0x1532 DEFINED (__CCP7Interrupt)?ABSOLUTE (__CCP7Interrupt):ABSOLUTE (__DefaultInterrupt)
                  0x0000a8          0x4 LONG 0x1532 DEFINED (__Interrupt74)?ABSOLUTE (__Interrupt74):ABSOLUTE (__DefaultInterrupt)
                  0x0000aa          0x4 LONG 0x1532 DEFINED (__Interrupt75)?ABSOLUTE (__Interrupt75):ABSOLUTE (__DefaultInterrupt)
                  0x0000ac          0x4 LONG 0x1532 DEFINED (__Interrupt76)?ABSOLUTE (__Interrupt76):ABSOLUTE (__DefaultInterrupt)
                  0x0000ae          0x4 LONG 0x1532 DEFINED (__CTMUInterrupt)?ABSOLUTE (__CTMUInterrupt):ABSOLUTE (__DefaultInterrupt)
                  0x0000b0          0x4 LONG 0x1532 DEFINED (__DAC1Interrupt)?ABSOLUTE (__DAC1Interrupt):ABSOLUTE (__DefaultInterrupt)
                  0x0000b2          0x4 LONG 0x1532 DEFINED (__Interrupt79)?ABSOLUTE (__Interrupt79):ABSOLUTE (__DefaultInterrupt)
                  0x0000b4          0x4 LONG 0x1532 DEFINED (__Interrupt80)?ABSOLUTE (__Interrupt80):ABSOLUTE (__DefaultInterrupt)
                  0x0000b6          0x4 LONG 0x1532 DEFINED (__U3ErrInterrupt)?ABSOLUTE (__U3ErrInterrupt):ABSOLUTE (__DefaultInterrupt)
                  0x0000b8          0x4 LONG 0x5400 DEFINED (__U3RXInterrupt)?ABSOLUTE (__U3RXInterrupt):ABSOLUTE (__DefaultInterrupt)
                  0x0000ba          0x4 LONG 0x53f8 DEFINED (__U3TXInterrupt)?ABSOLUTE (__U3TXInterrupt):ABSOLUTE (__DefaultInterrupt)
                  0x0000bc          0x4 LONG 0x1532 DEFINED (__I2C1BCLInterrupt)?ABSOLUTE (__I2C1BCLInterrupt):ABSOLUTE (__DefaultInterrupt)
                  0x0000be          0x4 LONG 0x1532 DEFINED (__I2C2BCLInterrupt)?ABSOLUTE (__I2C2BCLInterrupt):ABSOLUTE (__DefaultInterrupt)
                  0x0000c0          0x4 LONG 0x1532 DEFINED (__USB1Interrupt)?ABSOLUTE (__USB1Interrupt):ABSOLUTE (__DefaultInterrupt)
                  0x0000c2          0x4 LONG 0x1532 DEFINED (__U4ErrInterrupt)?ABSOLUTE (__U4ErrInterrupt):ABSOLUTE (__DefaultInterrupt)
                  0x0000c4          0x4 LONG 0x545c DEFINED (__U4RXInterrupt)?ABSOLUTE (__U4RXInterrupt):ABSOLUTE (__DefaultInterrupt)
                  0x0000c6          0x4 LONG 0x5454 DEFINED (__U4TXInterrupt)?ABSOLUTE (__U4TXInterrupt):ABSOLUTE (__DefaultInterrupt)
                  0x0000c8          0x4 LONG 0x1532 DEFINED (__SPI3Interrupt)?ABSOLUTE (__SPI3Interrupt):ABSOLUTE (__DefaultInterrupt)
                  0x0000ca          0x4 LONG 0x1532 DEFINED (__SPI3TXInterrupt)?ABSOLUTE (__SPI3TXInterrupt):ABSOLUTE (__DefaultInterrupt)
                  0x0000cc          0x4 LONG 0x1532 DEFINED (__SPI4Interrupt)?ABSOLUTE (__SPI4Interrupt):ABSOLUTE (__DefaultInterrupt)
                  0x0000ce          0x4 LONG 0x1532 DEFINED (__SPI4TXInterrupt)?ABSOLUTE (__SPI4TXInterrupt):ABSOLUTE (__DefaultInterrupt)
                  0x0000d0          0x4 LONG 0x1532 DEFINED (__CCP3Interrupt)?ABSOLUTE (__CCP3Interrupt):ABSOLUTE (__DefaultInterrupt)
                  0x0000d2          0x4 LONG 0x1532 DEFINED (__CCP4Interrupt)?ABSOLUTE (__CCP4Interrupt):ABSOLUTE (__DefaultInterrupt)
                  0x0000d4          0x4 LONG 0x1532 DEFINED (__CLC1Interrupt)?ABSOLUTE (__CLC1Interrupt):ABSOLUTE (__DefaultInterrupt)
                  0x0000d6          0x4 LONG 0x1532 DEFINED (__CLC2Interrupt)?ABSOLUTE (__CLC2Interrupt):ABSOLUTE (__DefaultInterrupt)
                  0x0000d8          0x4 LONG 0x1532 DEFINED (__CLC3Interrupt)?ABSOLUTE (__CLC3Interrupt):ABSOLUTE (__DefaultInterrupt)
                  0x0000da          0x4 LONG 0x1532 DEFINED (__CLC4Interrupt)?ABSOLUTE (__CLC4Interrupt):ABSOLUTE (__DefaultInterrupt)
                  0x0000dc          0x4 LONG 0x1532 DEFINED (__LCDInterrupt)?ABSOLUTE (__LCDInterrupt):ABSOLUTE (__DefaultInterrupt)
                  0x0000de          0x4 LONG 0x1532 DEFINED (__CCT1Interrupt)?ABSOLUTE (__CCT1Interrupt):ABSOLUTE (__DefaultInterrupt)
                  0x0000e0          0x4 LONG 0x1532 DEFINED (__CCT2Interrupt)?ABSOLUTE (__CCT2Interrupt):ABSOLUTE (__DefaultInterrupt)
                  0x0000e2          0x4 LONG 0x1532 DEFINED (__Interrupt103)?ABSOLUTE (__Interrupt103):ABSOLUTE (__DefaultInterrupt)
                  0x0000e4          0x4 LONG 0x1532 DEFINED (__Interrupt104)?ABSOLUTE (__Interrupt104):ABSOLUTE (__DefaultInterrupt)
                  0x0000e6          0x4 LONG 0x1532 DEFINED (__Interrupt105)?ABSOLUTE (__Interrupt105):ABSOLUTE (__DefaultInterrupt)
                  0x0000e8          0x4 LONG 0x1532 DEFINED (__FSTInterrupt)?ABSOLUTE (__FSTInterrupt):ABSOLUTE (__DefaultInterrupt)
                  0x0000ea          0x4 LONG 0x1532 DEFINED (__Interrupt107)?ABSOLUTE (__Interrupt107):ABSOLUTE (__DefaultInterrupt)
                  0x0000ec          0x4 LONG 0x1532 DEFINED (__Interrupt108)?ABSOLUTE (__Interrupt108):ABSOLUTE (__DefaultInterrupt)
                  0x0000ee          0x4 LONG 0x1532 DEFINED (__I2C3BCLInterrupt)?ABSOLUTE (__I2C3BCLInterrupt):ABSOLUTE (__DefaultInterrupt)
                  0x0000f0          0x4 LONG 0x1532 DEFINED (__RTCCTSInterrupt)?ABSOLUTE (__RTCCTSInterrupt):ABSOLUTE (__DefaultInterrupt)
                  0x0000f2          0x4 LONG 0x54b8 DEFINED (__U5RXInterrupt)?ABSOLUTE (__U5RXInterrupt):ABSOLUTE (__DefaultInterrupt)
                  0x0000f4          0x4 LONG 0x54b0 DEFINED (__U5TXInterrupt)?ABSOLUTE (__U5TXInterrupt):ABSOLUTE (__DefaultInterrupt)
                  0x0000f6          0x4 LONG 0x1532 DEFINED (__U5ErrInterrupt)?ABSOLUTE (__U5ErrInterrupt):ABSOLUTE (__DefaultInterrupt)
                  0x0000f8          0x4 LONG 0x6db8 DEFINED (__U6RXInterrupt)?ABSOLUTE (__U6RXInterrupt):ABSOLUTE (__DefaultInterrupt)
                  0x0000fa          0x4 LONG 0x6d98 DEFINED (__U6TXInterrupt)?ABSOLUTE (__U6TXInterrupt):ABSOLUTE (__DefaultInterrupt)
                  0x0000fc          0x4 LONG 0x1532 DEFINED (__U6ErrInterrupt)?ABSOLUTE (__U6ErrInterrupt):ABSOLUTE (__DefaultInterrupt)
                  0x0000fe          0x4 LONG 0x1532 DEFINED (__JTAGInterrupt)?ABSOLUTE (__JTAGInterrupt):ABSOLUTE (__DefaultInterrupt)
                    0x0000                  WREG0 = 0x0
                    0x0000                  _WREG0 = 0x0
                    0x0002                  WREG1 = 0x2
                    0x0002                  _WREG1 = 0x2
                    0x0004                  WREG2 = 0x4
                    0x0004                  _WREG2 = 0x4
                    0x0006                  WREG3 = 0x6
                    0x0006                  _WREG3 = 0x6
                    0x0008                  WREG4 = 0x8
                    0x0008                  _WREG4 = 0x8
                    0x000a                  WREG5 = 0xa
                    0x000a                  _WREG5 = 0xa
                    0x000c                  WREG6 = 0xc
                    0x000c                  _WREG6 = 0xc
                    0x000e                  WREG7 = 0xe
                    0x000e                  _WREG7 = 0xe
                    0x0010                  WREG8 = 0x10
                    0x0010                  _WREG8 = 0x10
                    0x0012                  WREG9 = 0x12
                    0x0012                  _WREG9 = 0x12
                    0x0014                  WREG10 = 0x14
                    0x0014                  _WREG10 = 0x14
                    0x0016                  WREG11 = 0x16
                    0x0016                  _WREG11 = 0x16
                    0x0018                  WREG12 = 0x18
                    0x0018                  _WREG12 = 0x18
                    0x001a                  WREG13 = 0x1a
                    0x001a                  _WREG13 = 0x1a
                    0x001c                  WREG14 = 0x1c
                    0x001c                  _WREG14 = 0x1c
                    0x001e                  WREG15 = 0x1e
                    0x001e                  _WREG15 = 0x1e
                    0x0020                  SPLIM = 0x20
                    0x0020                  _SPLIM = 0x20
                    0x002e                  PCL = 0x2e
                    0x002e                  _PCL = 0x2e
                    0x0030                  PCH = 0x30
                    0x0030                  _PCH = 0x30
                    0x0032                  DSRPAG = 0x32
                    0x0032                  _DSRPAG = 0x32
                    0x0032                  _DSRPAGbits = 0x32
                    0x0034                  DSWPAG = 0x34
                    0x0034                  _DSWPAG = 0x34
                    0x0034                  _DSWPAGbits = 0x34
                    0x0036                  RCOUNT = 0x36
                    0x0036                  _RCOUNT = 0x36
                    0x0042                  SR = 0x42
                    0x0042                  _SR = 0x42
                    0x0042                  _SRbits = 0x42
                    0x0044                  CORCON = 0x44
                    0x0044                  _CORCON = 0x44
                    0x0044                  _CORCONbits = 0x44
                    0x0052                  DISICNT = 0x52
                    0x0052                  _DISICNT = 0x52
                    0x0052                  _DISICNTbits = 0x52
                    0x0054                  TBLPAG = 0x54
                    0x0054                  _TBLPAG = 0x54
                    0x0054                  _TBLPAGbits = 0x54
                    0x0080                  INTCON1 = 0x80
                    0x0080                  _INTCON1 = 0x80
                    0x0080                  _INTCON1bits = 0x80
                    0x0082                  INTCON2 = 0x82
                    0x0082                  _INTCON2 = 0x82
                    0x0082                  _INTCON2bits = 0x82
                    0x0084                  INTCON3 = 0x84
                    0x0084                  _INTCON3 = 0x84
                    0x0086                  INTCON4 = 0x86
                    0x0086                  _INTCON4 = 0x86
                    0x0086                  _INTCON4bits = 0x86
                    0x0088                  IFS0 = 0x88
                    0x0088                  _IFS0 = 0x88
                    0x0088                  _IFS0bits = 0x88
                    0x008a                  IFS1 = 0x8a
                    0x008a                  _IFS1 = 0x8a
                    0x008a                  _IFS1bits = 0x8a
                    0x008c                  IFS2 = 0x8c
                    0x008c                  _IFS2 = 0x8c
                    0x008c                  _IFS2bits = 0x8c
                    0x008e                  IFS3 = 0x8e
                    0x008e                  _IFS3 = 0x8e
                    0x008e                  _IFS3bits = 0x8e
                    0x0090                  IFS4 = 0x90
                    0x0090                  _IFS4 = 0x90
                    0x0090                  _IFS4bits = 0x90
                    0x0092                  IFS5 = 0x92
                    0x0092                  _IFS5 = 0x92
                    0x0092                  _IFS5bits = 0x92
                    0x0094                  IFS6 = 0x94
                    0x0094                  _IFS6 = 0x94
                    0x0094                  _IFS6bits = 0x94
                    0x0096                  IFS7 = 0x96
                    0x0096                  _IFS7 = 0x96
                    0x0096                  _IFS7bits = 0x96
                    0x0098                  IEC0 = 0x98
                    0x0098                  _IEC0 = 0x98
                    0x0098                  _IEC0bits = 0x98
                    0x009a                  IEC1 = 0x9a
                    0x009a                  _IEC1 = 0x9a
                    0x009a                  _IEC1bits = 0x9a
                    0x009c                  IEC2 = 0x9c
                    0x009c                  _IEC2 = 0x9c
                    0x009c                  _IEC2bits = 0x9c
                    0x009e                  IEC3 = 0x9e
                    0x009e                  _IEC3 = 0x9e
                    0x009e                  _IEC3bits = 0x9e
                    0x00a0                  IEC4 = 0xa0
                    0x00a0                  _IEC4 = 0xa0
                    0x00a0                  _IEC4bits = 0xa0
                    0x00a2                  IEC5 = 0xa2
                    0x00a2                  _IEC5 = 0xa2
                    0x00a2                  _IEC5bits = 0xa2
                    0x00a4                  IEC6 = 0xa4
                    0x00a4                  _IEC6 = 0xa4
                    0x00a4                  _IEC6bits = 0xa4
                    0x00a6                  IEC7 = 0xa6
                    0x00a6                  _IEC7 = 0xa6
                    0x00a6                  _IEC7bits = 0xa6
                    0x00a8                  IPC0 = 0xa8
                    0x00a8                  _IPC0 = 0xa8
                    0x00a8                  _IPC0bits = 0xa8
                    0x00aa                  IPC1 = 0xaa
                    0x00aa                  _IPC1 = 0xaa
                    0x00aa                  _IPC1bits = 0xaa
                    0x00ac                  IPC2 = 0xac
                    0x00ac                  _IPC2 = 0xac
                    0x00ac                  _IPC2bits = 0xac
                    0x00ae                  IPC3 = 0xae
                    0x00ae                  _IPC3 = 0xae
                    0x00ae                  _IPC3bits = 0xae
                    0x00b0                  IPC4 = 0xb0
                    0x00b0                  _IPC4 = 0xb0
                    0x00b0                  _IPC4bits = 0xb0
                    0x00b2                  IPC5 = 0xb2
                    0x00b2                  _IPC5 = 0xb2
                    0x00b2                  _IPC5bits = 0xb2
                    0x00b4                  IPC6 = 0xb4
                    0x00b4                  _IPC6 = 0xb4
                    0x00b4                  _IPC6bits = 0xb4
                    0x00b6                  IPC7 = 0xb6
                    0x00b6                  _IPC7 = 0xb6
                    0x00b6                  _IPC7bits = 0xb6
                    0x00b8                  IPC8 = 0xb8
                    0x00b8                  _IPC8 = 0xb8
                    0x00b8                  _IPC8bits = 0xb8
                    0x00ba                  IPC9 = 0xba
                    0x00ba                  _IPC9 = 0xba
                    0x00ba                  _IPC9bits = 0xba
                    0x00bc                  IPC10 = 0xbc
                    0x00bc                  _IPC10 = 0xbc
                    0x00bc                  _IPC10bits = 0xbc
                    0x00be                  IPC11 = 0xbe
                    0x00be                  _IPC11 = 0xbe
                    0x00be                  _IPC11bits = 0xbe
                    0x00c0                  IPC12 = 0xc0
                    0x00c0                  _IPC12 = 0xc0
                    0x00c0                  _IPC12bits = 0xc0
                    0x00c2                  IPC13 = 0xc2
                    0x00c2                  _IPC13 = 0xc2
                    0x00c2                  _IPC13bits = 0xc2
                    0x00c4                  IPC14 = 0xc4
                    0x00c4                  _IPC14 = 0xc4
                    0x00c4                  _IPC14bits = 0xc4
                    0x00c6                  IPC15 = 0xc6
                    0x00c6                  _IPC15 = 0xc6
                    0x00c6                  _IPC15bits = 0xc6
                    0x00c8                  IPC16 = 0xc8
                    0x00c8                  _IPC16 = 0xc8
                    0x00c8                  _IPC16bits = 0xc8
                    0x00ca                  IPC17 = 0xca
                    0x00ca                  _IPC17 = 0xca
                    0x00ca                  _IPC17bits = 0xca
                    0x00cc                  IPC18 = 0xcc
                    0x00cc                  _IPC18 = 0xcc
                    0x00cc                  _IPC18bits = 0xcc
                    0x00ce                  IPC19 = 0xce
                    0x00ce                  _IPC19 = 0xce
                    0x00ce                  _IPC19bits = 0xce
                    0x00d0                  IPC20 = 0xd0
                    0x00d0                  _IPC20 = 0xd0
                    0x00d0                  _IPC20bits = 0xd0
                    0x00d2                  IPC21 = 0xd2
                    0x00d2                  _IPC21 = 0xd2
                    0x00d2                  _IPC21bits = 0xd2
                    0x00d4                  IPC22 = 0xd4
                    0x00d4                  _IPC22 = 0xd4
                    0x00d4                  _IPC22bits = 0xd4
                    0x00d6                  IPC23 = 0xd6
                    0x00d6                  _IPC23 = 0xd6
                    0x00d6                  _IPC23bits = 0xd6
                    0x00d8                  IPC24 = 0xd8
                    0x00d8                  _IPC24 = 0xd8
                    0x00d8                  _IPC24bits = 0xd8
                    0x00da                  IPC25 = 0xda
                    0x00da                  _IPC25 = 0xda
                    0x00da                  _IPC25bits = 0xda
                    0x00dc                  IPC26 = 0xdc
                    0x00dc                  _IPC26 = 0xdc
                    0x00dc                  _IPC26bits = 0xdc
                    0x00de                  IPC27 = 0xde
                    0x00de                  _IPC27 = 0xde
                    0x00de                  _IPC27bits = 0xde
                    0x00e0                  IPC28 = 0xe0
                    0x00e0                  _IPC28 = 0xe0
                    0x00e0                  _IPC28bits = 0xe0
                    0x00e2                  IPC29 = 0xe2
                    0x00e2                  _IPC29 = 0xe2
                    0x00e2                  _IPC29bits = 0xe2
                    0x00e4                  INTTREG = 0xe4
                    0x00e4                  _INTTREG = 0xe4
                    0x00e4                  _INTTREGbits = 0xe4
                    0x0100                  OSCCON = 0x100
                    0x0100                  _OSCCON = 0x100
                    0x0100                  _OSCCONbits = 0x100
                    0x0100                  OSCCONL = 0x100
                    0x0100                  _OSCCONL = 0x100
                    0x0101                  OSCCONH = 0x101
                    0x0101                  _OSCCONH = 0x101
                    0x0102                  CLKDIV = 0x102
                    0x0102                  _CLKDIV = 0x102
                    0x0102                  _CLKDIVbits = 0x102
                    0x0104                  CLKDIV2 = 0x104
                    0x0104                  _CLKDIV2 = 0x104
                    0x0106                  OSCTUN = 0x106
                    0x0106                  _OSCTUN = 0x106
                    0x0106                  _OSCTUNbits = 0x106
                    0x010c                  RCON = 0x10c
                    0x010c                  _RCON = 0x10c
                    0x010c                  _RCONbits = 0x10c
                    0x010e                  RCON2 = 0x10e
                    0x010e                  _RCON2 = 0x10e
                    0x010e                  _RCON2bits = 0x10e
                    0x0110                  HLVDCON = 0x110
                    0x0110                  _HLVDCON = 0x110
                    0x0110                  _HLVDCONbits = 0x110
                    0x0112                  DSCON = 0x112
                    0x0112                  _DSCON = 0x112
                    0x0112                  _DSCONbits = 0x112
                    0x0114                  DSWAKE = 0x114
                    0x0114                  _DSWAKE = 0x114
                    0x0114                  _DSWAKEbits = 0x114
                    0x0116                  DSGPR0 = 0x116
                    0x0116                  _DSGPR0 = 0x116
                    0x0118                  DSGPR1 = 0x118
                    0x0118                  _DSGPR1 = 0x118
                    0x0128                  PMCON1 = 0x128
                    0x0128                  _PMCON1 = 0x128
                    0x0128                  _PMCON1bits = 0x128
                    0x012a                  PMCON2 = 0x12a
                    0x012a                  _PMCON2 = 0x12a
                    0x012a                  _PMCON2bits = 0x12a
                    0x012c                  PMCON3 = 0x12c
                    0x012c                  _PMCON3 = 0x12c
                    0x012c                  _PMCON3bits = 0x12c
                    0x012e                  PMCON4 = 0x12e
                    0x012e                  _PMCON4 = 0x12e
                    0x012e                  _PMCON4bits = 0x12e
                    0x0130                  PMCS1CF = 0x130
                    0x0130                  _PMCS1CF = 0x130
                    0x0130                  _PMCS1CFbits = 0x130
                    0x0132                  PMCS1BS = 0x132
                    0x0132                  _PMCS1BS = 0x132
                    0x0132                  _PMCS1BSbits = 0x132
                    0x0134                  PMCS1MD = 0x134
                    0x0134                  _PMCS1MD = 0x134
                    0x0134                  _PMCS1MDbits = 0x134
                    0x0136                  PMCS2CF = 0x136
                    0x0136                  _PMCS2CF = 0x136
                    0x0136                  _PMCS2CFbits = 0x136
                    0x0138                  PMCS2BS = 0x138
                    0x0138                  _PMCS2BS = 0x138
                    0x0138                  _PMCS2BSbits = 0x138
                    0x013a                  PMCS2MD = 0x13a
                    0x013a                  _PMCS2MD = 0x13a
                    0x013a                  _PMCS2MDbits = 0x13a
                    0x013c                  PMDOUT1 = 0x13c
                    0x013c                  _PMDOUT1 = 0x13c
                    0x013e                  PMDOUT2 = 0x13e
                    0x013e                  _PMDOUT2 = 0x13e
                    0x0140                  PMDIN1 = 0x140
                    0x0140                  _PMDIN1 = 0x140
                    0x0142                  PMDIN2 = 0x142
                    0x0142                  _PMDIN2 = 0x142
                    0x0144                  PMSTAT = 0x144
                    0x0144                  _PMSTAT = 0x144
                    0x0144                  _PMSTATbits = 0x144
                    0x0158                  CRCCON1 = 0x158
                    0x0158                  _CRCCON1 = 0x158
                    0x0158                  _CRCCON1bits = 0x158
                    0x015a                  CRCCON2 = 0x15a
                    0x015a                  _CRCCON2 = 0x15a
                    0x015a                  _CRCCON2bits = 0x15a
                    0x015c                  CRCXORL = 0x15c
                    0x015c                  _CRCXORL = 0x15c
                    0x015c                  _CRCXORLbits = 0x15c
                    0x015e                  CRCXORH = 0x15e
                    0x015e                  _CRCXORH = 0x15e
                    0x015e                  _CRCXORHbits = 0x15e
                    0x0160                  CRCDAT = 0x160
                    0x0160                  _CRCDAT = 0x160
                    0x0160                  CRCDATL = 0x160
                    0x0160                  _CRCDATL = 0x160
                    0x0162                  CRCDATH = 0x162
                    0x0162                  _CRCDATH = 0x162
                    0x0164                  CRCWDAT = 0x164
                    0x0164                  _CRCWDAT = 0x164
                    0x0164                  CRCWDATL = 0x164
                    0x0164                  _CRCWDATL = 0x164
                    0x0166                  CRCWDATH = 0x166
                    0x0166                  _CRCWDATH = 0x166
                    0x0168                  REFOCON1 = 0x168
                    0x0168                  _REFOCON1 = 0x168
                    0x0168                  _REFOCON1bits = 0x168
                    0x0168                  REFOCONL = 0x168
                    0x0168                  _REFOCONL = 0x168
                    0x0168                  _REFOCONLbits = 0x168
                    0x016a                  REFOCON2 = 0x16a
                    0x016a                  _REFOCON2 = 0x16a
                    0x016a                  _REFOCON2bits = 0x16a
                    0x016a                  REFOCONH = 0x16a
                    0x016a                  _REFOCONH = 0x16a
                    0x016a                  _REFOCONHbits = 0x16a
                    0x016c                  REFOTRIML = 0x16c
                    0x016c                  _REFOTRIML = 0x16c
                    0x016c                  _REFOTRIMLbits = 0x16c
                    0x016e                  REFOTRIMH = 0x16e
                    0x016e                  _REFOTRIMH = 0x16e
                    0x0178                  PMD1 = 0x178
                    0x0178                  _PMD1 = 0x178
                    0x0178                  _PMD1bits = 0x178
                    0x017a                  PMD2 = 0x17a
                    0x017a                  _PMD2 = 0x17a
                    0x017a                  _PMD2bits = 0x17a
                    0x017c                  PMD3 = 0x17c
                    0x017c                  _PMD3 = 0x17c
                    0x017c                  _PMD3bits = 0x17c
                    0x017e                  PMD4 = 0x17e
                    0x017e                  _PMD4 = 0x17e
                    0x017e                  _PMD4bits = 0x17e
                    0x0180                  PMD5 = 0x180
                    0x0180                  _PMD5 = 0x180
                    0x0180                  _PMD5bits = 0x180
                    0x0182                  PMD6 = 0x182
                    0x0182                  _PMD6 = 0x182
                    0x0182                  _PMD6bits = 0x182
                    0x0184                  PMD7 = 0x184
                    0x0184                  _PMD7 = 0x184
                    0x0184                  _PMD7bits = 0x184
                    0x0186                  PMD8 = 0x186
                    0x0186                  _PMD8 = 0x186
                    0x0186                  _PMD8bits = 0x186
                    0x0190                  TMR1 = 0x190
                    0x0190                  _TMR1 = 0x190
                    0x0192                  PR1 = 0x192
                    0x0192                  _PR1 = 0x192
                    0x0194                  T1CON = 0x194
                    0x0194                  _T1CON = 0x194
                    0x0194                  _T1CONbits = 0x194
                    0x0196                  TMR2 = 0x196
                    0x0196                  _TMR2 = 0x196
                    0x0198                  TMR3HLD = 0x198
                    0x0198                  _TMR3HLD = 0x198
                    0x019a                  TMR3 = 0x19a
                    0x019a                  _TMR3 = 0x19a
                    0x019c                  PR2 = 0x19c
                    0x019c                  _PR2 = 0x19c
                    0x019e                  PR3 = 0x19e
                    0x019e                  _PR3 = 0x19e
                    0x01a0                  T2CON = 0x1a0
                    0x01a0                  _T2CON = 0x1a0
                    0x01a0                  _T2CONbits = 0x1a0
                    0x01a2                  T3CON = 0x1a2
                    0x01a2                  _T3CON = 0x1a2
                    0x01a2                  _T3CONbits = 0x1a2
                    0x01a4                  TMR4 = 0x1a4
                    0x01a4                  _TMR4 = 0x1a4
                    0x01a6                  TMR5HLD = 0x1a6
                    0x01a6                  _TMR5HLD = 0x1a6
                    0x01a8                  TMR5 = 0x1a8
                    0x01a8                  _TMR5 = 0x1a8
                    0x01aa                  PR4 = 0x1aa
                    0x01aa                  _PR4 = 0x1aa
                    0x01ac                  PR5 = 0x1ac
                    0x01ac                  _PR5 = 0x1ac
                    0x01ae                  T4CON = 0x1ae
                    0x01ae                  _T4CON = 0x1ae
                    0x01ae                  _T4CONbits = 0x1ae
                    0x01b0                  T5CON = 0x1b0
                    0x01b0                  _T5CON = 0x1b0
                    0x01b0                  _T5CONbits = 0x1b0
                    0x01c0                  CTMUCON1L = 0x1c0
                    0x01c0                  _CTMUCON1L = 0x1c0
                    0x01c0                  _CTMUCON1Lbits = 0x1c0
                    0x01c2                  CTMUCON1H = 0x1c2
                    0x01c2                  _CTMUCON1H = 0x1c2
                    0x01c2                  _CTMUCON1Hbits = 0x1c2
                    0x01c4                  CTMUCON2 = 0x1c4
                    0x01c4                  _CTMUCON2 = 0x1c4
                    0x01c4                  _CTMUCON2bits = 0x1c4
                    0x01c4                  CTMUCON2L = 0x1c4
                    0x01c4                  _CTMUCON2L = 0x1c4
                    0x01c4                  _CTMUCON2Lbits = 0x1c4
                    0x01c6                  CTMUCON2H = 0x1c6
                    0x01c6                  _CTMUCON2H = 0x1c6
                    0x01cc                  RTCCON1L = 0x1cc
                    0x01cc                  _RTCCON1L = 0x1cc
                    0x01cc                  _RTCCON1Lbits = 0x1cc
                    0x01ce                  RTCCON1H = 0x1ce
                    0x01ce                  _RTCCON1H = 0x1ce
                    0x01ce                  _RTCCON1Hbits = 0x1ce
                    0x01d0                  RTCCON2L = 0x1d0
                    0x01d0                  _RTCCON2L = 0x1d0
                    0x01d0                  _RTCCON2Lbits = 0x1d0
                    0x01d2                  RTCCON2H = 0x1d2
                    0x01d2                  _RTCCON2H = 0x1d2
                    0x01d4                  RTCCON3L = 0x1d4
                    0x01d4                  _RTCCON3L = 0x1d4
                    0x01d4                  _RTCCON3Lbits = 0x1d4
                    0x01d6                  RTCCON3H = 0x1d6
                    0x01d6                  _RTCCON3H = 0x1d6
                    0x01d8                  RTCSTATL = 0x1d8
                    0x01d8                  _RTCSTATL = 0x1d8
                    0x01d8                  _RTCSTATLbits = 0x1d8
                    0x01da                  RTCSTATH = 0x1da
                    0x01da                  _RTCSTATH = 0x1da
                    0x01dc                  TIMEL = 0x1dc
                    0x01dc                  _TIMEL = 0x1dc
                    0x01dc                  _TIMELbits = 0x1dc
                    0x01de                  TIMEH = 0x1de
                    0x01de                  _TIMEH = 0x1de
                    0x01de                  _TIMEHbits = 0x1de
                    0x01e0                  DATEL = 0x1e0
                    0x01e0                  _DATEL = 0x1e0
                    0x01e0                  _DATELbits = 0x1e0
                    0x01e2                  DATEH = 0x1e2
                    0x01e2                  _DATEH = 0x1e2
                    0x01e2                  _DATEHbits = 0x1e2
                    0x01e4                  ALMTIMEL = 0x1e4
                    0x01e4                  _ALMTIMEL = 0x1e4
                    0x01e4                  _ALMTIMELbits = 0x1e4
                    0x01e6                  ALMTIMEH = 0x1e6
                    0x01e6                  _ALMTIMEH = 0x1e6
                    0x01e6                  _ALMTIMEHbits = 0x1e6
                    0x01e8                  ALMDATEL = 0x1e8
                    0x01e8                  _ALMDATEL = 0x1e8
                    0x01e8                  _ALMDATELbits = 0x1e8
                    0x01ea                  ALMDATEH = 0x1ea
                    0x01ea                  _ALMDATEH = 0x1ea
                    0x01ea                  _ALMDATEHbits = 0x1ea
                    0x01ec                  TSATIMEL = 0x1ec
                    0x01ec                  _TSATIMEL = 0x1ec
                    0x01ec                  _TSATIMELbits = 0x1ec
                    0x01ee                  TSATIMEH = 0x1ee
                    0x01ee                  _TSATIMEH = 0x1ee
                    0x01ee                  _TSATIMEHbits = 0x1ee
                    0x01f0                  TSADATEL = 0x1f0
                    0x01f0                  _TSADATEL = 0x1f0
                    0x01f0                  _TSADATELbits = 0x1f0
                    0x01f2                  TSADATEH = 0x1f2
                    0x01f2                  _TSADATEH = 0x1f2
                    0x01f2                  _TSADATEHbits = 0x1f2
                    0x01f4                  TSBTIMEL = 0x1f4
                    0x01f4                  _TSBTIMEL = 0x1f4
                    0x01f4                  _TSBTIMELbits = 0x1f4
                    0x01f6                  TSBTIMEH = 0x1f6
                    0x01f6                  _TSBTIMEH = 0x1f6
                    0x01f6                  _TSBTIMEHbits = 0x1f6
                    0x01f8                  TSBDATEL = 0x1f8
                    0x01f8                  _TSBDATEL = 0x1f8
                    0x01f8                  _TSBDATELbits = 0x1f8
                    0x01fa                  TSBDATEH = 0x1fa
                    0x01fa                  _TSBDATEH = 0x1fa
                    0x01fa                  _TSBDATEHbits = 0x1fa
                    0x0200                  IC1CON1 = 0x200
                    0x0200                  _IC1CON1 = 0x200
                    0x0200                  _IC1CON1bits = 0x200
                    0x0202                  IC1CON2 = 0x202
                    0x0202                  _IC1CON2 = 0x202
                    0x0202                  _IC1CON2bits = 0x202
                    0x0204                  IC1BUF = 0x204
                    0x0204                  _IC1BUF = 0x204
                    0x0206                  IC1TMR = 0x206
                    0x0206                  _IC1TMR = 0x206
                    0x0208                  IC2CON1 = 0x208
                    0x0208                  _IC2CON1 = 0x208
                    0x0208                  _IC2CON1bits = 0x208
                    0x020a                  IC2CON2 = 0x20a
                    0x020a                  _IC2CON2 = 0x20a
                    0x020a                  _IC2CON2bits = 0x20a
                    0x020c                  IC2BUF = 0x20c
                    0x020c                  _IC2BUF = 0x20c
                    0x020e                  IC2TMR = 0x20e
                    0x020e                  _IC2TMR = 0x20e
                    0x0210                  IC3CON1 = 0x210
                    0x0210                  _IC3CON1 = 0x210
                    0x0210                  _IC3CON1bits = 0x210
                    0x0212                  IC3CON2 = 0x212
                    0x0212                  _IC3CON2 = 0x212
                    0x0212                  _IC3CON2bits = 0x212
                    0x0214                  IC3BUF = 0x214
                    0x0214                  _IC3BUF = 0x214
                    0x0216                  IC3TMR = 0x216
                    0x0216                  _IC3TMR = 0x216
                    0x0218                  IC4CON1 = 0x218
                    0x0218                  _IC4CON1 = 0x218
                    0x0218                  _IC4CON1bits = 0x218
                    0x021a                  IC4CON2 = 0x21a
                    0x021a                  _IC4CON2 = 0x21a
                    0x021a                  _IC4CON2bits = 0x21a
                    0x021c                  IC4BUF = 0x21c
                    0x021c                  _IC4BUF = 0x21c
                    0x021e                  IC4TMR = 0x21e
                    0x021e                  _IC4TMR = 0x21e
                    0x0220                  IC5CON1 = 0x220
                    0x0220                  _IC5CON1 = 0x220
                    0x0220                  _IC5CON1bits = 0x220
                    0x0222                  IC5CON2 = 0x222
                    0x0222                  _IC5CON2 = 0x222
                    0x0222                  _IC5CON2bits = 0x222
                    0x0224                  IC5BUF = 0x224
                    0x0224                  _IC5BUF = 0x224
                    0x0226                  IC5TMR = 0x226
                    0x0226                  _IC5TMR = 0x226
                    0x0228                  IC6CON1 = 0x228
                    0x0228                  _IC6CON1 = 0x228
                    0x0228                  _IC6CON1bits = 0x228
                    0x022a                  IC6CON2 = 0x22a
                    0x022a                  _IC6CON2 = 0x22a
                    0x022a                  _IC6CON2bits = 0x22a
                    0x022c                  IC6BUF = 0x22c
                    0x022c                  _IC6BUF = 0x22c
                    0x022e                  IC6TMR = 0x22e
                    0x022e                  _IC6TMR = 0x22e
                    0x0230                  OC1CON1 = 0x230
                    0x0230                  _OC1CON1 = 0x230
                    0x0230                  _OC1CON1bits = 0x230
                    0x0232                  OC1CON2 = 0x232
                    0x0232                  _OC1CON2 = 0x232
                    0x0232                  _OC1CON2bits = 0x232
                    0x0234                  OC1RS = 0x234
                    0x0234                  _OC1RS = 0x234
                    0x0236                  OC1R = 0x236
                    0x0236                  _OC1R = 0x236
                    0x0238                  OC1TMR = 0x238
                    0x0238                  _OC1TMR = 0x238
                    0x023a                  OC2CON1 = 0x23a
                    0x023a                  _OC2CON1 = 0x23a
                    0x023a                  _OC2CON1bits = 0x23a
                    0x023c                  OC2CON2 = 0x23c
                    0x023c                  _OC2CON2 = 0x23c
                    0x023c                  _OC2CON2bits = 0x23c
                    0x023e                  OC2RS = 0x23e
                    0x023e                  _OC2RS = 0x23e
                    0x0240                  OC2R = 0x240
                    0x0240                  _OC2R = 0x240
                    0x0242                  OC2TMR = 0x242
                    0x0242                  _OC2TMR = 0x242
                    0x0244                  OC3CON1 = 0x244
                    0x0244                  _OC3CON1 = 0x244
                    0x0244                  _OC3CON1bits = 0x244
                    0x0246                  OC3CON2 = 0x246
                    0x0246                  _OC3CON2 = 0x246
                    0x0246                  _OC3CON2bits = 0x246
                    0x0248                  OC3RS = 0x248
                    0x0248                  _OC3RS = 0x248
                    0x024a                  OC3R = 0x24a
                    0x024a                  _OC3R = 0x24a
                    0x024c                  OC3TMR = 0x24c
                    0x024c                  _OC3TMR = 0x24c
                    0x024e                  OC4CON1 = 0x24e
                    0x024e                  _OC4CON1 = 0x24e
                    0x024e                  _OC4CON1bits = 0x24e
                    0x0250                  OC4CON2 = 0x250
                    0x0250                  _OC4CON2 = 0x250
                    0x0250                  _OC4CON2bits = 0x250
                    0x0252                  OC4RS = 0x252
                    0x0252                  _OC4RS = 0x252
                    0x0254                  OC4R = 0x254
                    0x0254                  _OC4R = 0x254
                    0x0256                  OC4TMR = 0x256
                    0x0256                  _OC4TMR = 0x256
                    0x0258                  OC5CON1 = 0x258
                    0x0258                  _OC5CON1 = 0x258
                    0x0258                  _OC5CON1bits = 0x258
                    0x025a                  OC5CON2 = 0x25a
                    0x025a                  _OC5CON2 = 0x25a
                    0x025a                  _OC5CON2bits = 0x25a
                    0x025c                  OC5RS = 0x25c
                    0x025c                  _OC5RS = 0x25c
                    0x025e                  OC5R = 0x25e
                    0x025e                  _OC5R = 0x25e
                    0x0260                  OC5TMR = 0x260
                    0x0260                  _OC5TMR = 0x260
                    0x0262                  OC6CON1 = 0x262
                    0x0262                  _OC6CON1 = 0x262
                    0x0262                  _OC6CON1bits = 0x262
                    0x0264                  OC6CON2 = 0x264
                    0x0264                  _OC6CON2 = 0x264
                    0x0264                  _OC6CON2bits = 0x264
                    0x0266                  OC6RS = 0x266
                    0x0266                  _OC6RS = 0x266
                    0x0268                  OC6R = 0x268
                    0x0268                  _OC6R = 0x268
                    0x026a                  OC6TMR = 0x26a
                    0x026a                  _OC6TMR = 0x26a
                    0x026c                  CCP1CON1L = 0x26c
                    0x026c                  _CCP1CON1L = 0x26c
                    0x026c                  _CCP1CON1Lbits = 0x26c
                    0x026e                  CCP1CON1H = 0x26e
                    0x026e                  _CCP1CON1H = 0x26e
                    0x026e                  _CCP1CON1Hbits = 0x26e
                    0x0270                  CCP1CON2L = 0x270
                    0x0270                  _CCP1CON2L = 0x270
                    0x0270                  _CCP1CON2Lbits = 0x270
                    0x0272                  CCP1CON2H = 0x272
                    0x0272                  _CCP1CON2H = 0x272
                    0x0272                  _CCP1CON2Hbits = 0x272
                    0x0274                  CCP1CON3L = 0x274
                    0x0274                  _CCP1CON3L = 0x274
                    0x0274                  _CCP1CON3Lbits = 0x274
                    0x0276                  CCP1CON3H = 0x276
                    0x0276                  _CCP1CON3H = 0x276
                    0x0276                  _CCP1CON3Hbits = 0x276
                    0x0278                  CCP1STAT = 0x278
                    0x0278                  _CCP1STAT = 0x278
                    0x0278                  _CCP1STATbits = 0x278
                    0x0278                  CCP1STATL = 0x278
                    0x0278                  _CCP1STATL = 0x278
                    0x0278                  _CCP1STATLbits = 0x278
                    0x027a                  CCP1STATH = 0x27a
                    0x027a                  _CCP1STATH = 0x27a
                    0x027a                  _CCP1STATHbits = 0x27a
                    0x027c                  CCP1TMRL = 0x27c
                    0x027c                  _CCP1TMRL = 0x27c
                    0x027e                  CCP1TMRH = 0x27e
                    0x027e                  _CCP1TMRH = 0x27e
                    0x0280                  CCP1PRL = 0x280
                    0x0280                  _CCP1PRL = 0x280
                    0x0282                  CCP1PRH = 0x282
                    0x0282                  _CCP1PRH = 0x282
                    0x0284                  CCP1RA = 0x284
                    0x0284                  _CCP1RA = 0x284
                    0x0284                  CCP1RAL = 0x284
                    0x0284                  _CCP1RAL = 0x284
                    0x0286                  CCP1RAH = 0x286
                    0x0286                  _CCP1RAH = 0x286
                    0x0288                  CCP1RB = 0x288
                    0x0288                  _CCP1RB = 0x288
                    0x0288                  CCP1RBL = 0x288
                    0x0288                  _CCP1RBL = 0x288
                    0x028a                  CCP1RBH = 0x28a
                    0x028a                  _CCP1RBH = 0x28a
                    0x028c                  CCP1BUFL = 0x28c
                    0x028c                  _CCP1BUFL = 0x28c
                    0x028e                  CCP1BUFH = 0x28e
                    0x028e                  _CCP1BUFH = 0x28e
                    0x0290                  CCP2CON1L = 0x290
                    0x0290                  _CCP2CON1L = 0x290
                    0x0290                  _CCP2CON1Lbits = 0x290
                    0x0292                  CCP2CON1H = 0x292
                    0x0292                  _CCP2CON1H = 0x292
                    0x0292                  _CCP2CON1Hbits = 0x292
                    0x0294                  CCP2CON2L = 0x294
                    0x0294                  _CCP2CON2L = 0x294
                    0x0294                  _CCP2CON2Lbits = 0x294
                    0x0296                  CCP2CON2H = 0x296
                    0x0296                  _CCP2CON2H = 0x296
                    0x0296                  _CCP2CON2Hbits = 0x296
                    0x0298                  CCP2CON3L = 0x298
                    0x0298                  _CCP2CON3L = 0x298
                    0x0298                  _CCP2CON3Lbits = 0x298
                    0x029a                  CCP2CON3H = 0x29a
                    0x029a                  _CCP2CON3H = 0x29a
                    0x029a                  _CCP2CON3Hbits = 0x29a
                    0x029c                  CCP2STAT = 0x29c
                    0x029c                  _CCP2STAT = 0x29c
                    0x029c                  _CCP2STATbits = 0x29c
                    0x029c                  CCP2STATL = 0x29c
                    0x029c                  _CCP2STATL = 0x29c
                    0x029c                  _CCP2STATLbits = 0x29c
                    0x029e                  CCP2STATH = 0x29e
                    0x029e                  _CCP2STATH = 0x29e
                    0x029e                  _CCP2STATHbits = 0x29e
                    0x02a0                  CCP2TMRL = 0x2a0
                    0x02a0                  _CCP2TMRL = 0x2a0
                    0x02a2                  CCP2TMRH = 0x2a2
                    0x02a2                  _CCP2TMRH = 0x2a2
                    0x02a4                  CCP2PRL = 0x2a4
                    0x02a4                  _CCP2PRL = 0x2a4
                    0x02a6                  CCP2PRH = 0x2a6
                    0x02a6                  _CCP2PRH = 0x2a6
                    0x02a8                  CCP2RA = 0x2a8
                    0x02a8                  _CCP2RA = 0x2a8
                    0x02a8                  CCP2RAL = 0x2a8
                    0x02a8                  _CCP2RAL = 0x2a8
                    0x02aa                  CCP2RAH = 0x2aa
                    0x02aa                  _CCP2RAH = 0x2aa
                    0x02ac                  CCP2RB = 0x2ac
                    0x02ac                  _CCP2RB = 0x2ac
                    0x02ac                  CCP2RBL = 0x2ac
                    0x02ac                  _CCP2RBL = 0x2ac
                    0x02ae                  CCP2RBH = 0x2ae
                    0x02ae                  _CCP2RBH = 0x2ae
                    0x02b0                  CCP2BUFL = 0x2b0
                    0x02b0                  _CCP2BUFL = 0x2b0
                    0x02b2                  CCP2BUFH = 0x2b2
                    0x02b2                  _CCP2BUFH = 0x2b2
                    0x02b4                  CCP3CON1L = 0x2b4
                    0x02b4                  _CCP3CON1L = 0x2b4
                    0x02b4                  _CCP3CON1Lbits = 0x2b4
                    0x02b6                  CCP3CON1H = 0x2b6
                    0x02b6                  _CCP3CON1H = 0x2b6
                    0x02b6                  _CCP3CON1Hbits = 0x2b6
                    0x02b8                  CCP3CON2L = 0x2b8
                    0x02b8                  _CCP3CON2L = 0x2b8
                    0x02b8                  _CCP3CON2Lbits = 0x2b8
                    0x02ba                  CCP3CON2H = 0x2ba
                    0x02ba                  _CCP3CON2H = 0x2ba
                    0x02ba                  _CCP3CON2Hbits = 0x2ba
                    0x02bc                  CCP3CON3L = 0x2bc
                    0x02bc                  _CCP3CON3L = 0x2bc
                    0x02bc                  _CCP3CON3Lbits = 0x2bc
                    0x02be                  CCP3CON3H = 0x2be
                    0x02be                  _CCP3CON3H = 0x2be
                    0x02be                  _CCP3CON3Hbits = 0x2be
                    0x02c0                  CCP3STAT = 0x2c0
                    0x02c0                  _CCP3STAT = 0x2c0
                    0x02c0                  _CCP3STATbits = 0x2c0
                    0x02c0                  CCP3STATL = 0x2c0
                    0x02c0                  _CCP3STATL = 0x2c0
                    0x02c0                  _CCP3STATLbits = 0x2c0
                    0x02c2                  CCP3STATH = 0x2c2
                    0x02c2                  _CCP3STATH = 0x2c2
                    0x02c2                  _CCP3STATHbits = 0x2c2
                    0x02c4                  CCP3TMRL = 0x2c4
                    0x02c4                  _CCP3TMRL = 0x2c4
                    0x02c6                  CCP3TMRH = 0x2c6
                    0x02c6                  _CCP3TMRH = 0x2c6
                    0x02c8                  CCP3PRL = 0x2c8
                    0x02c8                  _CCP3PRL = 0x2c8
                    0x02ca                  CCP3PRH = 0x2ca
                    0x02ca                  _CCP3PRH = 0x2ca
                    0x02cc                  CCP3RA = 0x2cc
                    0x02cc                  _CCP3RA = 0x2cc
                    0x02cc                  CCP3RAL = 0x2cc
                    0x02cc                  _CCP3RAL = 0x2cc
                    0x02ce                  CCP3RAH = 0x2ce
                    0x02ce                  _CCP3RAH = 0x2ce
                    0x02d0                  CCP3RB = 0x2d0
                    0x02d0                  _CCP3RB = 0x2d0
                    0x02d0                  CCP3RBL = 0x2d0
                    0x02d0                  _CCP3RBL = 0x2d0
                    0x02d2                  CCP3RBH = 0x2d2
                    0x02d2                  _CCP3RBH = 0x2d2
                    0x02d4                  CCP3BUFL = 0x2d4
                    0x02d4                  _CCP3BUFL = 0x2d4
                    0x02d6                  CCP3BUFH = 0x2d6
                    0x02d6                  _CCP3BUFH = 0x2d6
                    0x02e6                  CMSTAT = 0x2e6
                    0x02e6                  _CMSTAT = 0x2e6
                    0x02e6                  _CMSTATbits = 0x2e6
                    0x02e8                  CVRCON = 0x2e8
                    0x02e8                  _CVRCON = 0x2e8
                    0x02e8                  _CVRCONbits = 0x2e8
                    0x02ea                  CM1CON = 0x2ea
                    0x02ea                  _CM1CON = 0x2ea
                    0x02ea                  _CM1CONbits = 0x2ea
                    0x02ec                  CM2CON = 0x2ec
                    0x02ec                  _CM2CON = 0x2ec
                    0x02ec                  _CM2CONbits = 0x2ec
                    0x02ee                  CM3CON = 0x2ee
                    0x02ee                  _CM3CON = 0x2ee
                    0x02ee                  _CM3CONbits = 0x2ee
                    0x02f4                  ANCFG = 0x2f4
                    0x02f4                  _ANCFG = 0x2f4
                    0x02f4                  _ANCFGbits = 0x2f4
                    0x02f8                  DAC1CON = 0x2f8
                    0x02f8                  _DAC1CON = 0x2f8
                    0x02f8                  _DAC1CONbits = 0x2f8
                    0x02fa                  DAC1DAT = 0x2fa
                    0x02fa                  _DAC1DAT = 0x2fa
                    0x0300                  CCP4CON1L = 0x300
                    0x0300                  _CCP4CON1L = 0x300
                    0x0300                  _CCP4CON1Lbits = 0x300
                    0x0302                  CCP4CON1H = 0x302
                    0x0302                  _CCP4CON1H = 0x302
                    0x0302                  _CCP4CON1Hbits = 0x302
                    0x0304                  CCP4CON2L = 0x304
                    0x0304                  _CCP4CON2L = 0x304
                    0x0304                  _CCP4CON2Lbits = 0x304
                    0x0306                  CCP4CON2H = 0x306
                    0x0306                  _CCP4CON2H = 0x306
                    0x0306                  _CCP4CON2Hbits = 0x306
                    0x0308                  CCP4CON3L = 0x308
                    0x0308                  _CCP4CON3L = 0x308
                    0x030a                  CCP4CON3H = 0x30a
                    0x030a                  _CCP4CON3H = 0x30a
                    0x030a                  _CCP4CON3Hbits = 0x30a
                    0x030c                  CCP4STAT = 0x30c
                    0x030c                  _CCP4STAT = 0x30c
                    0x030c                  _CCP4STATbits = 0x30c
                    0x030c                  CCP4STATL = 0x30c
                    0x030c                  _CCP4STATL = 0x30c
                    0x030c                  _CCP4STATLbits = 0x30c
                    0x030e                  CCP4STATH = 0x30e
                    0x030e                  _CCP4STATH = 0x30e
                    0x030e                  _CCP4STATHbits = 0x30e
                    0x0310                  CCP4TMRL = 0x310
                    0x0310                  _CCP4TMRL = 0x310
                    0x0312                  CCP4TMRH = 0x312
                    0x0312                  _CCP4TMRH = 0x312
                    0x0314                  CCP4PRL = 0x314
                    0x0314                  _CCP4PRL = 0x314
                    0x0316                  CCP4PRH = 0x316
                    0x0316                  _CCP4PRH = 0x316
                    0x0318                  CCP4RA = 0x318
                    0x0318                  _CCP4RA = 0x318
                    0x0318                  CCP4RAL = 0x318
                    0x0318                  _CCP4RAL = 0x318
                    0x031a                  CCP4RAH = 0x31a
                    0x031a                  _CCP4RAH = 0x31a
                    0x031c                  CCP4RB = 0x31c
                    0x031c                  _CCP4RB = 0x31c
                    0x031c                  CCP4RBL = 0x31c
                    0x031c                  _CCP4RBL = 0x31c
                    0x031e                  CCP4RBH = 0x31e
                    0x031e                  _CCP4RBH = 0x31e
                    0x0320                  CCP4BUFL = 0x320
                    0x0320                  _CCP4BUFL = 0x320
                    0x0322                  CCP4BUFH = 0x322
                    0x0322                  _CCP4BUFH = 0x322
                    0x0324                  CCP5CON1L = 0x324
                    0x0324                  _CCP5CON1L = 0x324
                    0x0324                  _CCP5CON1Lbits = 0x324
                    0x0326                  CCP5CON1H = 0x326
                    0x0326                  _CCP5CON1H = 0x326
                    0x0326                  _CCP5CON1Hbits = 0x326
                    0x0328                  CCP5CON2L = 0x328
                    0x0328                  _CCP5CON2L = 0x328
                    0x0328                  _CCP5CON2Lbits = 0x328
                    0x032a                  CCP5CON2H = 0x32a
                    0x032a                  _CCP5CON2H = 0x32a
                    0x032a                  _CCP5CON2Hbits = 0x32a
                    0x032c                  CCP5CON3L = 0x32c
                    0x032c                  _CCP5CON3L = 0x32c
                    0x032c                  _CCP5CON3Lbits = 0x32c
                    0x032e                  CCP5CON3H = 0x32e
                    0x032e                  _CCP5CON3H = 0x32e
                    0x032e                  _CCP5CON3Hbits = 0x32e
                    0x0330                  CCP5STAT = 0x330
                    0x0330                  _CCP5STAT = 0x330
                    0x0330                  _CCP5STATbits = 0x330
                    0x0330                  CCP5STATL = 0x330
                    0x0330                  _CCP5STATL = 0x330
                    0x0330                  _CCP5STATLbits = 0x330
                    0x0332                  CCP5STATH = 0x332
                    0x0332                  _CCP5STATH = 0x332
                    0x0332                  _CCP5STATHbits = 0x332
                    0x0334                  CCP5TMRL = 0x334
                    0x0334                  _CCP5TMRL = 0x334
                    0x0336                  CCP5TMRH = 0x336
                    0x0336                  _CCP5TMRH = 0x336
                    0x0338                  CCP5PRL = 0x338
                    0x0338                  _CCP5PRL = 0x338
                    0x033a                  CCP5PRH = 0x33a
                    0x033a                  _CCP5PRH = 0x33a
                    0x033c                  CCP5RA = 0x33c
                    0x033c                  _CCP5RA = 0x33c
                    0x033c                  CCP5RAL = 0x33c
                    0x033c                  _CCP5RAL = 0x33c
                    0x033e                  CCP5RAH = 0x33e
                    0x033e                  _CCP5RAH = 0x33e
                    0x0340                  CCP5RB = 0x340
                    0x0340                  _CCP5RB = 0x340
                    0x0340                  CCP5RBL = 0x340
                    0x0340                  _CCP5RBL = 0x340
                    0x0342                  CCP5RBH = 0x342
                    0x0342                  _CCP5RBH = 0x342
                    0x0344                  CCP5BUFL = 0x344
                    0x0344                  _CCP5BUFL = 0x344
                    0x0346                  CCP5BUFH = 0x346
                    0x0346                  _CCP5BUFH = 0x346
                    0x0348                  CCP6CON1L = 0x348
                    0x0348                  _CCP6CON1L = 0x348
                    0x0348                  _CCP6CON1Lbits = 0x348
                    0x034a                  CCP6CON1H = 0x34a
                    0x034a                  _CCP6CON1H = 0x34a
                    0x034a                  _CCP6CON1Hbits = 0x34a
                    0x034c                  CCP6CON2L = 0x34c
                    0x034c                  _CCP6CON2L = 0x34c
                    0x034c                  _CCP6CON2Lbits = 0x34c
                    0x034e                  CCP6CON2H = 0x34e
                    0x034e                  _CCP6CON2H = 0x34e
                    0x034e                  _CCP6CON2Hbits = 0x34e
                    0x0350                  CCP6CON3L = 0x350
                    0x0350                  _CCP6CON3L = 0x350
                    0x0350                  _CCP6CON3Lbits = 0x350
                    0x0352                  CCP6CON3H = 0x352
                    0x0352                  _CCP6CON3H = 0x352
                    0x0352                  _CCP6CON3Hbits = 0x352
                    0x0354                  CCP6STAT = 0x354
                    0x0354                  _CCP6STAT = 0x354
                    0x0354                  _CCP6STATbits = 0x354
                    0x0354                  CCP6STATL = 0x354
                    0x0354                  _CCP6STATL = 0x354
                    0x0354                  _CCP6STATLbits = 0x354
                    0x0356                  CCP6STATH = 0x356
                    0x0356                  _CCP6STATH = 0x356
                    0x0356                  _CCP6STATHbits = 0x356
                    0x0358                  CCP6TMRL = 0x358
                    0x0358                  _CCP6TMRL = 0x358
                    0x035a                  CCP6TMRH = 0x35a
                    0x035a                  _CCP6TMRH = 0x35a
                    0x035c                  CCP6PRL = 0x35c
                    0x035c                  _CCP6PRL = 0x35c
                    0x035e                  CCP6PRH = 0x35e
                    0x035e                  _CCP6PRH = 0x35e
                    0x0360                  CCP6RA = 0x360
                    0x0360                  _CCP6RA = 0x360
                    0x0360                  CCP6RAL = 0x360
                    0x0360                  _CCP6RAL = 0x360
                    0x0362                  CCP6RAH = 0x362
                    0x0362                  _CCP6RAH = 0x362
                    0x0364                  CCP6RB = 0x364
                    0x0364                  _CCP6RB = 0x364
                    0x0364                  CCP6RBL = 0x364
                    0x0364                  _CCP6RBL = 0x364
                    0x0366                  CCP6RBH = 0x366
                    0x0366                  _CCP6RBH = 0x366
                    0x0368                  CCP6BUFL = 0x368
                    0x0368                  _CCP6BUFL = 0x368
                    0x036a                  CCP6BUFH = 0x36a
                    0x036a                  _CCP6BUFH = 0x36a
                    0x036c                  CCP7CON1L = 0x36c
                    0x036c                  _CCP7CON1L = 0x36c
                    0x036c                  _CCP7CON1Lbits = 0x36c
                    0x036e                  CCP7CON1H = 0x36e
                    0x036e                  _CCP7CON1H = 0x36e
                    0x036e                  _CCP7CON1Hbits = 0x36e
                    0x0370                  CCP7CON2L = 0x370
                    0x0370                  _CCP7CON2L = 0x370
                    0x0370                  _CCP7CON2Lbits = 0x370
                    0x0372                  CCP7CON2H = 0x372
                    0x0372                  _CCP7CON2H = 0x372
                    0x0372                  _CCP7CON2Hbits = 0x372
                    0x0374                  CCP7CON3L = 0x374
                    0x0374                  _CCP7CON3L = 0x374
                    0x0374                  _CCP7CON3Lbits = 0x374
                    0x0376                  CCP7CON3H = 0x376
                    0x0376                  _CCP7CON3H = 0x376
                    0x0376                  _CCP7CON3Hbits = 0x376
                    0x0378                  CCP7STAT = 0x378
                    0x0378                  _CCP7STAT = 0x378
                    0x0378                  _CCP7STATbits = 0x378
                    0x0378                  CCP7STATL = 0x378
                    0x0378                  _CCP7STATL = 0x378
                    0x0378                  _CCP7STATLbits = 0x378
                    0x037a                  CCP7STATH = 0x37a
                    0x037a                  _CCP7STATH = 0x37a
                    0x037a                  _CCP7STATHbits = 0x37a
                    0x037c                  CCP7TMRL = 0x37c
                    0x037c                  _CCP7TMRL = 0x37c
                    0x037e                  CCP7TMRH = 0x37e
                    0x037e                  _CCP7TMRH = 0x37e
                    0x0380                  CCP7PRL = 0x380
                    0x0380                  _CCP7PRL = 0x380
                    0x0382                  CCP7PRH = 0x382
                    0x0382                  _CCP7PRH = 0x382
                    0x0384                  CCP7RA = 0x384
                    0x0384                  _CCP7RA = 0x384
                    0x0384                  CCP7RAL = 0x384
                    0x0384                  _CCP7RAL = 0x384
                    0x0386                  CCP7RAH = 0x386
                    0x0386                  _CCP7RAH = 0x386
                    0x0388                  CCP7RB = 0x388
                    0x0388                  _CCP7RB = 0x388
                    0x0388                  CCP7RBL = 0x388
                    0x0388                  _CCP7RBL = 0x388
                    0x038a                  CCP7RBH = 0x38a
                    0x038a                  _CCP7RBH = 0x38a
                    0x038c                  CCP7BUFL = 0x38c
                    0x038c                  _CCP7BUFL = 0x38c
                    0x038e                  CCP7BUFH = 0x38e
                    0x038e                  _CCP7BUFH = 0x38e
                    0x0398                  U1MODE = 0x398
                    0x0398                  _U1MODE = 0x398
                    0x0398                  _U1MODEbits = 0x398
                    0x039a                  U1STA = 0x39a
                    0x039a                  _U1STA = 0x39a
                    0x039a                  _U1STAbits = 0x39a
                    0x039c                  U1TXREG = 0x39c
                    0x039c                  _U1TXREG = 0x39c
                    0x039c                  _U1TXREGbits = 0x39c
                    0x039e                  U1RXREG = 0x39e
                    0x039e                  _U1RXREG = 0x39e
                    0x03a0                  U1BRG = 0x3a0
                    0x03a0                  _U1BRG = 0x3a0
                    0x03a2                  U1ADMD = 0x3a2
                    0x03a2                  _U1ADMD = 0x3a2
                    0x03a2                  _U1ADMDbits = 0x3a2
                    0x03a4                  U1SCCON = 0x3a4
                    0x03a4                  _U1SCCON = 0x3a4
                    0x03a4                  _U1SCCONbits = 0x3a4
                    0x03a6                  U1SCINT = 0x3a6
                    0x03a6                  _U1SCINT = 0x3a6
                    0x03a6                  _U1SCINTbits = 0x3a6
                    0x03a8                  U1GTC = 0x3a8
                    0x03a8                  _U1GTC = 0x3a8
                    0x03a8                  _U1GTCbits = 0x3a8
                    0x03aa                  U1WTCH = 0x3aa
                    0x03aa                  _U1WTCH = 0x3aa
                    0x03aa                  _U1WTCHbits = 0x3aa
                    0x03ac                  U1WTCL = 0x3ac
                    0x03ac                  _U1WTCL = 0x3ac
                    0x03ac                  _U1WTCLbits = 0x3ac
                    0x03ae                  U2MODE = 0x3ae
                    0x03ae                  _U2MODE = 0x3ae
                    0x03ae                  _U2MODEbits = 0x3ae
                    0x03b0                  U2STA = 0x3b0
                    0x03b0                  _U2STA = 0x3b0
                    0x03b0                  _U2STAbits = 0x3b0
                    0x03b2                  U2TXREG = 0x3b2
                    0x03b2                  _U2TXREG = 0x3b2
                    0x03b2                  _U2TXREGbits = 0x3b2
                    0x03b4                  U2RXREG = 0x3b4
                    0x03b4                  _U2RXREG = 0x3b4
                    0x03b6                  U2BRG = 0x3b6
                    0x03b6                  _U2BRG = 0x3b6
                    0x03b8                  U2ADMD = 0x3b8
                    0x03b8                  _U2ADMD = 0x3b8
                    0x03b8                  _U2ADMDbits = 0x3b8
                    0x03ba                  U2SCCON = 0x3ba
                    0x03ba                  _U2SCCON = 0x3ba
                    0x03ba                  _U2SCCONbits = 0x3ba
                    0x03bc                  U2SCINT = 0x3bc
                    0x03bc                  _U2SCINT = 0x3bc
                    0x03bc                  _U2SCINTbits = 0x3bc
                    0x03be                  U2GTC = 0x3be
                    0x03be                  _U2GTC = 0x3be
                    0x03be                  _U2GTCbits = 0x3be
                    0x03c0                  U2WTCH = 0x3c0
                    0x03c0                  _U2WTCH = 0x3c0
                    0x03c0                  _U2WTCHbits = 0x3c0
                    0x03c2                  U2WTCL = 0x3c2
                    0x03c2                  _U2WTCL = 0x3c2
                    0x03c2                  _U2WTCLbits = 0x3c2
                    0x03c4                  U3MODE = 0x3c4
                    0x03c4                  _U3MODE = 0x3c4
                    0x03c4                  _U3MODEbits = 0x3c4
                    0x03c6                  U3STA = 0x3c6
                    0x03c6                  _U3STA = 0x3c6
                    0x03c6                  _U3STAbits = 0x3c6
                    0x03c8                  U3TXREG = 0x3c8
                    0x03c8                  _U3TXREG = 0x3c8
                    0x03c8                  _U3TXREGbits = 0x3c8
                    0x03ca                  U3RXREG = 0x3ca
                    0x03ca                  _U3RXREG = 0x3ca
                    0x03cc                  U3BRG = 0x3cc
                    0x03cc                  _U3BRG = 0x3cc
                    0x03ce                  U3ADMD = 0x3ce
                    0x03ce                  _U3ADMD = 0x3ce
                    0x03ce                  _U3ADMDbits = 0x3ce
                    0x03d0                  U4MODE = 0x3d0
                    0x03d0                  _U4MODE = 0x3d0
                    0x03d0                  _U4MODEbits = 0x3d0
                    0x03d2                  U4STA = 0x3d2
                    0x03d2                  _U4STA = 0x3d2
                    0x03d2                  _U4STAbits = 0x3d2
                    0x03d4                  U4TXREG = 0x3d4
                    0x03d4                  _U4TXREG = 0x3d4
                    0x03d4                  _U4TXREGbits = 0x3d4
                    0x03d6                  U4RXREG = 0x3d6
                    0x03d6                  _U4RXREG = 0x3d6
                    0x03d8                  U4BRG = 0x3d8
                    0x03d8                  _U4BRG = 0x3d8
                    0x03da                  U4ADMD = 0x3da
                    0x03da                  _U4ADMD = 0x3da
                    0x03da                  _U4ADMDbits = 0x3da
                    0x03dc                  U5MODE = 0x3dc
                    0x03dc                  _U5MODE = 0x3dc
                    0x03dc                  _U5MODEbits = 0x3dc
                    0x03de                  U5STA = 0x3de
                    0x03de                  _U5STA = 0x3de
                    0x03de                  _U5STAbits = 0x3de
                    0x03e0                  U5TXREG = 0x3e0
                    0x03e0                  _U5TXREG = 0x3e0
                    0x03e0                  _U5TXREGbits = 0x3e0
                    0x03e2                  U5RXREG = 0x3e2
                    0x03e2                  _U5RXREG = 0x3e2
                    0x03e4                  U5BRG = 0x3e4
                    0x03e4                  _U5BRG = 0x3e4
                    0x03e6                  U5ADMD = 0x3e6
                    0x03e6                  _U5ADMD = 0x3e6
                    0x03e6                  _U5ADMDbits = 0x3e6
                    0x03e8                  U6MODE = 0x3e8
                    0x03e8                  _U6MODE = 0x3e8
                    0x03e8                  _U6MODEbits = 0x3e8
                    0x03ea                  U6STA = 0x3ea
                    0x03ea                  _U6STA = 0x3ea
                    0x03ea                  _U6STAbits = 0x3ea
                    0x03ec                  U6TXREG = 0x3ec
                    0x03ec                  _U6TXREG = 0x3ec
                    0x03ec                  _U6TXREGbits = 0x3ec
                    0x03ee                  U6RXREG = 0x3ee
                    0x03ee                  _U6RXREG = 0x3ee
                    0x03f0                  U6BRG = 0x3f0
                    0x03f0                  _U6BRG = 0x3f0
                    0x03f2                  U6ADMD = 0x3f2
                    0x03f2                  _U6ADMD = 0x3f2
                    0x03f2                  _U6ADMDbits = 0x3f2
                    0x03f4                  SPI1CON1 = 0x3f4
                    0x03f4                  _SPI1CON1 = 0x3f4
                    0x03f4                  _SPI1CON1bits = 0x3f4
                    0x03f4                  SPI1CON1L = 0x3f4
                    0x03f4                  _SPI1CON1L = 0x3f4
                    0x03f4                  _SPI1CON1Lbits = 0x3f4
                    0x03f6                  SPI1CON1H = 0x3f6
                    0x03f6                  _SPI1CON1H = 0x3f6
                    0x03f6                  _SPI1CON1Hbits = 0x3f6
                    0x03f6                  SPI1CON2 = 0x3f6
                    0x03f6                  _SPI1CON2 = 0x3f6
                    0x03f6                  _SPI1CON2bits = 0x3f6
                    0x03f8                  SPI1CON2L = 0x3f8
                    0x03f8                  _SPI1CON2L = 0x3f8
                    0x03f8                  _SPI1CON2Lbits = 0x3f8
                    0x03f8                  SPI1CON3 = 0x3f8
                    0x03f8                  _SPI1CON3 = 0x3f8
                    0x03f8                  _SPI1CON3bits = 0x3f8
                    0x03fa                  SPI1CON2H = 0x3fa
                    0x03fa                  _SPI1CON2H = 0x3fa
                    0x03fa                  SPI1CON4 = 0x3fa
                    0x03fa                  _SPI1CON4 = 0x3fa
                    0x03fc                  SPI1STATL = 0x3fc
                    0x03fc                  _SPI1STATL = 0x3fc
                    0x03fc                  _SPI1STATLbits = 0x3fc
                    0x03fe                  SPI1STATH = 0x3fe
                    0x03fe                  _SPI1STATH = 0x3fe
                    0x03fe                  _SPI1STATHbits = 0x3fe
                    0x0400                  SPI1BUFL = 0x400
                    0x0400                  _SPI1BUFL = 0x400
                    0x0400                  _SPI1BUFLbits = 0x400
                    0x0402                  SPI1BUFH = 0x402
                    0x0402                  _SPI1BUFH = 0x402
                    0x0402                  _SPI1BUFHbits = 0x402
                    0x0404                  SPI1BRGL = 0x404
                    0x0404                  _SPI1BRGL = 0x404
                    0x0404                  _SPI1BRGLbits = 0x404
                    0x0406                  SPI1BRGH = 0x406
                    0x0406                  _SPI1BRGH = 0x406
                    0x0408                  SPI1IMSK1 = 0x408
                    0x0408                  _SPI1IMSK1 = 0x408
                    0x0408                  _SPI1IMSK1bits = 0x408
                    0x0408                  SPI1IMSKL = 0x408
                    0x0408                  _SPI1IMSKL = 0x408
                    0x0408                  _SPI1IMSKLbits = 0x408
                    0x040a                  SPI1IMSK2 = 0x40a
                    0x040a                  _SPI1IMSK2 = 0x40a
                    0x040a                  _SPI1IMSK2bits = 0x40a
                    0x040a                  SPI1IMSKH = 0x40a
                    0x040a                  _SPI1IMSKH = 0x40a
                    0x040a                  _SPI1IMSKHbits = 0x40a
                    0x040c                  SPI1URDTL = 0x40c
                    0x040c                  _SPI1URDTL = 0x40c
                    0x040c                  _SPI1URDTLbits = 0x40c
                    0x040e                  SPI1URDTH = 0x40e
                    0x040e                  _SPI1URDTH = 0x40e
                    0x040e                  _SPI1URDTHbits = 0x40e
                    0x0410                  SPI2CON1 = 0x410
                    0x0410                  _SPI2CON1 = 0x410
                    0x0410                  _SPI2CON1bits = 0x410
                    0x0410                  SPI2CON1L = 0x410
                    0x0410                  _SPI2CON1L = 0x410
                    0x0410                  _SPI2CON1Lbits = 0x410
                    0x0412                  SPI2CON1H = 0x412
                    0x0412                  _SPI2CON1H = 0x412
                    0x0412                  _SPI2CON1Hbits = 0x412
                    0x0412                  SPI2CON2 = 0x412
                    0x0412                  _SPI2CON2 = 0x412
                    0x0412                  _SPI2CON2bits = 0x412
                    0x0414                  SPI2CON2L = 0x414
                    0x0414                  _SPI2CON2L = 0x414
                    0x0414                  _SPI2CON2Lbits = 0x414
                    0x0414                  SPI2CON3 = 0x414
                    0x0414                  _SPI2CON3 = 0x414
                    0x0414                  _SPI2CON3bits = 0x414
                    0x0416                  SPI2CON2H = 0x416
                    0x0416                  _SPI2CON2H = 0x416
                    0x0416                  SPI2CON4 = 0x416
                    0x0416                  _SPI2CON4 = 0x416
                    0x0418                  SPI2STATL = 0x418
                    0x0418                  _SPI2STATL = 0x418
                    0x0418                  _SPI2STATLbits = 0x418
                    0x041a                  SPI2STATH = 0x41a
                    0x041a                  _SPI2STATH = 0x41a
                    0x041a                  _SPI2STATHbits = 0x41a
                    0x041c                  SPI2BUFL = 0x41c
                    0x041c                  _SPI2BUFL = 0x41c
                    0x041c                  _SPI2BUFLbits = 0x41c
                    0x041e                  SPI2BUFH = 0x41e
                    0x041e                  _SPI2BUFH = 0x41e
                    0x041e                  _SPI2BUFHbits = 0x41e
                    0x0420                  SPI2BRGL = 0x420
                    0x0420                  _SPI2BRGL = 0x420
                    0x0420                  _SPI2BRGLbits = 0x420
                    0x0422                  SPI2BRGH = 0x422
                    0x0422                  _SPI2BRGH = 0x422
                    0x0424                  SPI2IMSK1 = 0x424
                    0x0424                  _SPI2IMSK1 = 0x424
                    0x0424                  _SPI2IMSK1bits = 0x424
                    0x0424                  SPI2IMSKL = 0x424
                    0x0424                  _SPI2IMSKL = 0x424
                    0x0424                  _SPI2IMSKLbits = 0x424
                    0x0426                  SPI2IMSK2 = 0x426
                    0x0426                  _SPI2IMSK2 = 0x426
                    0x0426                  _SPI2IMSK2bits = 0x426
                    0x0426                  SPI2IMSKH = 0x426
                    0x0426                  _SPI2IMSKH = 0x426
                    0x0426                  _SPI2IMSKHbits = 0x426
                    0x0428                  SPI2URDTL = 0x428
                    0x0428                  _SPI2URDTL = 0x428
                    0x0428                  _SPI2URDTLbits = 0x428
                    0x042a                  SPI2URDTH = 0x42a
                    0x042a                  _SPI2URDTH = 0x42a
                    0x042a                  _SPI2URDTHbits = 0x42a
                    0x042c                  SPI3CON1 = 0x42c
                    0x042c                  _SPI3CON1 = 0x42c
                    0x042c                  _SPI3CON1bits = 0x42c
                    0x042c                  SPI3CON1L = 0x42c
                    0x042c                  _SPI3CON1L = 0x42c
                    0x042c                  _SPI3CON1Lbits = 0x42c
                    0x042e                  SPI3CON1H = 0x42e
                    0x042e                  _SPI3CON1H = 0x42e
                    0x042e                  _SPI3CON1Hbits = 0x42e
                    0x042e                  SPI3CON2 = 0x42e
                    0x042e                  _SPI3CON2 = 0x42e
                    0x042e                  _SPI3CON2bits = 0x42e
                    0x0430                  SPI3CON2L = 0x430
                    0x0430                  _SPI3CON2L = 0x430
                    0x0430                  _SPI3CON2Lbits = 0x430
                    0x0430                  SPI3CON3 = 0x430
                    0x0430                  _SPI3CON3 = 0x430
                    0x0430                  _SPI3CON3bits = 0x430
                    0x0432                  SPI3CON2H = 0x432
                    0x0432                  _SPI3CON2H = 0x432
                    0x0432                  SPI3CON4 = 0x432
                    0x0432                  _SPI3CON4 = 0x432
                    0x0434                  SPI3STATL = 0x434
                    0x0434                  _SPI3STATL = 0x434
                    0x0434                  _SPI3STATLbits = 0x434
                    0x0436                  SPI3STATH = 0x436
                    0x0436                  _SPI3STATH = 0x436
                    0x0436                  _SPI3STATHbits = 0x436
                    0x0438                  SPI3BUFL = 0x438
                    0x0438                  _SPI3BUFL = 0x438
                    0x0438                  _SPI3BUFLbits = 0x438
                    0x043a                  SPI3BUFH = 0x43a
                    0x043a                  _SPI3BUFH = 0x43a
                    0x043a                  _SPI3BUFHbits = 0x43a
                    0x043c                  SPI3BRGL = 0x43c
                    0x043c                  _SPI3BRGL = 0x43c
                    0x043c                  _SPI3BRGLbits = 0x43c
                    0x043e                  SPI3BRGH = 0x43e
                    0x043e                  _SPI3BRGH = 0x43e
                    0x0440                  SPI3IMSK1 = 0x440
                    0x0440                  _SPI3IMSK1 = 0x440
                    0x0440                  _SPI3IMSK1bits = 0x440
                    0x0440                  SPI3IMSKL = 0x440
                    0x0440                  _SPI3IMSKL = 0x440
                    0x0440                  _SPI3IMSKLbits = 0x440
                    0x0442                  SPI3IMSK2 = 0x442
                    0x0442                  _SPI3IMSK2 = 0x442
                    0x0442                  _SPI3IMSK2bits = 0x442
                    0x0442                  SPI3IMSKH = 0x442
                    0x0442                  _SPI3IMSKH = 0x442
                    0x0442                  _SPI3IMSKHbits = 0x442
                    0x0444                  SPI3URDTL = 0x444
                    0x0444                  _SPI3URDTL = 0x444
                    0x0444                  _SPI3URDTLbits = 0x444
                    0x0446                  SPI3URDTH = 0x446
                    0x0446                  _SPI3URDTH = 0x446
                    0x0446                  _SPI3URDTHbits = 0x446
                    0x0448                  SPI4CON1 = 0x448
                    0x0448                  _SPI4CON1 = 0x448
                    0x0448                  _SPI4CON1bits = 0x448
                    0x0448                  SPI4CON1L = 0x448
                    0x0448                  _SPI4CON1L = 0x448
                    0x0448                  _SPI4CON1Lbits = 0x448
                    0x044a                  SPI4CON1H = 0x44a
                    0x044a                  _SPI4CON1H = 0x44a
                    0x044a                  _SPI4CON1Hbits = 0x44a
                    0x044a                  SPI4CON2 = 0x44a
                    0x044a                  _SPI4CON2 = 0x44a
                    0x044a                  _SPI4CON2bits = 0x44a
                    0x044c                  SPI4CON2L = 0x44c
                    0x044c                  _SPI4CON2L = 0x44c
                    0x044c                  _SPI4CON2Lbits = 0x44c
                    0x044c                  SPI4CON3 = 0x44c
                    0x044c                  _SPI4CON3 = 0x44c
                    0x044c                  _SPI4CON3bits = 0x44c
                    0x044e                  SPI4CON2H = 0x44e
                    0x044e                  _SPI4CON2H = 0x44e
                    0x044e                  SPI4CON4 = 0x44e
                    0x044e                  _SPI4CON4 = 0x44e
                    0x0450                  SPI4STATL = 0x450
                    0x0450                  _SPI4STATL = 0x450
                    0x0450                  _SPI4STATLbits = 0x450
                    0x0452                  SPI4STATH = 0x452
                    0x0452                  _SPI4STATH = 0x452
                    0x0452                  _SPI4STATHbits = 0x452
                    0x0454                  SPI4BUFL = 0x454
                    0x0454                  _SPI4BUFL = 0x454
                    0x0454                  _SPI4BUFLbits = 0x454
                    0x0456                  SPI4BUFH = 0x456
                    0x0456                  _SPI4BUFH = 0x456
                    0x0456                  _SPI4BUFHbits = 0x456
                    0x0458                  SPI4BRGL = 0x458
                    0x0458                  _SPI4BRGL = 0x458
                    0x0458                  _SPI4BRGLbits = 0x458
                    0x045a                  SPI4BRGH = 0x45a
                    0x045a                  _SPI4BRGH = 0x45a
                    0x045c                  SPI4IMSK1 = 0x45c
                    0x045c                  _SPI4IMSK1 = 0x45c
                    0x045c                  _SPI4IMSK1bits = 0x45c
                    0x045c                  SPI4IMSKL = 0x45c
                    0x045c                  _SPI4IMSKL = 0x45c
                    0x045c                  _SPI4IMSKLbits = 0x45c
                    0x045e                  SPI4IMSK2 = 0x45e
                    0x045e                  _SPI4IMSK2 = 0x45e
                    0x045e                  _SPI4IMSK2bits = 0x45e
                    0x045e                  SPI4IMSKH = 0x45e
                    0x045e                  _SPI4IMSKH = 0x45e
                    0x045e                  _SPI4IMSKHbits = 0x45e
                    0x0460                  SPI4URDTL = 0x460
                    0x0460                  _SPI4URDTL = 0x460
                    0x0460                  _SPI4URDTLbits = 0x460
                    0x0462                  SPI4URDTH = 0x462
                    0x0462                  _SPI4URDTH = 0x462
                    0x0462                  _SPI4URDTHbits = 0x462
                    0x0464                  CLC1CONL = 0x464
                    0x0464                  _CLC1CONL = 0x464
                    0x0464                  _CLC1CONLbits = 0x464
                    0x0466                  CLC1CONH = 0x466
                    0x0466                  _CLC1CONH = 0x466
                    0x0466                  _CLC1CONHbits = 0x466
                    0x0468                  CLC1SEL = 0x468
                    0x0468                  _CLC1SEL = 0x468
                    0x0468                  _CLC1SELbits = 0x468
                    0x0468                  CLC1SELL = 0x468
                    0x0468                  _CLC1SELL = 0x468
                    0x0468                  _CLC1SELLbits = 0x468
                    0x046c                  CLC1GLSL = 0x46c
                    0x046c                  _CLC1GLSL = 0x46c
                    0x046c                  _CLC1GLSLbits = 0x46c
                    0x046e                  CLC1GLSH = 0x46e
                    0x046e                  _CLC1GLSH = 0x46e
                    0x046e                  _CLC1GLSHbits = 0x46e
                    0x0470                  CLC2CONL = 0x470
                    0x0470                  _CLC2CONL = 0x470
                    0x0470                  _CLC2CONLbits = 0x470
                    0x0472                  CLC2CONH = 0x472
                    0x0472                  _CLC2CONH = 0x472
                    0x0472                  _CLC2CONHbits = 0x472
                    0x0474                  CLC2SEL = 0x474
                    0x0474                  _CLC2SEL = 0x474
                    0x0474                  _CLC2SELbits = 0x474
                    0x0474                  CLC2SELL = 0x474
                    0x0474                  _CLC2SELL = 0x474
                    0x0474                  _CLC2SELLbits = 0x474
                    0x0478                  CLC2GLSL = 0x478
                    0x0478                  _CLC2GLSL = 0x478
                    0x0478                  _CLC2GLSLbits = 0x478
                    0x047a                  CLC2GLSH = 0x47a
                    0x047a                  _CLC2GLSH = 0x47a
                    0x047a                  _CLC2GLSHbits = 0x47a
                    0x047c                  CLC3CONL = 0x47c
                    0x047c                  _CLC3CONL = 0x47c
                    0x047c                  _CLC3CONLbits = 0x47c
                    0x047e                  CLC3CONH = 0x47e
                    0x047e                  _CLC3CONH = 0x47e
                    0x047e                  _CLC3CONHbits = 0x47e
                    0x0480                  CLC3SEL = 0x480
                    0x0480                  _CLC3SEL = 0x480
                    0x0480                  _CLC3SELbits = 0x480
                    0x0480                  CLC3SELL = 0x480
                    0x0480                  _CLC3SELL = 0x480
                    0x0480                  _CLC3SELLbits = 0x480
                    0x0484                  CLC3GLSL = 0x484
                    0x0484                  _CLC3GLSL = 0x484
                    0x0484                  _CLC3GLSLbits = 0x484
                    0x0486                  CLC3GLSH = 0x486
                    0x0486                  _CLC3GLSH = 0x486
                    0x0486                  _CLC3GLSHbits = 0x486
                    0x0488                  CLC4CONL = 0x488
                    0x0488                  _CLC4CONL = 0x488
                    0x0488                  _CLC4CONLbits = 0x488
                    0x048a                  CLC4CONH = 0x48a
                    0x048a                  _CLC4CONH = 0x48a
                    0x048a                  _CLC4CONHbits = 0x48a
                    0x048c                  CLC4SEL = 0x48c
                    0x048c                  _CLC4SEL = 0x48c
                    0x048c                  _CLC4SELbits = 0x48c
                    0x048c                  CLC4SELL = 0x48c
                    0x048c                  _CLC4SELL = 0x48c
                    0x048c                  _CLC4SELLbits = 0x48c
                    0x0490                  CLC4GLSL = 0x490
                    0x0490                  _CLC4GLSL = 0x490
                    0x0490                  _CLC4GLSLbits = 0x490
                    0x0492                  CLC4GLSH = 0x492
                    0x0492                  _CLC4GLSH = 0x492
                    0x0492                  _CLC4GLSHbits = 0x492
                    0x0494                  I2C1RCV = 0x494
                    0x0494                  _I2C1RCV = 0x494
                    0x0494                  _I2C1RCVbits = 0x494
                    0x0496                  I2C1TRN = 0x496
                    0x0496                  _I2C1TRN = 0x496
                    0x0496                  _I2C1TRNbits = 0x496
                    0x0498                  I2C1BRG = 0x498
                    0x0498                  _I2C1BRG = 0x498
                    0x049a                  I2C1CON1 = 0x49a
                    0x049a                  _I2C1CON1 = 0x49a
                    0x049a                  _I2C1CON1bits = 0x49a
                    0x049a                  I2C1CONL = 0x49a
                    0x049a                  _I2C1CONL = 0x49a
                    0x049a                  _I2C1CONLbits = 0x49a
                    0x049c                  I2C1CON2 = 0x49c
                    0x049c                  _I2C1CON2 = 0x49c
                    0x049c                  _I2C1CON2bits = 0x49c
                    0x049c                  I2C1CONH = 0x49c
                    0x049c                  _I2C1CONH = 0x49c
                    0x049c                  _I2C1CONHbits = 0x49c
                    0x049e                  I2C1STAT = 0x49e
                    0x049e                  _I2C1STAT = 0x49e
                    0x049e                  _I2C1STATbits = 0x49e
                    0x04a0                  I2C1ADD = 0x4a0
                    0x04a0                  _I2C1ADD = 0x4a0
                    0x04a0                  _I2C1ADDbits = 0x4a0
                    0x04a2                  I2C1MSK = 0x4a2
                    0x04a2                  _I2C1MSK = 0x4a2
                    0x04a2                  _I2C1MSKbits = 0x4a2
                    0x04a4                  I2C2RCV = 0x4a4
                    0x04a4                  _I2C2RCV = 0x4a4
                    0x04a4                  _I2C2RCVbits = 0x4a4
                    0x04a6                  I2C2TRN = 0x4a6
                    0x04a6                  _I2C2TRN = 0x4a6
                    0x04a6                  _I2C2TRNbits = 0x4a6
                    0x04a8                  I2C2BRG = 0x4a8
                    0x04a8                  _I2C2BRG = 0x4a8
                    0x04aa                  I2C2CON1 = 0x4aa
                    0x04aa                  _I2C2CON1 = 0x4aa
                    0x04aa                  _I2C2CON1bits = 0x4aa
                    0x04aa                  I2C2CONL = 0x4aa
                    0x04aa                  _I2C2CONL = 0x4aa
                    0x04aa                  _I2C2CONLbits = 0x4aa
                    0x04ac                  I2C2CON2 = 0x4ac
                    0x04ac                  _I2C2CON2 = 0x4ac
                    0x04ac                  _I2C2CON2bits = 0x4ac
                    0x04ac                  I2C2CONH = 0x4ac
                    0x04ac                  _I2C2CONH = 0x4ac
                    0x04ac                  _I2C2CONHbits = 0x4ac
                    0x04ae                  I2C2STAT = 0x4ae
                    0x04ae                  _I2C2STAT = 0x4ae
                    0x04ae                  _I2C2STATbits = 0x4ae
                    0x04b0                  I2C2ADD = 0x4b0
                    0x04b0                  _I2C2ADD = 0x4b0
                    0x04b0                  _I2C2ADDbits = 0x4b0
                    0x04b2                  I2C2MSK = 0x4b2
                    0x04b2                  _I2C2MSK = 0x4b2
                    0x04b2                  _I2C2MSKbits = 0x4b2
                    0x04b4                  I2C3RCV = 0x4b4
                    0x04b4                  _I2C3RCV = 0x4b4
                    0x04b4                  _I2C3RCVbits = 0x4b4
                    0x04b6                  I2C3TRN = 0x4b6
                    0x04b6                  _I2C3TRN = 0x4b6
                    0x04b6                  _I2C3TRNbits = 0x4b6
                    0x04b8                  I2C3BRG = 0x4b8
                    0x04b8                  _I2C3BRG = 0x4b8
                    0x04ba                  I2C3CON1 = 0x4ba
                    0x04ba                  _I2C3CON1 = 0x4ba
                    0x04ba                  _I2C3CON1bits = 0x4ba
                    0x04ba                  I2C3CONL = 0x4ba
                    0x04ba                  _I2C3CONL = 0x4ba
                    0x04ba                  _I2C3CONLbits = 0x4ba
                    0x04bc                  I2C3CON2 = 0x4bc
                    0x04bc                  _I2C3CON2 = 0x4bc
                    0x04bc                  _I2C3CON2bits = 0x4bc
                    0x04bc                  I2C3CONH = 0x4bc
                    0x04bc                  _I2C3CONH = 0x4bc
                    0x04bc                  _I2C3CONHbits = 0x4bc
                    0x04be                  I2C3STAT = 0x4be
                    0x04be                  _I2C3STAT = 0x4be
                    0x04be                  _I2C3STATbits = 0x4be
                    0x04c0                  I2C3ADD = 0x4c0
                    0x04c0                  _I2C3ADD = 0x4c0
                    0x04c0                  _I2C3ADDbits = 0x4c0
                    0x04c2                  I2C3MSK = 0x4c2
                    0x04c2                  _I2C3MSK = 0x4c2
                    0x04c2                  _I2C3MSKbits = 0x4c2
                    0x04c4                  DMACON = 0x4c4
                    0x04c4                  _DMACON = 0x4c4
                    0x04c4                  _DMACONbits = 0x4c4
                    0x04c6                  DMABUF = 0x4c6
                    0x04c6                  _DMABUF = 0x4c6
                    0x04c8                  DMAL = 0x4c8
                    0x04c8                  _DMAL = 0x4c8
                    0x04ca                  DMAH = 0x4ca
                    0x04ca                  _DMAH = 0x4ca
                    0x04cc                  DMACH0 = 0x4cc
                    0x04cc                  _DMACH0 = 0x4cc
                    0x04cc                  _DMACH0bits = 0x4cc
                    0x04ce                  DMAINT0 = 0x4ce
                    0x04ce                  _DMAINT0 = 0x4ce
                    0x04ce                  _DMAINT0bits = 0x4ce
                    0x04d0                  DMASRC0 = 0x4d0
                    0x04d0                  _DMASRC0 = 0x4d0
                    0x04d2                  DMADST0 = 0x4d2
                    0x04d2                  _DMADST0 = 0x4d2
                    0x04d4                  DMACNT0 = 0x4d4
                    0x04d4                  _DMACNT0 = 0x4d4
                    0x04d6                  DMACH1 = 0x4d6
                    0x04d6                  _DMACH1 = 0x4d6
                    0x04d6                  _DMACH1bits = 0x4d6
                    0x04d8                  DMAINT1 = 0x4d8
                    0x04d8                  _DMAINT1 = 0x4d8
                    0x04d8                  _DMAINT1bits = 0x4d8
                    0x04da                  DMASRC1 = 0x4da
                    0x04da                  _DMASRC1 = 0x4da
                    0x04dc                  DMADST1 = 0x4dc
                    0x04dc                  _DMADST1 = 0x4dc
                    0x04de                  DMACNT1 = 0x4de
                    0x04de                  _DMACNT1 = 0x4de
                    0x04e0                  DMACH2 = 0x4e0
                    0x04e0                  _DMACH2 = 0x4e0
                    0x04e0                  _DMACH2bits = 0x4e0
                    0x04e2                  DMAINT2 = 0x4e2
                    0x04e2                  _DMAINT2 = 0x4e2
                    0x04e2                  _DMAINT2bits = 0x4e2
                    0x04e4                  DMASRC2 = 0x4e4
                    0x04e4                  _DMASRC2 = 0x4e4
                    0x04e6                  DMADST2 = 0x4e6
                    0x04e6                  _DMADST2 = 0x4e6
                    0x04e8                  DMACNT2 = 0x4e8
                    0x04e8                  _DMACNT2 = 0x4e8
                    0x04ea                  DMACH3 = 0x4ea
                    0x04ea                  _DMACH3 = 0x4ea
                    0x04ea                  _DMACH3bits = 0x4ea
                    0x04ec                  DMAINT3 = 0x4ec
                    0x04ec                  _DMAINT3 = 0x4ec
                    0x04ec                  _DMAINT3bits = 0x4ec
                    0x04ee                  DMASRC3 = 0x4ee
                    0x04ee                  _DMASRC3 = 0x4ee
                    0x04f0                  DMADST3 = 0x4f0
                    0x04f0                  _DMADST3 = 0x4f0
                    0x04f2                  DMACNT3 = 0x4f2
                    0x04f2                  _DMACNT3 = 0x4f2
                    0x04f4                  DMACH4 = 0x4f4
                    0x04f4                  _DMACH4 = 0x4f4
                    0x04f4                  _DMACH4bits = 0x4f4
                    0x04f6                  DMAINT4 = 0x4f6
                    0x04f6                  _DMAINT4 = 0x4f6
                    0x04f6                  _DMAINT4bits = 0x4f6
                    0x04f8                  DMASRC4 = 0x4f8
                    0x04f8                  _DMASRC4 = 0x4f8
                    0x04fa                  DMADST4 = 0x4fa
                    0x04fa                  _DMADST4 = 0x4fa
                    0x04fc                  DMACNT4 = 0x4fc
                    0x04fc                  _DMACNT4 = 0x4fc
                    0x04fe                  DMACH5 = 0x4fe
                    0x04fe                  _DMACH5 = 0x4fe
                    0x04fe                  _DMACH5bits = 0x4fe
                    0x0500                  DMAINT5 = 0x500
                    0x0500                  _DMAINT5 = 0x500
                    0x0500                  _DMAINT5bits = 0x500
                    0x0502                  DMASRC5 = 0x502
                    0x0502                  _DMASRC5 = 0x502
                    0x0504                  DMADST5 = 0x504
                    0x0504                  _DMADST5 = 0x504
                    0x0506                  DMACNT5 = 0x506
                    0x0506                  _DMACNT5 = 0x506
                    0x051c                  CRYCONL = 0x51c
                    0x051c                  _CRYCONL = 0x51c
                    0x051c                  _CRYCONLbits = 0x51c
                    0x051e                  CRYCONH = 0x51e
                    0x051e                  _CRYCONH = 0x51e
                    0x051e                  _CRYCONHbits = 0x51e
                    0x0520                  CRYSTAT = 0x520
                    0x0520                  _CRYSTAT = 0x520
                    0x0520                  _CRYSTATbits = 0x520
                    0x0524                  CRYOTP = 0x524
                    0x0524                  _CRYOTP = 0x524
                    0x0524                  _CRYOTPbits = 0x524
                    0x0528                  CRYKEY = 0x528
                    0x0528                  _CRYKEY = 0x528
                    0x0528                  CRYKEY0 = 0x528
                    0x0528                  _CRYKEY0 = 0x528
                    0x052a                  CRYKEY1 = 0x52a
                    0x052a                  _CRYKEY1 = 0x52a
                    0x052c                  CRYKEY2 = 0x52c
                    0x052c                  _CRYKEY2 = 0x52c
                    0x052e                  CRYKEY3 = 0x52e
                    0x052e                  _CRYKEY3 = 0x52e
                    0x0530                  CRYKEY4 = 0x530
                    0x0530                  _CRYKEY4 = 0x530
                    0x0532                  CRYKEY5 = 0x532
                    0x0532                  _CRYKEY5 = 0x532
                    0x0534                  CRYKEY6 = 0x534
                    0x0534                  _CRYKEY6 = 0x534
                    0x0536                  CRYKEY7 = 0x536
                    0x0536                  _CRYKEY7 = 0x536
                    0x0538                  CRYKEY8 = 0x538
                    0x0538                  _CRYKEY8 = 0x538
                    0x053a                  CRYKEY9 = 0x53a
                    0x053a                  _CRYKEY9 = 0x53a
                    0x053c                  CRYKEY10 = 0x53c
                    0x053c                  _CRYKEY10 = 0x53c
                    0x053e                  CRYKEY11 = 0x53e
                    0x053e                  _CRYKEY11 = 0x53e
                    0x0540                  CRYKEY12 = 0x540
                    0x0540                  _CRYKEY12 = 0x540
                    0x0542                  CRYKEY13 = 0x542
                    0x0542                  _CRYKEY13 = 0x542
                    0x0544                  CRYKEY14 = 0x544
                    0x0544                  _CRYKEY14 = 0x544
                    0x0546                  CRYKEY15 = 0x546
                    0x0546                  _CRYKEY15 = 0x546
                    0x0548                  CRYTXTA = 0x548
                    0x0548                  _CRYTXTA = 0x548
                    0x0548                  CRYTXTA0 = 0x548
                    0x0548                  _CRYTXTA0 = 0x548
                    0x054a                  CRYTXTA1 = 0x54a
                    0x054a                  _CRYTXTA1 = 0x54a
                    0x054c                  CRYTXTA2 = 0x54c
                    0x054c                  _CRYTXTA2 = 0x54c
                    0x054e                  CRYTXTA3 = 0x54e
                    0x054e                  _CRYTXTA3 = 0x54e
                    0x0550                  CRYTXTA4 = 0x550
                    0x0550                  _CRYTXTA4 = 0x550
                    0x0552                  CRYTXTA5 = 0x552
                    0x0552                  _CRYTXTA5 = 0x552
                    0x0554                  CRYTXTA6 = 0x554
                    0x0554                  _CRYTXTA6 = 0x554
                    0x0556                  CRYTXTA7 = 0x556
                    0x0556                  _CRYTXTA7 = 0x556
                    0x0558                  CRYTXTB = 0x558
                    0x0558                  _CRYTXTB = 0x558
                    0x0558                  CRYTXTB0 = 0x558
                    0x0558                  _CRYTXTB0 = 0x558
                    0x055a                  CRYTXTB1 = 0x55a
                    0x055a                  _CRYTXTB1 = 0x55a
                    0x055c                  CRYTXTB2 = 0x55c
                    0x055c                  _CRYTXTB2 = 0x55c
                    0x055e                  CRYTXTB3 = 0x55e
                    0x055e                  _CRYTXTB3 = 0x55e
                    0x0560                  CRYTXTB4 = 0x560
                    0x0560                  _CRYTXTB4 = 0x560
                    0x0562                  CRYTXTB5 = 0x562
                    0x0562                  _CRYTXTB5 = 0x562
                    0x0564                  CRYTXTB6 = 0x564
                    0x0564                  _CRYTXTB6 = 0x564
                    0x0566                  CRYTXTB7 = 0x566
                    0x0566                  _CRYTXTB7 = 0x566
                    0x0568                  CRYTXTC = 0x568
                    0x0568                  _CRYTXTC = 0x568
                    0x0568                  CRYTXTC0 = 0x568
                    0x0568                  _CRYTXTC0 = 0x568
                    0x056a                  CRYTXTC1 = 0x56a
                    0x056a                  _CRYTXTC1 = 0x56a
                    0x056c                  CRYTXTC2 = 0x56c
                    0x056c                  _CRYTXTC2 = 0x56c
                    0x056e                  CRYTXTC3 = 0x56e
                    0x056e                  _CRYTXTC3 = 0x56e
                    0x0570                  CRYTXTC4 = 0x570
                    0x0570                  _CRYTXTC4 = 0x570
                    0x0572                  CRYTXTC5 = 0x572
                    0x0572                  _CRYTXTC5 = 0x572
                    0x0574                  CRYTXTC6 = 0x574
                    0x0574                  _CRYTXTC6 = 0x574
                    0x0576                  CRYTXTC7 = 0x576
                    0x0576                  _CRYTXTC7 = 0x576
                    0x0578                  U1OTGIR = 0x578
                    0x0578                  _U1OTGIR = 0x578
                    0x0578                  _U1OTGIRbits = 0x578
                    0x057a                  U1OTGIE = 0x57a
                    0x057a                  _U1OTGIE = 0x57a
                    0x057a                  _U1OTGIEbits = 0x57a
                    0x057c                  U1OTGSTAT = 0x57c
                    0x057c                  _U1OTGSTAT = 0x57c
                    0x057c                  _U1OTGSTATbits = 0x57c
                    0x057e                  U1OTGCON = 0x57e
                    0x057e                  _U1OTGCON = 0x57e
                    0x057e                  _U1OTGCONbits = 0x57e
                    0x0580                  U1PWRC = 0x580
                    0x0580                  _U1PWRC = 0x580
                    0x0580                  _U1PWRCbits = 0x580
                    0x0582                  U1IR = 0x582
                    0x0582                  _U1IR = 0x582
                    0x0582                  _U1IRbits = 0x582
                    0x0584                  U1IE = 0x584
                    0x0584                  _U1IE = 0x584
                    0x0584                  _U1IEbits = 0x584
                    0x0586                  U1EIR = 0x586
                    0x0586                  _U1EIR = 0x586
                    0x0586                  _U1EIRbits = 0x586
                    0x0588                  U1EIE = 0x588
                    0x0588                  _U1EIE = 0x588
                    0x0588                  _U1EIEbits = 0x588
                    0x058a                  U1STAT = 0x58a
                    0x058a                  _U1STAT = 0x58a
                    0x058a                  _U1STATbits = 0x58a
                    0x058c                  U1CON = 0x58c
                    0x058c                  _U1CON = 0x58c
                    0x058c                  _U1CONbits = 0x58c
                    0x058e                  U1ADDR = 0x58e
                    0x058e                  _U1ADDR = 0x58e
                    0x058e                  _U1ADDRbits = 0x58e
                    0x0590                  U1BDTP1 = 0x590
                    0x0590                  _U1BDTP1 = 0x590
                    0x0590                  _U1BDTP1bits = 0x590
                    0x0592                  U1FRML = 0x592
                    0x0592                  _U1FRML = 0x592
                    0x0592                  _U1FRMLbits = 0x592
                    0x0594                  U1FRMH = 0x594
                    0x0594                  _U1FRMH = 0x594
                    0x0594                  _U1FRMHbits = 0x594
                    0x0596                  U1TOK = 0x596
                    0x0596                  _U1TOK = 0x596
                    0x0596                  _U1TOKbits = 0x596
                    0x0598                  U1SOF = 0x598
                    0x0598                  _U1SOF = 0x598
                    0x0598                  _U1SOFbits = 0x598
                    0x059a                  U1BDTP2 = 0x59a
                    0x059a                  _U1BDTP2 = 0x59a
                    0x059a                  _U1BDTP2bits = 0x59a
                    0x059c                  U1BDTP3 = 0x59c
                    0x059c                  _U1BDTP3 = 0x59c
                    0x059c                  _U1BDTP3bits = 0x59c
                    0x059e                  U1CNFG1 = 0x59e
                    0x059e                  _U1CNFG1 = 0x59e
                    0x059e                  _U1CNFG1bits = 0x59e
                    0x05a0                  U1CNFG2 = 0x5a0
                    0x05a0                  _U1CNFG2 = 0x5a0
                    0x05a0                  _U1CNFG2bits = 0x5a0
                    0x05a2                  U1EP0 = 0x5a2
                    0x05a2                  _U1EP0 = 0x5a2
                    0x05a2                  _U1EP0bits = 0x5a2
                    0x05a4                  U1EP1 = 0x5a4
                    0x05a4                  _U1EP1 = 0x5a4
                    0x05a4                  _U1EP1bits = 0x5a4
                    0x05a6                  U1EP2 = 0x5a6
                    0x05a6                  _U1EP2 = 0x5a6
                    0x05a6                  _U1EP2bits = 0x5a6
                    0x05a8                  U1EP3 = 0x5a8
                    0x05a8                  _U1EP3 = 0x5a8
                    0x05a8                  _U1EP3bits = 0x5a8
                    0x05aa                  U1EP4 = 0x5aa
                    0x05aa                  _U1EP4 = 0x5aa
                    0x05aa                  _U1EP4bits = 0x5aa
                    0x05ac                  U1EP5 = 0x5ac
                    0x05ac                  _U1EP5 = 0x5ac
                    0x05ac                  _U1EP5bits = 0x5ac
                    0x05ae                  U1EP6 = 0x5ae
                    0x05ae                  _U1EP6 = 0x5ae
                    0x05ae                  _U1EP6bits = 0x5ae
                    0x05b0                  U1EP7 = 0x5b0
                    0x05b0                  _U1EP7 = 0x5b0
                    0x05b0                  _U1EP7bits = 0x5b0
                    0x05b2                  U1EP8 = 0x5b2
                    0x05b2                  _U1EP8 = 0x5b2
                    0x05b2                  _U1EP8bits = 0x5b2
                    0x05b4                  U1EP9 = 0x5b4
                    0x05b4                  _U1EP9 = 0x5b4
                    0x05b4                  _U1EP9bits = 0x5b4
                    0x05b6                  U1EP10 = 0x5b6
                    0x05b6                  _U1EP10 = 0x5b6
                    0x05b6                  _U1EP10bits = 0x5b6
                    0x05b8                  U1EP11 = 0x5b8
                    0x05b8                  _U1EP11 = 0x5b8
                    0x05b8                  _U1EP11bits = 0x5b8
                    0x05ba                  U1EP12 = 0x5ba
                    0x05ba                  _U1EP12 = 0x5ba
                    0x05ba                  _U1EP12bits = 0x5ba
                    0x05bc                  U1EP13 = 0x5bc
                    0x05bc                  _U1EP13 = 0x5bc
                    0x05bc                  _U1EP13bits = 0x5bc
                    0x05be                  U1EP14 = 0x5be
                    0x05be                  _U1EP14 = 0x5be
                    0x05be                  _U1EP14bits = 0x5be
                    0x05c0                  U1EP15 = 0x5c0
                    0x05c0                  _U1EP15 = 0x5c0
                    0x05c0                  _U1EP15bits = 0x5c0
                    0x05c2                  LCDCON = 0x5c2
                    0x05c2                  _LCDCON = 0x5c2
                    0x05c2                  _LCDCONbits = 0x5c2
                    0x05c4                  LCDREF = 0x5c4
                    0x05c4                  _LCDREF = 0x5c4
                    0x05c4                  _LCDREFbits = 0x5c4
                    0x05c6                  LCDPS = 0x5c6
                    0x05c6                  _LCDPS = 0x5c6
                    0x05c6                  _LCDPSbits = 0x5c6
                    0x05c8                  LCDDATA0 = 0x5c8
                    0x05c8                  _LCDDATA0 = 0x5c8
                    0x05c8                  _LCDDATA0bits = 0x5c8
                    0x05ca                  LCDDATA1 = 0x5ca
                    0x05ca                  _LCDDATA1 = 0x5ca
                    0x05ca                  _LCDDATA1bits = 0x5ca
                    0x05cc                  LCDDATA2 = 0x5cc
                    0x05cc                  _LCDDATA2 = 0x5cc
                    0x05cc                  _LCDDATA2bits = 0x5cc
                    0x05ce                  LCDDATA3 = 0x5ce
                    0x05ce                  _LCDDATA3 = 0x5ce
                    0x05ce                  _LCDDATA3bits = 0x5ce
                    0x05d0                  LCDDATA4 = 0x5d0
                    0x05d0                  _LCDDATA4 = 0x5d0
                    0x05d0                  _LCDDATA4bits = 0x5d0
                    0x05d2                  LCDDATA5 = 0x5d2
                    0x05d2                  _LCDDATA5 = 0x5d2
                    0x05d2                  _LCDDATA5bits = 0x5d2
                    0x05d4                  LCDDATA6 = 0x5d4
                    0x05d4                  _LCDDATA6 = 0x5d4
                    0x05d4                  _LCDDATA6bits = 0x5d4
                    0x05d6                  LCDDATA7 = 0x5d6
                    0x05d6                  _LCDDATA7 = 0x5d6
                    0x05d6                  _LCDDATA7bits = 0x5d6
                    0x05d8                  LCDDATA8 = 0x5d8
                    0x05d8                  _LCDDATA8 = 0x5d8
                    0x05d8                  _LCDDATA8bits = 0x5d8
                    0x05da                  LCDDATA9 = 0x5da
                    0x05da                  _LCDDATA9 = 0x5da
                    0x05da                  _LCDDATA9bits = 0x5da
                    0x05dc                  LCDDATA10 = 0x5dc
                    0x05dc                  _LCDDATA10 = 0x5dc
                    0x05dc                  _LCDDATA10bits = 0x5dc
                    0x05de                  LCDDATA11 = 0x5de
                    0x05de                  _LCDDATA11 = 0x5de
                    0x05de                  _LCDDATA11bits = 0x5de
                    0x05e0                  LCDDATA12 = 0x5e0
                    0x05e0                  _LCDDATA12 = 0x5e0
                    0x05e0                  _LCDDATA12bits = 0x5e0
                    0x05e2                  LCDDATA13 = 0x5e2
                    0x05e2                  _LCDDATA13 = 0x5e2
                    0x05e2                  _LCDDATA13bits = 0x5e2
                    0x05e4                  LCDDATA14 = 0x5e4
                    0x05e4                  _LCDDATA14 = 0x5e4
                    0x05e4                  _LCDDATA14bits = 0x5e4
                    0x05e6                  LCDDATA15 = 0x5e6
                    0x05e6                  _LCDDATA15 = 0x5e6
                    0x05e6                  _LCDDATA15bits = 0x5e6
                    0x05e8                  LCDDATA16 = 0x5e8
                    0x05e8                  _LCDDATA16 = 0x5e8
                    0x05e8                  _LCDDATA16bits = 0x5e8
                    0x05ea                  LCDDATA17 = 0x5ea
                    0x05ea                  _LCDDATA17 = 0x5ea
                    0x05ea                  _LCDDATA17bits = 0x5ea
                    0x05ec                  LCDDATA18 = 0x5ec
                    0x05ec                  _LCDDATA18 = 0x5ec
                    0x05ec                  _LCDDATA18bits = 0x5ec
                    0x05ee                  LCDDATA19 = 0x5ee
                    0x05ee                  _LCDDATA19 = 0x5ee
                    0x05ee                  _LCDDATA19bits = 0x5ee
                    0x05f0                  LCDDATA20 = 0x5f0
                    0x05f0                  _LCDDATA20 = 0x5f0
                    0x05f0                  _LCDDATA20bits = 0x5f0
                    0x05f2                  LCDDATA21 = 0x5f2
                    0x05f2                  _LCDDATA21 = 0x5f2
                    0x05f2                  _LCDDATA21bits = 0x5f2
                    0x05f4                  LCDDATA22 = 0x5f4
                    0x05f4                  _LCDDATA22 = 0x5f4
                    0x05f4                  _LCDDATA22bits = 0x5f4
                    0x05f6                  LCDDATA23 = 0x5f6
                    0x05f6                  _LCDDATA23 = 0x5f6
                    0x05f6                  _LCDDATA23bits = 0x5f6
                    0x05f8                  LCDDATA24 = 0x5f8
                    0x05f8                  _LCDDATA24 = 0x5f8
                    0x05f8                  _LCDDATA24bits = 0x5f8
                    0x05fa                  LCDDATA25 = 0x5fa
                    0x05fa                  _LCDDATA25 = 0x5fa
                    0x05fa                  _LCDDATA25bits = 0x5fa
                    0x05fc                  LCDDATA26 = 0x5fc
                    0x05fc                  _LCDDATA26 = 0x5fc
                    0x05fc                  _LCDDATA26bits = 0x5fc
                    0x05fe                  LCDDATA27 = 0x5fe
                    0x05fe                  _LCDDATA27 = 0x5fe
                    0x05fe                  _LCDDATA27bits = 0x5fe
                    0x0600                  LCDDATA28 = 0x600
                    0x0600                  _LCDDATA28 = 0x600
                    0x0600                  _LCDDATA28bits = 0x600
                    0x0602                  LCDDATA29 = 0x602
                    0x0602                  _LCDDATA29 = 0x602
                    0x0602                  _LCDDATA29bits = 0x602
                    0x0604                  LCDDATA30 = 0x604
                    0x0604                  _LCDDATA30 = 0x604
                    0x0604                  _LCDDATA30bits = 0x604
                    0x0606                  LCDDATA31 = 0x606
                    0x0606                  _LCDDATA31 = 0x606
                    0x0606                  _LCDDATA31bits = 0x606
                    0x0608                  LCDSE0 = 0x608
                    0x0608                  _LCDSE0 = 0x608
                    0x0608                  _LCDSE0bits = 0x608
                    0x060a                  LCDSE1 = 0x60a
                    0x060a                  _LCDSE1 = 0x60a
                    0x060a                  _LCDSE1bits = 0x60a
                    0x060c                  LCDSE2 = 0x60c
                    0x060c                  _LCDSE2 = 0x60c
                    0x060c                  _LCDSE2bits = 0x60c
                    0x060e                  LCDSE3 = 0x60e
                    0x060e                  _LCDSE3 = 0x60e
                    0x060e                  _LCDSE3bits = 0x60e
                    0x0610                  LCDREG = 0x610
                    0x0610                  _LCDREG = 0x610
                    0x0610                  _LCDREGbits = 0x610
                    0x065a                  PADCON = 0x65a
                    0x065a                  _PADCON = 0x65a
                    0x065a                  _PADCONbits = 0x65a
                    0x065c                  IOCSTAT = 0x65c
                    0x065c                  _IOCSTAT = 0x65c
                    0x065c                  _IOCSTATbits = 0x65c
                    0x065e                  TRISA = 0x65e
                    0x065e                  _TRISA = 0x65e
                    0x065e                  _TRISAbits = 0x65e
                    0x0660                  PORTA = 0x660
                    0x0660                  _PORTA = 0x660
                    0x0660                  _PORTAbits = 0x660
                    0x0662                  LATA = 0x662
                    0x0662                  _LATA = 0x662
                    0x0662                  _LATAbits = 0x662
                    0x0664                  ODCA = 0x664
                    0x0664                  _ODCA = 0x664
                    0x0664                  _ODCAbits = 0x664
                    0x0666                  ANSA = 0x666
                    0x0666                  _ANSA = 0x666
                    0x0666                  _ANSAbits = 0x666
                    0x0668                  IOCPA = 0x668
                    0x0668                  _IOCPA = 0x668
                    0x0668                  _IOCPAbits = 0x668
                    0x066a                  IOCNA = 0x66a
                    0x066a                  _IOCNA = 0x66a
                    0x066a                  _IOCNAbits = 0x66a
                    0x066c                  IOCFA = 0x66c
                    0x066c                  _IOCFA = 0x66c
                    0x066c                  _IOCFAbits = 0x66c
                    0x066e                  IOCPUA = 0x66e
                    0x066e                  _IOCPUA = 0x66e
                    0x066e                  _IOCPUAbits = 0x66e
                    0x0670                  IOCPDA = 0x670
                    0x0670                  _IOCPDA = 0x670
                    0x0670                  _IOCPDAbits = 0x670
                    0x0672                  TRISB = 0x672
                    0x0672                  _TRISB = 0x672
                    0x0672                  _TRISBbits = 0x672
                    0x0674                  PORTB = 0x674
                    0x0674                  _PORTB = 0x674
                    0x0674                  _PORTBbits = 0x674
                    0x0676                  LATB = 0x676
                    0x0676                  _LATB = 0x676
                    0x0676                  _LATBbits = 0x676
                    0x0678                  ODCB = 0x678
                    0x0678                  _ODCB = 0x678
                    0x0678                  _ODCBbits = 0x678
                    0x067a                  ANSB = 0x67a
                    0x067a                  _ANSB = 0x67a
                    0x067a                  _ANSBbits = 0x67a
                    0x067c                  IOCPB = 0x67c
                    0x067c                  _IOCPB = 0x67c
                    0x067c                  _IOCPBbits = 0x67c
                    0x067e                  IOCNB = 0x67e
                    0x067e                  _IOCNB = 0x67e
                    0x067e                  _IOCNBbits = 0x67e
                    0x0680                  IOCFB = 0x680
                    0x0680                  _IOCFB = 0x680
                    0x0680                  _IOCFBbits = 0x680
                    0x0682                  IOCPUB = 0x682
                    0x0682                  _IOCPUB = 0x682
                    0x0682                  _IOCPUBbits = 0x682
                    0x0684                  IOCPDB = 0x684
                    0x0684                  _IOCPDB = 0x684
                    0x0684                  _IOCPDBbits = 0x684
                    0x0686                  TRISC = 0x686
                    0x0686                  _TRISC = 0x686
                    0x0686                  _TRISCbits = 0x686
                    0x0688                  PORTC = 0x688
                    0x0688                  _PORTC = 0x688
                    0x0688                  _PORTCbits = 0x688
                    0x068a                  LATC = 0x68a
                    0x068a                  _LATC = 0x68a
                    0x068a                  _LATCbits = 0x68a
                    0x068c                  ODCC = 0x68c
                    0x068c                  _ODCC = 0x68c
                    0x068c                  _ODCCbits = 0x68c
                    0x068e                  ANSC = 0x68e
                    0x068e                  _ANSC = 0x68e
                    0x068e                  _ANSCbits = 0x68e
                    0x0690                  IOCPC = 0x690
                    0x0690                  _IOCPC = 0x690
                    0x0690                  _IOCPCbits = 0x690
                    0x0692                  IOCNC = 0x692
                    0x0692                  _IOCNC = 0x692
                    0x0692                  _IOCNCbits = 0x692
                    0x0694                  IOCFC = 0x694
                    0x0694                  _IOCFC = 0x694
                    0x0694                  _IOCFCbits = 0x694
                    0x0696                  IOCPUC = 0x696
                    0x0696                  _IOCPUC = 0x696
                    0x0696                  _IOCPUCbits = 0x696
                    0x0698                  IOCPDC = 0x698
                    0x0698                  _IOCPDC = 0x698
                    0x0698                  _IOCPDCbits = 0x698
                    0x069a                  TRISD = 0x69a
                    0x069a                  _TRISD = 0x69a
                    0x069a                  _TRISDbits = 0x69a
                    0x069c                  PORTD = 0x69c
                    0x069c                  _PORTD = 0x69c
                    0x069c                  _PORTDbits = 0x69c
                    0x069e                  LATD = 0x69e
                    0x069e                  _LATD = 0x69e
                    0x069e                  _LATDbits = 0x69e
                    0x06a0                  ODCD = 0x6a0
                    0x06a0                  _ODCD = 0x6a0
                    0x06a0                  _ODCDbits = 0x6a0
                    0x06a2                  ANSD = 0x6a2
                    0x06a2                  _ANSD = 0x6a2
                    0x06a2                  _ANSDbits = 0x6a2
                    0x06a4                  IOCPD = 0x6a4
                    0x06a4                  _IOCPD = 0x6a4
                    0x06a4                  _IOCPDbits = 0x6a4
                    0x06a6                  IOCND = 0x6a6
                    0x06a6                  _IOCND = 0x6a6
                    0x06a6                  _IOCNDbits = 0x6a6
                    0x06a8                  IOCFD = 0x6a8
                    0x06a8                  _IOCFD = 0x6a8
                    0x06a8                  _IOCFDbits = 0x6a8
                    0x06aa                  IOCPUD = 0x6aa
                    0x06aa                  _IOCPUD = 0x6aa
                    0x06aa                  _IOCPUDbits = 0x6aa
                    0x06ac                  IOCPDD = 0x6ac
                    0x06ac                  _IOCPDD = 0x6ac
                    0x06ac                  _IOCPDDbits = 0x6ac
                    0x06ae                  TRISE = 0x6ae
                    0x06ae                  _TRISE = 0x6ae
                    0x06ae                  _TRISEbits = 0x6ae
                    0x06b0                  PORTE = 0x6b0
                    0x06b0                  _PORTE = 0x6b0
                    0x06b0                  _PORTEbits = 0x6b0
                    0x06b2                  LATE = 0x6b2
                    0x06b2                  _LATE = 0x6b2
                    0x06b2                  _LATEbits = 0x6b2
                    0x06b4                  ODCE = 0x6b4
                    0x06b4                  _ODCE = 0x6b4
                    0x06b4                  _ODCEbits = 0x6b4
                    0x06b6                  ANSE = 0x6b6
                    0x06b6                  _ANSE = 0x6b6
                    0x06b6                  _ANSEbits = 0x6b6
                    0x06b8                  IOCPE = 0x6b8
                    0x06b8                  _IOCPE = 0x6b8
                    0x06b8                  _IOCPEbits = 0x6b8
                    0x06ba                  IOCNE = 0x6ba
                    0x06ba                  _IOCNE = 0x6ba
                    0x06ba                  _IOCNEbits = 0x6ba
                    0x06bc                  IOCFE = 0x6bc
                    0x06bc                  _IOCFE = 0x6bc
                    0x06bc                  _IOCFEbits = 0x6bc
                    0x06be                  IOCPUE = 0x6be
                    0x06be                  _IOCPUE = 0x6be
                    0x06be                  _IOCPUEbits = 0x6be
                    0x06c0                  IOCPDE = 0x6c0
                    0x06c0                  _IOCPDE = 0x6c0
                    0x06c0                  _IOCPDEbits = 0x6c0
                    0x06c2                  TRISF = 0x6c2
                    0x06c2                  _TRISF = 0x6c2
                    0x06c2                  _TRISFbits = 0x6c2
                    0x06c4                  PORTF = 0x6c4
                    0x06c4                  _PORTF = 0x6c4
                    0x06c4                  _PORTFbits = 0x6c4
                    0x06c6                  LATF = 0x6c6
                    0x06c6                  _LATF = 0x6c6
                    0x06c6                  _LATFbits = 0x6c6
                    0x06c8                  ODCF = 0x6c8
                    0x06c8                  _ODCF = 0x6c8
                    0x06c8                  _ODCFbits = 0x6c8
                    0x06ca                  ANSF = 0x6ca
                    0x06ca                  _ANSF = 0x6ca
                    0x06ca                  _ANSFbits = 0x6ca
                    0x06cc                  IOCPF = 0x6cc
                    0x06cc                  _IOCPF = 0x6cc
                    0x06cc                  _IOCPFbits = 0x6cc
                    0x06ce                  IOCNF = 0x6ce
                    0x06ce                  _IOCNF = 0x6ce
                    0x06ce                  _IOCNFbits = 0x6ce
                    0x06d0                  IOCFF = 0x6d0
                    0x06d0                  _IOCFF = 0x6d0
                    0x06d0                  _IOCFFbits = 0x6d0
                    0x06d2                  IOCPUF = 0x6d2
                    0x06d2                  _IOCPUF = 0x6d2
                    0x06d2                  _IOCPUFbits = 0x6d2
                    0x06d4                  IOCPDF = 0x6d4
                    0x06d4                  _IOCPDF = 0x6d4
                    0x06d4                  _IOCPDFbits = 0x6d4
                    0x06d6                  TRISG = 0x6d6
                    0x06d6                  _TRISG = 0x6d6
                    0x06d6                  _TRISGbits = 0x6d6
                    0x06d8                  PORTG = 0x6d8
                    0x06d8                  _PORTG = 0x6d8
                    0x06d8                  _PORTGbits = 0x6d8
                    0x06da                  LATG = 0x6da
                    0x06da                  _LATG = 0x6da
                    0x06da                  _LATGbits = 0x6da
                    0x06dc                  ODCG = 0x6dc
                    0x06dc                  _ODCG = 0x6dc
                    0x06dc                  _ODCGbits = 0x6dc
                    0x06de                  ANSG = 0x6de
                    0x06de                  _ANSG = 0x6de
                    0x06de                  _ANSGbits = 0x6de
                    0x06e0                  IOCPG = 0x6e0
                    0x06e0                  _IOCPG = 0x6e0
                    0x06e0                  _IOCPGbits = 0x6e0
                    0x06e2                  IOCNG = 0x6e2
                    0x06e2                  _IOCNG = 0x6e2
                    0x06e2                  _IOCNGbits = 0x6e2
                    0x06e4                  IOCFG = 0x6e4
                    0x06e4                  _IOCFG = 0x6e4
                    0x06e4                  _IOCFGbits = 0x6e4
                    0x06e6                  IOCPUG = 0x6e6
                    0x06e6                  _IOCPUG = 0x6e6
                    0x06e6                  _IOCPUGbits = 0x6e6
                    0x06e8                  IOCPDG = 0x6e8
                    0x06e8                  _IOCPDG = 0x6e8
                    0x06e8                  _IOCPDGbits = 0x6e8
                    0x06ea                  TRISH = 0x6ea
                    0x06ea                  _TRISH = 0x6ea
                    0x06ea                  _TRISHbits = 0x6ea
                    0x06ec                  PORTH = 0x6ec
                    0x06ec                  _PORTH = 0x6ec
                    0x06ec                  _PORTHbits = 0x6ec
                    0x06ee                  LATH = 0x6ee
                    0x06ee                  _LATH = 0x6ee
                    0x06ee                  _LATHbits = 0x6ee
                    0x06f0                  ODCH = 0x6f0
                    0x06f0                  _ODCH = 0x6f0
                    0x06f0                  _ODCHbits = 0x6f0
                    0x06f2                  ANSH = 0x6f2
                    0x06f2                  _ANSH = 0x6f2
                    0x06f2                  _ANSHbits = 0x6f2
                    0x06f4                  IOCPH = 0x6f4
                    0x06f4                  _IOCPH = 0x6f4
                    0x06f4                  _IOCPHbits = 0x6f4
                    0x06f6                  IOCNH = 0x6f6
                    0x06f6                  _IOCNH = 0x6f6
                    0x06f6                  _IOCNHbits = 0x6f6
                    0x06f8                  IOCFH = 0x6f8
                    0x06f8                  _IOCFH = 0x6f8
                    0x06f8                  _IOCFHbits = 0x6f8
                    0x06fa                  IOCPUH = 0x6fa
                    0x06fa                  _IOCPUH = 0x6fa
                    0x06fa                  _IOCPUHbits = 0x6fa
                    0x06fc                  IOCPDH = 0x6fc
                    0x06fc                  _IOCPDH = 0x6fc
                    0x06fc                  _IOCPDHbits = 0x6fc
                    0x06fe                  TRISJ = 0x6fe
                    0x06fe                  _TRISJ = 0x6fe
                    0x06fe                  _TRISJbits = 0x6fe
                    0x0700                  PORTJ = 0x700
                    0x0700                  _PORTJ = 0x700
                    0x0700                  _PORTJbits = 0x700
                    0x0702                  LATJ = 0x702
                    0x0702                  _LATJ = 0x702
                    0x0702                  _LATJbits = 0x702
                    0x0704                  ODCJ = 0x704
                    0x0704                  _ODCJ = 0x704
                    0x0704                  _ODCJbits = 0x704
                    0x0706                  ANSJ = 0x706
                    0x0706                  _ANSJ = 0x706
                    0x0708                  IOCPJ = 0x708
                    0x0708                  _IOCPJ = 0x708
                    0x0708                  _IOCPJbits = 0x708
                    0x070a                  IOCNJ = 0x70a
                    0x070a                  _IOCNJ = 0x70a
                    0x070a                  _IOCNJbits = 0x70a
                    0x070c                  IOCFJ = 0x70c
                    0x070c                  _IOCFJ = 0x70c
                    0x070c                  _IOCFJbits = 0x70c
                    0x070e                  IOCPUJ = 0x70e
                    0x070e                  _IOCPUJ = 0x70e
                    0x070e                  _IOCPUJbits = 0x70e
                    0x0710                  IOCPDJ = 0x710
                    0x0710                  _IOCPDJ = 0x710
                    0x0710                  _IOCPDJbits = 0x710
                    0x0712                  ADC1BUF0 = 0x712
                    0x0712                  _ADC1BUF0 = 0x712
                    0x0714                  ADC1BUF1 = 0x714
                    0x0714                  _ADC1BUF1 = 0x714
                    0x0716                  ADC1BUF2 = 0x716
                    0x0716                  _ADC1BUF2 = 0x716
                    0x0718                  ADC1BUF3 = 0x718
                    0x0718                  _ADC1BUF3 = 0x718
                    0x071a                  ADC1BUF4 = 0x71a
                    0x071a                  _ADC1BUF4 = 0x71a
                    0x071c                  ADC1BUF5 = 0x71c
                    0x071c                  _ADC1BUF5 = 0x71c
                    0x071e                  ADC1BUF6 = 0x71e
                    0x071e                  _ADC1BUF6 = 0x71e
                    0x0720                  ADC1BUF7 = 0x720
                    0x0720                  _ADC1BUF7 = 0x720
                    0x0722                  ADC1BUF8 = 0x722
                    0x0722                  _ADC1BUF8 = 0x722
                    0x0724                  ADC1BUF9 = 0x724
                    0x0724                  _ADC1BUF9 = 0x724
                    0x0726                  ADC1BUF10 = 0x726
                    0x0726                  _ADC1BUF10 = 0x726
                    0x0728                  ADC1BUF11 = 0x728
                    0x0728                  _ADC1BUF11 = 0x728
                    0x072a                  ADC1BUF12 = 0x72a
                    0x072a                  _ADC1BUF12 = 0x72a
                    0x072c                  ADC1BUF13 = 0x72c
                    0x072c                  _ADC1BUF13 = 0x72c
                    0x072e                  ADC1BUF14 = 0x72e
                    0x072e                  _ADC1BUF14 = 0x72e
                    0x0730                  ADC1BUF15 = 0x730
                    0x0730                  _ADC1BUF15 = 0x730
                    0x0732                  ADC1BUF16 = 0x732
                    0x0732                  _ADC1BUF16 = 0x732
                    0x0734                  ADC1BUF17 = 0x734
                    0x0734                  _ADC1BUF17 = 0x734
                    0x0736                  ADC1BUF18 = 0x736
                    0x0736                  _ADC1BUF18 = 0x736
                    0x0738                  ADC1BUF19 = 0x738
                    0x0738                  _ADC1BUF19 = 0x738
                    0x073a                  ADC1BUF20 = 0x73a
                    0x073a                  _ADC1BUF20 = 0x73a
                    0x073c                  ADC1BUF21 = 0x73c
                    0x073c                  _ADC1BUF21 = 0x73c
                    0x073e                  ADC1BUF22 = 0x73e
                    0x073e                  _ADC1BUF22 = 0x73e
                    0x0740                  ADC1BUF23 = 0x740
                    0x0740                  _ADC1BUF23 = 0x740
                    0x0742                  ADC1BUF24 = 0x742
                    0x0742                  _ADC1BUF24 = 0x742
                    0x0744                  ADC1BUF25 = 0x744
                    0x0744                  _ADC1BUF25 = 0x744
                    0x0746                  AD1CON1 = 0x746
                    0x0746                  _AD1CON1 = 0x746
                    0x0746                  _AD1CON1bits = 0x746
                    0x0748                  AD1CON2 = 0x748
                    0x0748                  _AD1CON2 = 0x748
                    0x0748                  _AD1CON2bits = 0x748
                    0x074a                  AD1CON3 = 0x74a
                    0x074a                  _AD1CON3 = 0x74a
                    0x074a                  _AD1CON3bits = 0x74a
                    0x074c                  AD1CHS = 0x74c
                    0x074c                  _AD1CHS = 0x74c
                    0x074c                  _AD1CHSbits = 0x74c
                    0x074c                  AD1CHS0 = 0x74c
                    0x074c                  _AD1CHS0 = 0x74c
                    0x074c                  _AD1CHS0bits = 0x74c
                    0x074e                  AD1CSSH = 0x74e
                    0x074e                  _AD1CSSH = 0x74e
                    0x074e                  _AD1CSSHbits = 0x74e
                    0x0750                  AD1CSSL = 0x750
                    0x0750                  _AD1CSSL = 0x750
                    0x0750                  _AD1CSSLbits = 0x750
                    0x0752                  AD1CON4 = 0x752
                    0x0752                  _AD1CON4 = 0x752
                    0x0752                  _AD1CON4bits = 0x752
                    0x0754                  AD1CON5 = 0x754
                    0x0754                  _AD1CON5 = 0x754
                    0x0754                  _AD1CON5bits = 0x754
                    0x0756                  AD1CHITH = 0x756
                    0x0756                  _AD1CHITH = 0x756
                    0x0756                  _AD1CHITHbits = 0x756
                    0x0758                  AD1CHITL = 0x758
                    0x0758                  _AD1CHITL = 0x758
                    0x0758                  _AD1CHITLbits = 0x758
                    0x075a                  AD1CTMENH = 0x75a
                    0x075a                  _AD1CTMENH = 0x75a
                    0x075a                  _AD1CTMENHbits = 0x75a
                    0x075c                  AD1CTMENL = 0x75c
                    0x075c                  _AD1CTMENL = 0x75c
                    0x075c                  _AD1CTMENLbits = 0x75c
                    0x075e                  AD1RESDMA = 0x75e
                    0x075e                  _AD1RESDMA = 0x75e
                    0x0760                  NVMCON = 0x760
                    0x0760                  _NVMCON = 0x760
                    0x0760                  _NVMCONbits = 0x760
                    0x0762                  NVMADR = 0x762
                    0x0762                  _NVMADR = 0x762
                    0x0762                  _NVMADRbits = 0x762
                    0x0762                  NVMADRL = 0x762
                    0x0762                  _NVMADRL = 0x762
                    0x0762                  _NVMADRLbits = 0x762
                    0x0764                  NVMADRH = 0x764
                    0x0764                  _NVMADRH = 0x764
                    0x0764                  _NVMADRHbits = 0x764
                    0x0764                  NVMADRU = 0x764
                    0x0764                  _NVMADRU = 0x764
                    0x0764                  _NVMADRUbits = 0x764
                    0x0766                  NVMKEY = 0x766
                    0x0766                  _NVMKEY = 0x766
                    0x0768                  NVMSRCADRL = 0x768
                    0x0768                  _NVMSRCADRL = 0x768
                    0x0768                  _NVMSRCADRLbits = 0x768
                    0x076a                  NVMSRCADRH = 0x76a
                    0x076a                  _NVMSRCADRH = 0x76a
                    0x076a                  _NVMSRCADRHbits = 0x76a
                    0x077c                  JDATAL = 0x77c
                    0x077c                  _JDATAL = 0x77c
                    0x077e                  JDATAH = 0x77e
                    0x077e                  _JDATAH = 0x77e
                    0x0790                  RPINR0 = 0x790
                    0x0790                  _RPINR0 = 0x790
                    0x0790                  _RPINR0bits = 0x790
                    0x0792                  RPINR1 = 0x792
                    0x0792                  _RPINR1 = 0x792
                    0x0792                  _RPINR1bits = 0x792
                    0x0794                  RPINR2 = 0x794
                    0x0794                  _RPINR2 = 0x794
                    0x0794                  _RPINR2bits = 0x794
                    0x0796                  RPINR3 = 0x796
                    0x0796                  _RPINR3 = 0x796
                    0x0796                  _RPINR3bits = 0x796
                    0x0798                  RPINR4 = 0x798
                    0x0798                  _RPINR4 = 0x798
                    0x0798                  _RPINR4bits = 0x798
                    0x079a                  RPINR5 = 0x79a
                    0x079a                  _RPINR5 = 0x79a
                    0x079a                  _RPINR5bits = 0x79a
                    0x079c                  RPINR6 = 0x79c
                    0x079c                  _RPINR6 = 0x79c
                    0x079c                  _RPINR6bits = 0x79c
                    0x079e                  RPINR7 = 0x79e
                    0x079e                  _RPINR7 = 0x79e
                    0x079e                  _RPINR7bits = 0x79e
                    0x07a0                  RPINR8 = 0x7a0
                    0x07a0                  _RPINR8 = 0x7a0
                    0x07a0                  _RPINR8bits = 0x7a0
                    0x07a2                  RPINR9 = 0x7a2
                    0x07a2                  _RPINR9 = 0x7a2
                    0x07a2                  _RPINR9bits = 0x7a2
                    0x07a4                  RPINR10 = 0x7a4
                    0x07a4                  _RPINR10 = 0x7a4
                    0x07a4                  _RPINR10bits = 0x7a4
                    0x07a6                  RPINR11 = 0x7a6
                    0x07a6                  _RPINR11 = 0x7a6
                    0x07a6                  _RPINR11bits = 0x7a6
                    0x07a8                  RPINR12 = 0x7a8
                    0x07a8                  _RPINR12 = 0x7a8
                    0x07a8                  _RPINR12bits = 0x7a8
                    0x07aa                  RPINR13 = 0x7aa
                    0x07aa                  _RPINR13 = 0x7aa
                    0x07aa                  _RPINR13bits = 0x7aa
                    0x07ac                  RPINR14 = 0x7ac
                    0x07ac                  _RPINR14 = 0x7ac
                    0x07ac                  _RPINR14bits = 0x7ac
                    0x07ae                  RPINR15 = 0x7ae
                    0x07ae                  _RPINR15 = 0x7ae
                    0x07ae                  _RPINR15bits = 0x7ae
                    0x07b0                  RPINR16 = 0x7b0
                    0x07b0                  _RPINR16 = 0x7b0
                    0x07b0                  _RPINR16bits = 0x7b0
                    0x07b2                  RPINR17 = 0x7b2
                    0x07b2                  _RPINR17 = 0x7b2
                    0x07b2                  _RPINR17bits = 0x7b2
                    0x07b4                  RPINR18 = 0x7b4
                    0x07b4                  _RPINR18 = 0x7b4
                    0x07b4                  _RPINR18bits = 0x7b4
                    0x07b6                  RPINR19 = 0x7b6
                    0x07b6                  _RPINR19 = 0x7b6
                    0x07b6                  _RPINR19bits = 0x7b6
                    0x07b8                  RPINR20 = 0x7b8
                    0x07b8                  _RPINR20 = 0x7b8
                    0x07b8                  _RPINR20bits = 0x7b8
                    0x07ba                  RPINR21 = 0x7ba
                    0x07ba                  _RPINR21 = 0x7ba
                    0x07ba                  _RPINR21bits = 0x7ba
                    0x07bc                  RPINR22 = 0x7bc
                    0x07bc                  _RPINR22 = 0x7bc
                    0x07bc                  _RPINR22bits = 0x7bc
                    0x07be                  RPINR23 = 0x7be
                    0x07be                  _RPINR23 = 0x7be
                    0x07be                  _RPINR23bits = 0x7be
                    0x07c0                  RPINR24 = 0x7c0
                    0x07c0                  _RPINR24 = 0x7c0
                    0x07c0                  _RPINR24bits = 0x7c0
                    0x07c2                  RPINR25 = 0x7c2
                    0x07c2                  _RPINR25 = 0x7c2
                    0x07c2                  _RPINR25bits = 0x7c2
                    0x07c4                  RPINR26 = 0x7c4
                    0x07c4                  _RPINR26 = 0x7c4
                    0x07c4                  _RPINR26bits = 0x7c4
                    0x07c6                  RPINR27 = 0x7c6
                    0x07c6                  _RPINR27 = 0x7c6
                    0x07c6                  _RPINR27bits = 0x7c6
                    0x07c8                  RPINR28 = 0x7c8
                    0x07c8                  _RPINR28 = 0x7c8
                    0x07c8                  _RPINR28bits = 0x7c8
                    0x07ca                  RPINR29 = 0x7ca
                    0x07ca                  _RPINR29 = 0x7ca
                    0x07ca                  _RPINR29bits = 0x7ca
                    0x07cc                  RPINR30 = 0x7cc
                    0x07cc                  _RPINR30 = 0x7cc
                    0x07cc                  _RPINR30bits = 0x7cc
                    0x07ce                  RPINR31 = 0x7ce
                    0x07ce                  _RPINR31 = 0x7ce
                    0x07ce                  _RPINR31bits = 0x7ce
                    0x07d4                  RPOR0 = 0x7d4
                    0x07d4                  _RPOR0 = 0x7d4
                    0x07d4                  _RPOR0bits = 0x7d4
                    0x07d6                  RPOR1 = 0x7d6
                    0x07d6                  _RPOR1 = 0x7d6
                    0x07d6                  _RPOR1bits = 0x7d6
                    0x07d8                  RPOR2 = 0x7d8
                    0x07d8                  _RPOR2 = 0x7d8
                    0x07d8                  _RPOR2bits = 0x7d8
                    0x07da                  RPOR3 = 0x7da
                    0x07da                  _RPOR3 = 0x7da
                    0x07da                  _RPOR3bits = 0x7da
                    0x07dc                  RPOR4 = 0x7dc
                    0x07dc                  _RPOR4 = 0x7dc
                    0x07dc                  _RPOR4bits = 0x7dc
                    0x07de                  RPOR5 = 0x7de
                    0x07de                  _RPOR5 = 0x7de
                    0x07de                  _RPOR5bits = 0x7de
                    0x07e0                  RPOR6 = 0x7e0
                    0x07e0                  _RPOR6 = 0x7e0
                    0x07e0                  _RPOR6bits = 0x7e0
                    0x07e2                  RPOR7 = 0x7e2
                    0x07e2                  _RPOR7 = 0x7e2
                    0x07e2                  _RPOR7bits = 0x7e2
                    0x07e4                  RPOR8 = 0x7e4
                    0x07e4                  _RPOR8 = 0x7e4
                    0x07e4                  _RPOR8bits = 0x7e4
                    0x07e6                  RPOR9 = 0x7e6
                    0x07e6                  _RPOR9 = 0x7e6
                    0x07e6                  _RPOR9bits = 0x7e6
                    0x07e8                  RPOR10 = 0x7e8
                    0x07e8                  _RPOR10 = 0x7e8
                    0x07e8                  _RPOR10bits = 0x7e8
                    0x07ea                  RPOR11 = 0x7ea
                    0x07ea                  _RPOR11 = 0x7ea
                    0x07ea                  _RPOR11bits = 0x7ea
                    0x07ec                  RPOR12 = 0x7ec
                    0x07ec                  _RPOR12 = 0x7ec
                    0x07ec                  _RPOR12bits = 0x7ec
                    0x07ee                  RPOR13 = 0x7ee
                    0x07ee                  _RPOR13 = 0x7ee
                    0x07ee                  _RPOR13bits = 0x7ee
                    0x07f0                  RPOR14 = 0x7f0
                    0x07f0                  _RPOR14 = 0x7f0
                    0x07f0                  _RPOR14bits = 0x7f0
                    0x07f2                  RPOR15 = 0x7f2
                    0x07f2                  _RPOR15 = 0x7f2
                    0x07f2                  _RPOR15bits = 0x7f2
                    0x0204                  IC1 = 0x204
                    0x0204                  _IC1 = 0x204
                    0x020c                  IC2 = 0x20c
                    0x020c                  _IC2 = 0x20c
                    0x0214                  IC3 = 0x214
                    0x0214                  _IC3 = 0x214
                    0x021c                  IC4 = 0x21c
                    0x021c                  _IC4 = 0x21c
                    0x0224                  IC5 = 0x224
                    0x0224                  _IC5 = 0x224
                    0x022c                  IC6 = 0x22c
                    0x022c                  _IC6 = 0x22c
                    0x0234                  OC1 = 0x234
                    0x0234                  _OC1 = 0x234
                    0x023e                  OC2 = 0x23e
                    0x023e                  _OC2 = 0x23e
                    0x0248                  OC3 = 0x248
                    0x0248                  _OC3 = 0x248
                    0x0252                  OC4 = 0x252
                    0x0252                  _OC4 = 0x252
                    0x025c                  OC5 = 0x25c
                    0x025c                  _OC5 = 0x25c
                    0x0266                  OC6 = 0x266
                    0x0266                  _OC6 = 0x266
                    0x0398                  UART1 = 0x398
                    0x0398                  _UART1 = 0x398
                    0x03ae                  UART2 = 0x3ae
                    0x03ae                  _UART2 = 0x3ae
START GROUP
LOAD c:/program files (x86)/microchip/xc16/v1.25/bin/bin/../../lib\libpic30-elf.a
LOAD c:/program files (x86)/microchip/xc16/v1.25/bin/bin/../../lib\libm-elf.a
LOAD c:/program files (x86)/microchip/xc16/v1.25/bin/bin/../../lib\libc-elf.a
END GROUP
OUTPUT(dist/default/production/O5DaughterDbg.production.elf elf32-pic30)
LOAD jump_table
LOAD default_isr
LOAD data_init

.debug_pubtypes
                  0x000240        0xff8
 .debug_pubtypes
                  0x000240         0x9b build/default/production/_ext/1470100448/mbascii.o
 .debug_pubtypes
                  0x0002db         0x49 build/default/production/_ext/833655638/mbfunccoils.o
 .debug_pubtypes
                  0x000324         0x49 build/default/production/_ext/833655638/mbfuncdisc.o
 .debug_pubtypes
                  0x00036d         0x49 build/default/production/_ext/833655638/mbfuncholding.o
 .debug_pubtypes
                  0x0003b6         0x49 build/default/production/_ext/833655638/mbfuncinput.o
 .debug_pubtypes
                  0x0003ff         0x67 build/default/production/_ext/833655638/mbfuncother.o
 .debug_pubtypes
                  0x000466         0x54 build/default/production/_ext/833655638/mbutils.o
 .debug_pubtypes
                  0x0004ba         0x36 build/default/production/_ext/1433339410/portevent.o
 .debug_pubtypes
                  0x0004f0        0x102 build/default/production/_ext/1433339410/portserial.o
 .debug_pubtypes
                  0x0005f2         0xa6 build/default/production/_ext/1433339410/porttimer.o
 .debug_pubtypes
                  0x000698         0x27 build/default/production/_ext/1477781822/mbcrc.o
 .debug_pubtypes
                  0x0006bf         0x8c build/default/production/_ext/1477781822/mbrtu.o
 .debug_pubtypes
                  0x00074b         0x12 build/default/production/_ext/1043210786/debug.o
 .debug_pubtypes
                  0x00075d        0x11f build/default/production/_ext/1043210786/mb.o
 .debug_pubtypes
                  0x00087c        0x10a build/default/production/_ext/1472/main.o
 .debug_pubtypes
                  0x000986         0x1e build/default/production/_ext/1472/mcc.o
 .debug_pubtypes
                  0x0009a4        0x2a5 build/default/production/_ext/1472/periph.o
 .debug_pubtypes
                  0x000c49         0xb2 build/default/production/_ext/1472/sys_timer.o
 .debug_pubtypes
                  0x000cfb         0x8f build/default/production/_ext/1472/misc.o
 .debug_pubtypes
                  0x000d8a         0x2b build/default/production/_ext/1472/buffer.o
 .debug_pubtypes
                  0x000db5        0x369 build/default/production/_ext/1472/serial.o
 .debug_pubtypes
                  0x00111e         0x31 build/default/production/_ext/1472/config.o
 .debug_pubtypes
                  0x00114f         0x6c build/default/production/_ext/1472/flash_mem.o
 .debug_pubtypes
                  0x0011bb         0x2a build/default/production/_ext/1472/inst_port.o
 .debug_pubtypes
                  0x0011e5         0x53 build/default/production/_ext/1472/dig_io.o

__c30_signature
                  0x001238        0x1c2
 __c30_signature
                  0x001238          0x6 build/default/production/_ext/1470100448/mbascii.o
 __c30_signature
                  0x00123e          0x6 build/default/production/_ext/833655638/mbfunccoils.o
 __c30_signature
                  0x001244          0x6 build/default/production/_ext/833655638/mbfuncdiag.o
 __c30_signature
                  0x00124a          0x6 build/default/production/_ext/833655638/mbfuncdisc.o
 __c30_signature
                  0x001250          0x6 build/default/production/_ext/833655638/mbfuncholding.o
 __c30_signature
                  0x001256          0x6 build/default/production/_ext/833655638/mbfuncinput.o
 __c30_signature
                  0x00125c          0x6 build/default/production/_ext/833655638/mbfuncother.o
 __c30_signature
                  0x001262          0x6 build/default/production/_ext/833655638/mbutils.o
 __c30_signature
                  0x001268          0x6 build/default/production/_ext/1433339410/portevent.o
 __c30_signature
                  0x00126e          0x6 build/default/production/_ext/1433339410/portserial.o
 __c30_signature
                  0x001274          0x6 build/default/production/_ext/1433339410/porttimer.o
 __c30_signature
                  0x00127a          0x6 build/default/production/_ext/1477781822/mbcrc.o
 __c30_signature
                  0x001280          0x6 build/default/production/_ext/1477781822/mbrtu.o
 __c30_signature
                  0x001286          0x6 build/default/production/_ext/1043210786/debug.o
 __c30_signature
                  0x00128c          0x6 build/default/production/_ext/1043210786/mb.o
 __c30_signature
                  0x001292          0x6 build/default/production/_ext/1472/main.o
 __c30_signature
                  0x001298          0x6 build/default/production/_ext/1472/mcc.o
 __c30_signature
                  0x00129e          0x6 build/default/production/_ext/1472/periph.o
 __c30_signature
                  0x0012a4          0x6 build/default/production/_ext/1472/sys_timer.o
 __c30_signature
                  0x0012aa          0x6 build/default/production/_ext/1472/misc.o
 __c30_signature
                  0x0012b0          0x6 build/default/production/_ext/1472/buffer.o
 __c30_signature
                  0x0012b6          0x6 build/default/production/_ext/1472/serial.o
 __c30_signature
                  0x0012bc          0x6 build/default/production/_ext/1472/config.o
 __c30_signature
                  0x0012c2          0x6 build/default/production/_ext/1472/flash_mem.o
 __c30_signature
                  0x0012c8          0x6 build/default/production/_ext/1472/inst_port.o
 __c30_signature
                  0x0012ce          0x6 build/default/production/_ext/1472/dig_io.o
 __c30_signature
                  0x0012d4          0x6 c:/program files (x86)/microchip/xc16/v1.25/bin/bin/../../lib\libpic30-elf.a(crt0_extended.o)
 __c30_signature
                  0x0012da          0x6 c:/program files (x86)/microchip/xc16/v1.25/bin/bin/../../lib\libpic30-elf.a(data_init_extended.o)
 __c30_signature
                  0x0012e0          0x6 c:/program files (x86)/microchip/xc16/v1.25/bin/bin/../../lib\libm-elf.a(divsi3.eo)
 __c30_signature
                  0x0012e6          0x6 c:/program files (x86)/microchip/xc16/v1.25/bin/bin/../../lib\libm-elf.a(udivsi3.eo)
 __c30_signature
                  0x0012ec          0x6 c:/program files (x86)/microchip/xc16/v1.25/bin/bin/../../lib\libc-elf.a(atoi.eo)
 __c30_signature
                  0x0012f2          0x6 c:/program files (x86)/microchip/xc16/v1.25/bin/bin/../../lib\libc-elf.a(atol.eo)
 __c30_signature
                  0x0012f8          0x6 c:/program files (x86)/microchip/xc16/v1.25/bin/bin/../../lib\libc-elf.a(fassert.eo)
 __c30_signature
                  0x0012fe          0x6 c:/program files (x86)/microchip/xc16/v1.25/bin/bin/../../lib\libc-elf.a(fprintf.eo)
 __c30_signature
                  0x001304          0x6 c:/program files (x86)/microchip/xc16/v1.25/bin/bin/../../lib\libc-elf.a(memcpy.eo)
 __c30_signature
                  0x00130a          0x6 c:/program files (x86)/microchip/xc16/v1.25/bin/bin/../../lib\libc-elf.a(memset.eo)
 __c30_signature
                  0x001310          0x6 c:/program files (x86)/microchip/xc16/v1.25/bin/bin/../../lib\libc-elf.a(strtol.eo)
 __c30_signature
                  0x001316          0x6 c:/program files (x86)/microchip/xc16/v1.25/bin/bin/../../lib\libc-elf.a(signal.eo)
 __c30_signature
                  0x00131c          0x6 c:/program files (x86)/microchip/xc16/v1.25/bin/bin/../../lib\libc-elf.a(_iob.eo)
 __c30_signature
                  0x001322          0x6 c:/program files (x86)/microchip/xc16/v1.25/bin/bin/../../lib\libc-elf.a(errno.elo)
 __c30_signature
                  0x001328          0x6 c:/program files (x86)/microchip/xc16/v1.25/bin/bin/../../lib\libc-elf.a(exit.elo)
 __c30_signature
                  0x00132e          0x6 c:/program files (x86)/microchip/xc16/v1.25/bin/bin/../../lib\libc-elf.a(stdclean.elo)
 __c30_signature
                  0x001334          0x6 c:/program files (x86)/microchip/xc16/v1.25/bin/bin/../../lib\libc-elf.a(sprintf_cdnopsuxX.XXeo)
 __c30_signature
                  0x00133a          0x6 c:/program files (x86)/microchip/xc16/v1.25/bin/bin/../../lib\libc-elf.a(doprnt_cdnopsuxX.XXeo)
 __c30_signature
                  0x001340          0x6 c:/program files (x86)/microchip/xc16/v1.25/bin/bin/../../lib\libc-elf.a(doprnt.eo)
 __c30_signature
                  0x001346          0x6 c:/program files (x86)/microchip/xc16/v1.25/bin/bin/../../lib\libc-elf.a(fputc.eo)
 __c30_signature
                  0x00134c          0x6 c:/program files (x86)/microchip/xc16/v1.25/bin/bin/../../lib\libc-elf.a(powers.eo)
 __c30_signature
                  0x001352          0x6 c:/program files (x86)/microchip/xc16/v1.25/bin/bin/../../lib\libc-elf.a(flsbuf.eo)
 __c30_signature
                  0x001358          0x6 c:/program files (x86)/microchip/xc16/v1.25/bin/bin/../../lib\libpic30-elf.a(_exit.eo)
 __c30_signature
                  0x00135e          0x6 c:/program files (x86)/microchip/xc16/v1.25/bin/bin/../../lib\libpic30-elf.a(write.eo)
 __c30_signature
                  0x001364          0x6 c:/program files (x86)/microchip/xc16/v1.25/bin/bin/../../lib\libpic30-elf.a(c30_uart.eo)
 __c30_signature
                  0x00136a          0x6 c:/program files (x86)/microchip/xc16/v1.25/bin/bin/../../lib\libm-elf.a(adddf3.eo)
 __c30_signature
                  0x001370          0x6 c:/program files (x86)/microchip/xc16/v1.25/bin/bin/../../lib\libm-elf.a(deqltle.eo)
 __c30_signature
                  0x001376          0x6 c:/program files (x86)/microchip/xc16/v1.25/bin/bin/../../lib\libm-elf.a(dgtge.eo)
 __c30_signature
                  0x00137c          0x6 c:/program files (x86)/microchip/xc16/v1.25/bin/bin/../../lib\libm-elf.a(divdf3.eo)
 __c30_signature
                  0x001382          0x6 c:/program files (x86)/microchip/xc16/v1.25/bin/bin/../../lib\libm-elf.a(dne.eo)
 __c30_signature
                  0x001388          0x6 c:/program files (x86)/microchip/xc16/v1.25/bin/bin/../../lib\libm-elf.a(dpack.eo)
 __c30_signature
                  0x00138e          0x6 c:/program files (x86)/microchip/xc16/v1.25/bin/bin/../../lib\libm-elf.a(dunpack2.eo)
 __c30_signature
                  0x001394          0x6 c:/program files (x86)/microchip/xc16/v1.25/bin/bin/../../lib\libm-elf.a(extendsfdf.eo)
 __c30_signature
                  0x00139a          0x6 c:/program files (x86)/microchip/xc16/v1.25/bin/bin/../../lib\libm-elf.a(fixunsdfdi.eo)
 __c30_signature
                  0x0013a0          0x6 c:/program files (x86)/microchip/xc16/v1.25/bin/bin/../../lib\libm-elf.a(fixunsdfsi.eo)
 __c30_signature
                  0x0013a6          0x6 c:/program files (x86)/microchip/xc16/v1.25/bin/bin/../../lib\libm-elf.a(floatundidf.eo)
 __c30_signature
                  0x0013ac          0x6 c:/program files (x86)/microchip/xc16/v1.25/bin/bin/../../lib\libm-elf.a(floatunsidf.eo)
 __c30_signature
                  0x0013b2          0x6 c:/program files (x86)/microchip/xc16/v1.25/bin/bin/../../lib\libm-elf.a(frexp.eo)
 __c30_signature
                  0x0013b8          0x6 c:/program files (x86)/microchip/xc16/v1.25/bin/bin/../../lib\libm-elf.a(funpack.eo)
 __c30_signature
                  0x0013be          0x6 c:/program files (x86)/microchip/xc16/v1.25/bin/bin/../../lib\libm-elf.a(muldf3.eo)
 __c30_signature
                  0x0013c4          0x6 c:/program files (x86)/microchip/xc16/v1.25/bin/bin/../../lib\libm-elf.a(subdf3.eo)
 __c30_signature
                  0x0013ca          0x6 c:/program files (x86)/microchip/xc16/v1.25/bin/bin/../../lib\libm-elf.a(mulsi3.eo)
 __c30_signature
                  0x0013d0          0x6 c:/program files (x86)/microchip/xc16/v1.25/bin/bin/../../lib\libm-elf.a(divmoddi3.eo)
 __c30_signature
                  0x0013d6          0x6 c:/program files (x86)/microchip/xc16/v1.25/bin/bin/../../lib\libm-elf.a(muldi3.eo)
 __c30_signature
                  0x0013dc          0x6 c:/program files (x86)/microchip/xc16/v1.25/bin/bin/../../lib\libm-elf.a(dcompare.eo)
 __c30_signature
                  0x0013e2          0x6 c:/program files (x86)/microchip/xc16/v1.25/bin/bin/../../lib\libm-elf.a(dpropagateNaN.eo)
 __c30_signature
                  0x0013e8          0x6 c:/program files (x86)/microchip/xc16/v1.25/bin/bin/../../lib\libm-elf.a(dtype.eo)
 __c30_signature
                  0x0013ee          0x6 c:/program files (x86)/microchip/xc16/v1.25/bin/bin/../../lib\libm-elf.a(dunpack.eo)
 __c30_signature
                  0x0013f4          0x6 c:/program files (x86)/microchip/xc16/v1.25/bin/bin/../../lib\libm-elf.a(umuldi3.eo)

.nbss               0x0800         0x64
 .nbss              0x0800         0x22 build/default/production/_ext/1043210786/mb.o
                    0x080e                  _pxMBFrameCBByteReceived
                    0x0810                  _pxMBFrameCBTransmitterEmpty
                    0x0812                  _pxMBPortCBTimerExpired
                    0x0814                  _pxMBFrameCBReceiveFSMCur
                    0x0816                  _pxMBFrameCBTransmitFSMCur
 .nbss              0x0822         0x12 build/default/production/_ext/1472/main.o
 .nbss              0x0834          0xe build/default/production/_ext/1470100448/mbascii.o
 .nbss              0x0842          0xa build/default/production/_ext/1477781822/mbrtu.o
 .nbss              0x084c          0xa build/default/production/_ext/1472/misc.o
 .nbss              0x0856          0x6 build/default/production/_ext/1472/sys_timer.o
 .nbss              0x085c          0x4 build/default/production/_ext/1433339410/portevent.o
 .nbss              0x0860          0x4 build/default/production/_ext/1433339410/portserial.o

.ndata              0x0864          0x4
 .ndata             0x0864          0x4 build/default/production/_ext/1472/main.o
                    0x0864                  _mbTimeout

.nbss               0x0868          0x4
 .nbss              0x0868          0x4 build/default/production/_ext/1472/serial.o

.ndata              0x086c          0x2
 .ndata             0x086c          0x2 build/default/production/_ext/1470100448/mbascii.o

.nbss               0x086e          0x2
 .nbss              0x086e          0x2 build/default/production/_ext/833655638/mbfuncother.o

.ndata              0x0870          0x4
 .ndata             0x0870          0x2 build/default/production/_ext/1043210786/mb.o
 .ndata             0x0872          0x2 build/default/production/_ext/1472/misc.o

.nbss               0x0874          0x2
 .nbss              0x0874          0x2 build/default/production/_ext/1472/dig_io.o

.bss                0x0876       0x2db8
 .bss               0x0876       0x2868 build/default/production/_ext/1472/serial.o
 .bss               0x30de        0x550 build/default/production/_ext/1472/inst_port.o

.data               0x362e        0x160
 .data              0x362e        0x160 c:/program files (x86)/microchip/xc16/v1.25/bin/bin/../../lib\libc-elf.a(powers.eo)
                    0x362e                  __powers_
                    0x36de                  __npowers_

.bss                0x378e        0x230
 .bss               0x378e        0x130 build/default/production/_ext/1472/main.o
 .bss               0x38be        0x100 build/default/production/_ext/1477781822/mbrtu.o
                    0x38be                  _ucRTUBuf

.data               0x39be        0x238
 .data              0x39be         0xca c:/program files (x86)/microchip/xc16/v1.25/bin/bin/../../lib\libc-elf.a(doprnt_cdnopsuxX.XXeo)
 .data              0x3a88         0xca c:/program files (x86)/microchip/xc16/v1.25/bin/bin/../../lib\libc-elf.a(doprnt.eo)
 .data              0x3b52         0x40 build/default/production/_ext/1043210786/mb.o
 .data              0x3b92         0x3e c:/program files (x86)/microchip/xc16/v1.25/bin/bin/../../lib\libc-elf.a(fassert.eo)
 .data              0x3bd0         0x26 c:/program files (x86)/microchip/xc16/v1.25/bin/bin/../../lib\libc-elf.a(_iob.eo)
                    0x3bd0                  __iob
                    0x3bf4                  __Files

.bss                0x3bf6         0x20
 .bss               0x3bf6         0x20 build/default/production/_ext/833655638/mbfuncother.o

.data               0x3c16         0x24
 .data              0x3c16         0x18 build/default/production/_ext/1472/serial.o
                    0x3c16                  _UxSTARegs
                    0x3c22                  _UxBRGRegs
 .data              0x3c2e          0xc build/default/production/_ext/1472/main.o

.bss                0x3c3a         0x16
 .bss               0x3c3a          0xc c:/program files (x86)/microchip/xc16/v1.25/bin/bin/../../lib\libc-elf.a(signal.eo)
 .bss               0x3c46          0x6 c:/program files (x86)/microchip/xc16/v1.25/bin/bin/../../lib\libc-elf.a(_iob.eo)
                    0x3c46                  __outdone
                    0x3c47                  __sibuf
                    0x3c49                  __sobuf
 .bss               0x3c4c          0x2 c:/program files (x86)/microchip/xc16/v1.25/bin/bin/../../lib\libc-elf.a(errno.elo)
                    0x3c4c                  _errno
 .bss               0x3c4e          0x2 c:/program files (x86)/microchip/xc16/v1.25/bin/bin/../../lib\libc-elf.a(stdclean.elo)
                    0x3c4e                  __atexitptr

.data               0x3c50          0x2
 .data              0x3c50          0x2 c:/program files (x86)/microchip/xc16/v1.25/bin/bin/../../lib\libpic30-elf.a(c30_uart.eo)
                    0x3c50                  ___C30_UART

.params           0x001000        0x400
 .params          0x001000        0x400 build/default/production/_ext/1472/flash_mem.o
                  0x001000                  _paramBuff

.config_BTMODE    0x801800          0x2
 .config_BTMODE
                  0x801800          0x2 build/default/production/_ext/1472/mcc.o

.config_ALTVREF
                  0x0157b0          0x2
 .config_ALTVREF
                  0x0157b0          0x2 build/default/production/_ext/1472/mcc.o

.config_DSWDTEN
                  0x0157ac          0x2
 .config_DSWDTEN
                  0x0157ac          0x2 build/default/production/_ext/1472/mcc.o

.config_BTSWP     0x0157a8          0x2
 .config_BTSWP    0x0157a8          0x2 build/default/production/_ext/1472/mcc.o

.config_LPCFG     0x0157a4          0x2
 .config_LPCFG    0x0157a4          0x2 build/default/production/_ext/1472/mcc.o

.config_WDTCLK    0x0157a0          0x2
 .config_WDTCLK
                  0x0157a0          0x2 build/default/production/_ext/1472/mcc.o

.config_FCKSM     0x01579c          0x2
 .config_FCKSM    0x01579c          0x2 build/default/production/_ext/1472/mcc.o

.config_IESO      0x015798          0x2
 .config_IESO     0x015798          0x2 build/default/production/_ext/1472/mcc.o

.config_AIVTDIS
                  0x015780          0x2
 .config_AIVTDIS
                  0x015780          0x2 build/default/production/_ext/1472/mcc.o

.const              0x8100        0x828 load address 0x000100  
 .const             0x8100        0x410 build/default/production/_ext/1472/main.o
 .const             0x8510        0x200 build/default/production/_ext/1477781822/mbcrc.o
 .const             0x8710         0xd8 build/default/production/_ext/1477781822/mbrtu.o
 .const             0x87e8         0xbe build/default/production/_ext/1470100448/mbascii.o
 .const             0x88a6         0x48 build/default/production/_ext/1472/dig_io.o
                    0x88a6                  _serEnblBits
                    0x88be                  _pwrBits
 .const             0x88ee         0x2e build/default/production/_ext/833655638/mbutils.o
 .const             0x891c          0xc build/default/production/_ext/1472/serial.o

.text             0x003e22       0x1dce
 .text            0x003e22        0xba6 build/default/production/_ext/1472/main.o
                  0x003e22                  _modBusTask
                  0x003e6a                  _main
                  0x003f18                  _eMBRegInputCB
                  0x003f92                  _eMBRegHoldingCB
                  0x0040c6                  _isBitSet
                  0x0040f8                  _bitSet
                  0x00415a                  _eMBRegCoilsCB
                  0x00437a                  _eMBRegDiscreteCB
                  0x00438c                  _getLine
                  0x00442c                  _signon
                  0x004448                  _checkMenuSeq
                  0x00448e                  _menuTask
                  0x0045cc                  _menuBanner
                  0x0045f8                  _menuConfig
                  0x004694                  _menuHelp
                  0x0046c2                  _menuOpt0
                  0x0046e4                  _menuOpt1
                  0x004700                  _menuOpt2
                  0x004766                  _menuOpt3
                  0x004820                  _menuOpt4
                  0x0048b2                  _menuOpt5
                  0x0048f0                  _menuOpt6
                  0x004974                  _menuOpt7
                  0x0049b4                  _menuOpt8
                  0x0049be                  _menuOpt9
 .text            0x0049c8        0xb44 build/default/production/_ext/1472/serial.o
                  0x0049c8                  _serInit
                  0x004ac4                  _serSetBaud
                  0x004b12                  _serGetBaud
                  0x004b34                  _serSetConfig
                  0x004c24                  _serGetConfig
                  0x004cda                  _serGetByte
                  0x004d12                  _serPutByte
                  0x004da0                  _serPutString
                  0x004e1a                  _serPutStringBool
                  0x004e44                  _serRxFlush
                  0x004ee0                  _serTxFlush
                  0x004f30                  _serSetBreak
                  0x005088                  _serGetBreak
                  0x0050aa                  _serIsRxFull
                  0x0050f0                  _serRxAvailable
                  0x00511c                  _serIsTxFull
                  0x005146                  _serIsTxEmpty
                  0x005170                  _serGetErrFlag
                  0x005198                  _serClrXERR
                  0x0051c4                  _serGetXERR
                  0x0051f4                  _serClrOERR
                  0x00523c                  _serGetOERR
                  0x00526a                  _serClrFERR
                  0x005296                  _serGetFERR
                  0x0052c4                  _serClrPERR
                  0x0052f0                  _serGetPERR
                  0x00531e                  _EnterAppCriticalSection
                  0x00532c                  _ExitAppCriticalSection
                  0x005340                  __U1TXInterrupt
                  0x005348                  __U1RXInterrupt
                  0x00539c                  __U2TXInterrupt
                  0x0053a4                  __U2RXInterrupt
                  0x0053f8                  __U3TXInterrupt
                  0x005400                  __U3RXInterrupt
                  0x005454                  __U4TXInterrupt
                  0x00545c                  __U4RXInterrupt
                  0x0054b0                  __U5TXInterrupt
                  0x0054b8                  __U5RXInterrupt
 .text            0x00550c        0x6e4 build/default/production/_ext/1472/inst_port.o
                  0x00550c                  _instPortInit
                  0x00554c                  _instPortTxTask
                  0x005590                  _instPortClearWriteReq
                  0x0055ac                  _instSnapshotRxAvail
                  0x0055d0                  _instPortReadReg
                  0x0058bc                  _instPortWriteReg

.text             0x000928        0x38c
 .text            0x000928        0x38c build/default/production/_ext/1470100448/mbascii.o
                  0x000928                  _eMBASCIIInit
                  0x000968                  _eMBASCIIStart
                  0x00097e                  _eMBASCIIStop
                  0x000990                  _eMBASCIIReceive
                  0x0009e6                  _eMBASCIISend
                  0x000a40                  _xMBASCIIReceiveFSM
                  0x000b20                  _xMBASCIITransmitFSM
                  0x000be2                  _xMBASCIITimerT1SExpired

.dinit            0x005bf0        0x358
 .dinit           0x005bf0        0x358 data_init

.text             0x000cb4        0x346
 .text            0x000cb4        0x346 build/default/production/_ext/1472/dig_io.o
                  0x000cb4                  _digInit
                  0x000cfe                  _digSerEnable
                  0x000d32                  _digSerDisable
                  0x000d68                  _digSetSerEnable
                  0x000dce                  _digGetSerEnable
                  0x000e02                  _digPwrSet
                  0x000ee8                  _digPwrVecSet
                  0x000fcc                  _digPwrIsOn
                  0x000ff2                  _digPwrGet

.text             0x005f48       0x19ac
 .text            0x005f48        0x308 build/default/production/_ext/833655638/mbfuncholding.o
                  0x005f48                  _eMBFuncWriteHoldingRegister
                  0x005fa0                  _eMBFuncWriteMultipleHoldingRegister
                  0x006044                  _eMBFuncReadHoldingRegister
                  0x006110                  _eMBFuncReadWriteMultipleHoldingRegister
 .text            0x006250        0x2e2 build/default/production/_ext/1472/misc.o
                  0x006250                  _miscInit
                  0x006266                  _miscRegRead
                  0x006306                  _miscRegWrite
                  0x0063c2                  _setBlinkyDebug
                  0x0063ee                  _getBlinkyDebug
                  0x0063f6                  _blinkyTask
 .text            0x006532        0x2da build/default/production/_ext/1043210786/mb.o
                  0x006532                  _eMBInit
                  0x0065ee                  _eMBRegisterCB
                  0x0066ac                  _eMBClose
                  0x0066ce                  _eMBEnable
                  0x0066ec                  _eMBDisable
                  0x006718                  _eMBPoll
 .text            0x00680c        0x26e build/default/production/_ext/1477781822/mbrtu.o
                  0x00680c                  _eMBRTUInit
                  0x006874                  _eMBRTUStart
                  0x006888                  _eMBRTUStop
                  0x00689a                  _eMBRTUReceive
                  0x0068f8                  _eMBRTUSend
                  0x006962                  _xMBRTUReceiveFSM
                  0x0069d2                  _xMBRTUTransmitFSM
                  0x006a2c                  _xMBRTUTimerT35Expired
 .text            0x006a7a        0x226 build/default/production/_ext/833655638/mbfunccoils.o
                  0x006a7a                  _eMBFuncReadCoils
                  0x006b58                  _eMBFuncWriteCoil
                  0x006bea                  _eMBFuncWriteMultipleCoils
 .text            0x006ca0        0x1ba build/default/production/_ext/1433339410/portserial.o
                  0x006ca0                  _vMBPortSerialEnable
                  0x006cc8                  _xMBPortSerialInit
                  0x006d78                  _xMBPortSerialPutByte
                  0x006d86                  _xMBPortSerialGetByte
                  0x006d98                  __U6TXInterrupt
                  0x006db8                  __U6RXInterrupt
                  0x006e28                  _EnterCriticalSection
                  0x006e3e                  _ExitCriticalSection
 .text            0x006e5a        0x1a6 build/default/production/_ext/1472/flash_mem.o
                  0x006e5a                  _memRead
                  0x006ee0                  _memWrite
                  0x006fca                  _memErase
 .text            0x007000        0x14e build/default/production/_ext/1472/sys_timer.o
                  0x007000                  _tmrInit
                  0x007020                  _tmrTask
                  0x007028                  _tmrDelayTicks
                  0x007046                  _tmrDelayMs
                  0x0070ac                  _tmrDelayUs
                  0x00710e                  _tmrGetTicks
                  0x00713a                  __T2Interrupt
 .text            0x00714e        0x128 build/default/production/_ext/833655638/mbutils.o
                  0x00714e                  _xMBUtilSetBits
                  0x0071ec                  _xMBUtilGetBits
                  0x007244                  _prveMBError2Exception
 .text            0x007276        0x124 build/default/production/_ext/1472/periph.o
                  0x007276                  _periphInit
 .text            0x00739a        0x11c build/default/production/_ext/1472/config.o
                  0x00739a                  _cfgCheck
                  0x007406                  _cfgRead
                  0x007434                  _cfgWrite
                  0x007462                  _cfgSetBootFlag
                  0x007486                  _calcCheckSum
 .text            0x0074b6         0xf0 build/default/production/_ext/1472/buffer.o
                  0x0074b6                  _bufInit
                  0x0074ea                  _bufPut
                  0x007532                  _bufGet
                  0x007588                  _bufClear
 .text            0x0075a6         0xdc build/default/production/_ext/833655638/mbfuncdisc.o
                  0x0075a6                  _eMBFuncReadDiscreteInputs
 .text            0x007682         0xce build/default/production/_ext/833655638/mbfuncinput.o
                  0x007682                  _eMBFuncReadInputRegister
 .text            0x007750         0x7e build/default/production/_ext/833655638/mbfuncother.o
                  0x007750                  _eMBSetSlaveID
                  0x0077b0                  _eMBFuncReportSlaveID
 .text            0x0077ce         0x68 build/default/production/_ext/1433339410/porttimer.o
                  0x0077ce                  _xMBPortTimersInit
                  0x0077fe                  _vMBPortTimersEnable
                  0x007808                  _vMBPortTimersDisable
                  0x007816                  __T1Interrupt
 .text            0x007836         0x5a build/default/production/_ext/1477781822/mbcrc.o
                  0x007836                  _usMBCRC16
 .text            0x007890         0x3c build/default/production/_ext/1433339410/portevent.o
                  0x007890                  _xMBPortEventInit
                  0x00789a                  _xMBPortEventPost
                  0x0078ac                  _xMBPortEventGet
 .text            0x0078cc         0x28 build/default/production/_ext/1472/mcc.o
                  0x0078cc                  _SYSTEM_Initialize
                  0x0078d4                  _OSCILLATOR_Initialize

Cross Reference Table

Symbol                                            File
CORCON                                            c:/program files (x86)/microchip/xc16/v1.25/bin/bin/../../lib\libpic30-elf.a(crt0_extended.o)
_ANSA                                             build/default/production/_ext/1472/dig_io.o
_ANSB                                             build/default/production/_ext/1472/dig_io.o
_ANSC                                             build/default/production/_ext/1472/dig_io.o
_ANSD                                             build/default/production/_ext/1472/dig_io.o
_ANSE                                             build/default/production/_ext/1472/dig_io.o
_ANSF                                             build/default/production/_ext/1472/dig_io.o
_ANSG                                             build/default/production/_ext/1472/dig_io.o
_ANSH                                             build/default/production/_ext/1472/dig_io.o
_ANSJ                                             build/default/production/_ext/1472/dig_io.o
_CLKDIV                                           build/default/production/_ext/1472/mcc.o
_DSCONbits                                        build/default/production/_ext/1472/periph.o
_DSRPAG                                           c:/program files (x86)/microchip/xc16/v1.25/bin/bin/../../lib\libpic30-elf.a(crt0_extended.o)
_DSWPAG                                           c:/program files (x86)/microchip/xc16/v1.25/bin/bin/../../lib\libpic30-elf.a(data_init_extended.o)
_EnterAppCriticalSection                          build/default/production/_ext/1472/serial.o
_EnterCriticalSection                             build/default/production/_ext/1433339410/portserial.o
                                                  build/default/production/_ext/1043210786/mb.o
                                                  build/default/production/_ext/1477781822/mbrtu.o
                                                  build/default/production/_ext/1433339410/porttimer.o
                                                  build/default/production/_ext/1470100448/mbascii.o
_ExitAppCriticalSection                           build/default/production/_ext/1472/serial.o
_ExitCriticalSection                              build/default/production/_ext/1433339410/portserial.o
                                                  build/default/production/_ext/1043210786/mb.o
                                                  build/default/production/_ext/1477781822/mbrtu.o
                                                  build/default/production/_ext/1433339410/porttimer.o
                                                  build/default/production/_ext/1470100448/mbascii.o
_IEC0bits                                         build/default/production/_ext/1472/serial.o
                                                  build/default/production/_ext/1472/sys_timer.o
                                                  build/default/production/_ext/1433339410/porttimer.o
_IEC1bits                                         build/default/production/_ext/1472/serial.o
_IEC5bits                                         build/default/production/_ext/1472/serial.o
_IEC6bits                                         build/default/production/_ext/1472/serial.o
_IEC7bits                                         build/default/production/_ext/1472/serial.o
                                                  build/default/production/_ext/1433339410/portserial.o
_IFS0bits                                         build/default/production/_ext/1472/serial.o
                                                  build/default/production/_ext/1472/sys_timer.o
                                                  build/default/production/_ext/1433339410/porttimer.o
_IFS1bits                                         build/default/production/_ext/1472/serial.o
_IFS5bits                                         build/default/production/_ext/1472/serial.o
_IFS6bits                                         build/default/production/_ext/1472/serial.o
_IFS7bits                                         build/default/production/_ext/1472/serial.o
                                                  build/default/production/_ext/1433339410/portserial.o
_INTCON1bits                                      build/default/production/_ext/1472/main.o
_IPC0bits                                         build/default/production/_ext/1433339410/porttimer.o
_IPC1bits                                         build/default/production/_ext/1472/sys_timer.o
_IPC20bits                                        build/default/production/_ext/1472/serial.o
_IPC22bits                                        build/default/production/_ext/1472/serial.o
_IPC27bits                                        build/default/production/_ext/1472/serial.o
_IPC28bits                                        build/default/production/_ext/1472/serial.o
                                                  build/default/production/_ext/1433339410/portserial.o
_IPC2bits                                         build/default/production/_ext/1472/serial.o
_IPC3bits                                         build/default/production/_ext/1472/serial.o
_IPC7bits                                         build/default/production/_ext/1472/serial.o
_LATA                                             build/default/production/_ext/1472/dig_io.o
_LATB                                             build/default/production/_ext/1472/dig_io.o
_LATBbits                                         build/default/production/_ext/1472/main.o
_LATC                                             build/default/production/_ext/1472/dig_io.o
_LATD                                             build/default/production/_ext/1472/dig_io.o
_LATDbits                                         build/default/production/_ext/1472/main.o
_LATE                                             build/default/production/_ext/1472/dig_io.o
_LATEbits                                         build/default/production/_ext/1472/dig_io.o
                                                  build/default/production/_ext/1472/misc.o
_LATF                                             build/default/production/_ext/1472/dig_io.o
_LATG                                             build/default/production/_ext/1472/dig_io.o
_LATGbits                                         build/default/production/_ext/1472/main.o
_LATH                                             build/default/production/_ext/1472/dig_io.o
_LATJ                                             build/default/production/_ext/1472/dig_io.o
_NVMADRH                                          build/default/production/_ext/1472/flash_mem.o
_NVMADRL                                          build/default/production/_ext/1472/flash_mem.o
_NVMCON                                           build/default/production/_ext/1472/flash_mem.o
_NVMCONbits                                       build/default/production/_ext/1472/flash_mem.o
_NVMKEY                                           build/default/production/_ext/1472/flash_mem.o
_OSCCON                                           build/default/production/_ext/1472/periph.o
                                                  build/default/production/_ext/1472/mcc.o
_OSCILLATOR_Initialize                            build/default/production/_ext/1472/mcc.o
_OSCTUN                                           build/default/production/_ext/1472/mcc.o
_PMD1bits                                         build/default/production/_ext/1472/periph.o
_PMD2bits                                         build/default/production/_ext/1472/periph.o
_PMD3bits                                         build/default/production/_ext/1472/periph.o
_PMD4bits                                         build/default/production/_ext/1472/periph.o
_PMD5bits                                         build/default/production/_ext/1472/periph.o
_PMD6bits                                         build/default/production/_ext/1472/periph.o
_PMD7bits                                         build/default/production/_ext/1472/periph.o
_PMD8bits                                         build/default/production/_ext/1472/periph.o
_PR1                                              build/default/production/_ext/1433339410/porttimer.o
_PR2                                              build/default/production/_ext/1472/sys_timer.o
_PR3                                              build/default/production/_ext/1472/sys_timer.o
_RCONbits                                         build/default/production/_ext/1472/periph.o
_RCOUNT                                           build/default/production/_ext/1433339410/porttimer.o
                                                  build/default/production/_ext/1433339410/portserial.o
_REFOCONH                                         build/default/production/_ext/1472/mcc.o
_REFOCONL                                         build/default/production/_ext/1472/mcc.o
_REFOTRIML                                        build/default/production/_ext/1472/mcc.o
_RPINR17bits                                      build/default/production/_ext/1472/periph.o
_RPINR18bits                                      build/default/production/_ext/1472/periph.o
_RPINR19bits                                      build/default/production/_ext/1472/periph.o
_RPINR20bits                                      build/default/production/_ext/1472/periph.o
_RPINR21bits                                      build/default/production/_ext/1472/periph.o
_RPINR27bits                                      build/default/production/_ext/1472/periph.o
_RPOR11bits                                       build/default/production/_ext/1472/periph.o
_RPOR1bits                                        build/default/production/_ext/1472/periph.o
_RPOR6bits                                        build/default/production/_ext/1472/periph.o
_RPOR8bits                                        build/default/production/_ext/1472/periph.o
_RPOR9bits                                        build/default/production/_ext/1472/periph.o
_SPI1BRGL                                         build/default/production/_ext/1472/misc.o
_SPLIM                                            c:/program files (x86)/microchip/xc16/v1.25/bin/bin/../../lib\libpic30-elf.a(crt0_extended.o)
_SR                                               c:/program files (x86)/microchip/xc16/v1.25/bin/bin/../../lib\libc-elf.a(doprnt.eo)
                                                  c:/program files (x86)/microchip/xc16/v1.25/bin/bin/../../lib\libc-elf.a(doprnt_cdnopsuxX.XXeo)
_SRbits                                           build/default/production/_ext/1472/main.o
                                                  build/default/production/_ext/1433339410/portserial.o
_SYSTEM_Initialize                                build/default/production/_ext/1472/mcc.o
                                                  build/default/production/_ext/1472/main.o
_T1CON                                            build/default/production/_ext/1433339410/porttimer.o
_T1CONbits                                        build/default/production/_ext/1433339410/porttimer.o
_T2CON                                            build/default/production/_ext/1472/sys_timer.o
_T2CONbits                                        build/default/production/_ext/1472/sys_timer.o
_T3CON                                            build/default/production/_ext/1472/sys_timer.o
_T3CONbits                                        build/default/production/_ext/1472/sys_timer.o
_TBLPAG                                           c:/program files (x86)/microchip/xc16/v1.25/bin/bin/../../lib\libpic30-elf.a(data_init_extended.o)
                                                  build/default/production/_ext/1472/flash_mem.o
_TMR1                                             build/default/production/_ext/1433339410/porttimer.o
_TMR2                                             build/default/production/_ext/1472/sys_timer.o
_TMR3                                             build/default/production/_ext/1472/sys_timer.o
_TRISA                                            build/default/production/_ext/1472/dig_io.o
_TRISB                                            build/default/production/_ext/1472/dig_io.o
_TRISC                                            build/default/production/_ext/1472/dig_io.o
_TRISD                                            build/default/production/_ext/1472/dig_io.o
_TRISE                                            build/default/production/_ext/1472/dig_io.o
_TRISF                                            build/default/production/_ext/1472/dig_io.o
_TRISG                                            build/default/production/_ext/1472/dig_io.o
_TRISH                                            build/default/production/_ext/1472/dig_io.o
_TRISJ                                            build/default/production/_ext/1472/dig_io.o
_U1BRG                                            c:/program files (x86)/microchip/xc16/v1.25/bin/bin/../../lib\libpic30-elf.a(write.eo)
                                                  build/default/production/_ext/1472/serial.o
_U1MODE                                           c:/program files (x86)/microchip/xc16/v1.25/bin/bin/../../lib\libpic30-elf.a(_exit.eo)
                                                  build/default/production/_ext/1472/serial.o
_U1MODEbits                                       c:/program files (x86)/microchip/xc16/v1.25/bin/bin/../../lib\libpic30-elf.a(write.eo)
                                                  build/default/production/_ext/1472/serial.o
_U1RXREG                                          build/default/production/_ext/1472/serial.o
_U1STA                                            c:/program files (x86)/microchip/xc16/v1.25/bin/bin/../../lib\libpic30-elf.a(_exit.eo)
                                                  build/default/production/_ext/1472/serial.o
_U1STAbits                                        c:/program files (x86)/microchip/xc16/v1.25/bin/bin/../../lib\libpic30-elf.a(write.eo)
                                                  build/default/production/_ext/1472/serial.o
_U1TXREG                                          c:/program files (x86)/microchip/xc16/v1.25/bin/bin/../../lib\libpic30-elf.a(write.eo)
                                                  build/default/production/_ext/1472/serial.o
_U2BRG                                            c:/program files (x86)/microchip/xc16/v1.25/bin/bin/../../lib\libpic30-elf.a(write.eo)
                                                  build/default/production/_ext/1472/serial.o
_U2MODE                                           build/default/production/_ext/1472/serial.o
_U2MODEbits                                       c:/program files (x86)/microchip/xc16/v1.25/bin/bin/../../lib\libpic30-elf.a(write.eo)
                                                  build/default/production/_ext/1472/serial.o
_U2RXREG                                          build/default/production/_ext/1472/serial.o
_U2STA                                            build/default/production/_ext/1472/serial.o
_U2STAbits                                        c:/program files (x86)/microchip/xc16/v1.25/bin/bin/../../lib\libpic30-elf.a(write.eo)
                                                  build/default/production/_ext/1472/serial.o
_U2TXREG                                          c:/program files (x86)/microchip/xc16/v1.25/bin/bin/../../lib\libpic30-elf.a(write.eo)
                                                  build/default/production/_ext/1472/serial.o
_U3BRG                                            build/default/production/_ext/1472/serial.o
_U3MODE                                           build/default/production/_ext/1472/serial.o
_U3MODEbits                                       build/default/production/_ext/1472/serial.o
_U3RXREG                                          build/default/production/_ext/1472/serial.o
_U3STA                                            build/default/production/_ext/1472/serial.o
_U3STAbits                                        build/default/production/_ext/1472/serial.o
_U3TXREG                                          build/default/production/_ext/1472/serial.o
_U4BRG                                            build/default/production/_ext/1472/serial.o
_U4MODE                                           build/default/production/_ext/1472/serial.o
_U4MODEbits                                       build/default/production/_ext/1472/serial.o
_U4RXREG                                          build/default/production/_ext/1472/serial.o
_U4STA                                            build/default/production/_ext/1472/serial.o
_U4STAbits                                        build/default/production/_ext/1472/serial.o
_U4TXREG                                          build/default/production/_ext/1472/serial.o
_U5BRG                                            build/default/production/_ext/1472/serial.o
_U5MODE                                           build/default/production/_ext/1472/serial.o
_U5MODEbits                                       build/default/production/_ext/1472/serial.o
_U5RXREG                                          build/default/production/_ext/1472/serial.o
_U5STA                                            build/default/production/_ext/1472/serial.o
_U5STAbits                                        build/default/production/_ext/1472/serial.o
_U5TXREG                                          build/default/production/_ext/1472/serial.o
_U6BRG                                            build/default/production/_ext/1472/serial.o
                                                  build/default/production/_ext/1433339410/portserial.o
_U6MODEbits                                       build/default/production/_ext/1433339410/portserial.o
_U6RXREG                                          build/default/production/_ext/1433339410/portserial.o
_U6STA                                            build/default/production/_ext/1472/serial.o
                                                  build/default/production/_ext/1433339410/portserial.o
_U6STAbits                                        build/default/production/_ext/1433339410/portserial.o
_U6TXREG                                          build/default/production/_ext/1433339410/portserial.o
_UxBRGRegs                                        build/default/production/_ext/1472/serial.o
_UxSTARegs                                        build/default/production/_ext/1472/serial.o
__DefaultInterrupt                                default_isr
__Files                                           c:/program files (x86)/microchip/xc16/v1.25/bin/bin/../../lib\libc-elf.a(_iob.eo)
__MIN_STACK_SIZE                                  dist/default/production/O5DaughterDbg.production.elf
__PROGRAM_END                                     dist/default/production/O5DaughterDbg.production.elf
__SPLIM_init                                      dist/default/production/O5DaughterDbg.production.elf
                                                  c:/program files (x86)/microchip/xc16/v1.25/bin/bin/../../lib\libpic30-elf.a(crt0_extended.o)
__SP_init                                         dist/default/production/O5DaughterDbg.production.elf
                                                  c:/program files (x86)/microchip/xc16/v1.25/bin/bin/../../lib\libpic30-elf.a(crt0_extended.o)
__STACKGUARD_SIZE                                 dist/default/production/O5DaughterDbg.production.elf
__T1Interrupt                                     build/default/production/_ext/1433339410/porttimer.o
__T2Interrupt                                     build/default/production/_ext/1472/sys_timer.o
__U1RXInterrupt                                   build/default/production/_ext/1472/serial.o
__U1TXInterrupt                                   build/default/production/_ext/1472/serial.o
__U2RXInterrupt                                   build/default/production/_ext/1472/serial.o
__U2TXInterrupt                                   build/default/production/_ext/1472/serial.o
__U3RXInterrupt                                   build/default/production/_ext/1472/serial.o
__U3TXInterrupt                                   build/default/production/_ext/1472/serial.o
__U4RXInterrupt                                   build/default/production/_ext/1472/serial.o
__U4TXInterrupt                                   build/default/production/_ext/1472/serial.o
__U5RXInterrupt                                   build/default/production/_ext/1472/serial.o
__U5TXInterrupt                                   build/default/production/_ext/1472/serial.o
__U6RXInterrupt                                   build/default/production/_ext/1433339410/portserial.o
__U6TXInterrupt                                   build/default/production/_ext/1433339410/portserial.o
___C30_UART                                       c:/program files (x86)/microchip/xc16/v1.25/bin/bin/../../lib\libpic30-elf.a(c30_uart.eo)
                                                  c:/program files (x86)/microchip/xc16/v1.25/bin/bin/../../lib\libpic30-elf.a(write.eo)
___adddf3                                         c:/program files (x86)/microchip/xc16/v1.25/bin/bin/../../lib\libm-elf.a(adddf3.eo)
                                                  c:/program files (x86)/microchip/xc16/v1.25/bin/bin/../../lib\libm-elf.a(subdf3.eo)
                                                  c:/program files (x86)/microchip/xc16/v1.25/bin/bin/../../lib\libc-elf.a(doprnt.eo)
___divdf3                                         c:/program files (x86)/microchip/xc16/v1.25/bin/bin/../../lib\libm-elf.a(divdf3.eo)
                                                  c:/program files (x86)/microchip/xc16/v1.25/bin/bin/../../lib\libc-elf.a(doprnt.eo)
___divdi3                                         c:/program files (x86)/microchip/xc16/v1.25/bin/bin/../../lib\libm-elf.a(divmoddi3.eo)
___divsi3                                         c:/program files (x86)/microchip/xc16/v1.25/bin/bin/../../lib\libm-elf.a(divsi3.eo)
                                                  build/default/production/_ext/1472/misc.o
                                                  build/default/production/_ext/1472/sys_timer.o
___eqdf2                                          c:/program files (x86)/microchip/xc16/v1.25/bin/bin/../../lib\libm-elf.a(deqltle.eo)
___extendsfdf2                                    c:/program files (x86)/microchip/xc16/v1.25/bin/bin/../../lib\libm-elf.a(extendsfdf.eo)
                                                  c:/program files (x86)/microchip/xc16/v1.25/bin/bin/../../lib\libc-elf.a(doprnt.eo)
___fixunsdfdi                                     c:/program files (x86)/microchip/xc16/v1.25/bin/bin/../../lib\libm-elf.a(fixunsdfdi.eo)
                                                  c:/program files (x86)/microchip/xc16/v1.25/bin/bin/../../lib\libc-elf.a(doprnt.eo)
___fixunsdfsi                                     c:/program files (x86)/microchip/xc16/v1.25/bin/bin/../../lib\libm-elf.a(fixunsdfsi.eo)
                                                  c:/program files (x86)/microchip/xc16/v1.25/bin/bin/../../lib\libc-elf.a(doprnt.eo)
___floatundidf                                    c:/program files (x86)/microchip/xc16/v1.25/bin/bin/../../lib\libm-elf.a(floatundidf.eo)
                                                  c:/program files (x86)/microchip/xc16/v1.25/bin/bin/../../lib\libm-elf.a(floatunsidf.eo)
                                                  c:/program files (x86)/microchip/xc16/v1.25/bin/bin/../../lib\libc-elf.a(doprnt.eo)
___floatunsidf                                    c:/program files (x86)/microchip/xc16/v1.25/bin/bin/../../lib\libm-elf.a(floatunsidf.eo)
                                                  c:/program files (x86)/microchip/xc16/v1.25/bin/bin/../../lib\libc-elf.a(doprnt.eo)
___gedf2                                          c:/program files (x86)/microchip/xc16/v1.25/bin/bin/../../lib\libm-elf.a(dgtge.eo)
                                                  c:/program files (x86)/microchip/xc16/v1.25/bin/bin/../../lib\libc-elf.a(doprnt.eo)
___gtdf2                                          c:/program files (x86)/microchip/xc16/v1.25/bin/bin/../../lib\libm-elf.a(dgtge.eo)
___ledf2                                          c:/program files (x86)/microchip/xc16/v1.25/bin/bin/../../lib\libm-elf.a(deqltle.eo)
___ltdf2                                          c:/program files (x86)/microchip/xc16/v1.25/bin/bin/../../lib\libm-elf.a(deqltle.eo)
                                                  c:/program files (x86)/microchip/xc16/v1.25/bin/bin/../../lib\libc-elf.a(doprnt.eo)
___moddi3                                         c:/program files (x86)/microchip/xc16/v1.25/bin/bin/../../lib\libm-elf.a(divmoddi3.eo)
___muldf3                                         c:/program files (x86)/microchip/xc16/v1.25/bin/bin/../../lib\libm-elf.a(muldf3.eo)
                                                  c:/program files (x86)/microchip/xc16/v1.25/bin/bin/../../lib\libc-elf.a(doprnt.eo)
___muldi3                                         c:/program files (x86)/microchip/xc16/v1.25/bin/bin/../../lib\libm-elf.a(muldi3.eo)
                                                  c:/program files (x86)/microchip/xc16/v1.25/bin/bin/../../lib\libc-elf.a(doprnt.eo)
                                                  c:/program files (x86)/microchip/xc16/v1.25/bin/bin/../../lib\libc-elf.a(doprnt_cdnopsuxX.XXeo)
___mulp32eds3                                     c:/program files (x86)/microchip/xc16/v1.25/bin/bin/../../lib\libm-elf.a(mulsi3.eo)
___mulp32peds3                                    c:/program files (x86)/microchip/xc16/v1.25/bin/bin/../../lib\libm-elf.a(mulsi3.eo)
___mulsi3                                         c:/program files (x86)/microchip/xc16/v1.25/bin/bin/../../lib\libm-elf.a(mulsi3.eo)
                                                  c:/program files (x86)/microchip/xc16/v1.25/bin/bin/../../lib\libc-elf.a(doprnt.eo)
                                                  c:/program files (x86)/microchip/xc16/v1.25/bin/bin/../../lib\libc-elf.a(doprnt_cdnopsuxX.XXeo)
                                                  c:/program files (x86)/microchip/xc16/v1.25/bin/bin/../../lib\libc-elf.a(strtol.eo)
                                                  c:/program files (x86)/microchip/xc16/v1.25/bin/bin/../../lib\libc-elf.a(atol.eo)
___nedf2                                          c:/program files (x86)/microchip/xc16/v1.25/bin/bin/../../lib\libm-elf.a(dne.eo)
                                                  c:/program files (x86)/microchip/xc16/v1.25/bin/bin/../../lib\libc-elf.a(doprnt.eo)
___subdf3                                         c:/program files (x86)/microchip/xc16/v1.25/bin/bin/../../lib\libm-elf.a(subdf3.eo)
                                                  c:/program files (x86)/microchip/xc16/v1.25/bin/bin/../../lib\libc-elf.a(doprnt.eo)
___udivdi3                                        c:/program files (x86)/microchip/xc16/v1.25/bin/bin/../../lib\libm-elf.a(divmoddi3.eo)
                                                  c:/program files (x86)/microchip/xc16/v1.25/bin/bin/../../lib\libc-elf.a(doprnt.eo)
                                                  c:/program files (x86)/microchip/xc16/v1.25/bin/bin/../../lib\libc-elf.a(doprnt_cdnopsuxX.XXeo)
___udivmoddi3                                     c:/program files (x86)/microchip/xc16/v1.25/bin/bin/../../lib\libm-elf.a(divmoddi3.eo)
___udivsi3                                        c:/program files (x86)/microchip/xc16/v1.25/bin/bin/../../lib\libm-elf.a(udivsi3.eo)
                                                  c:/program files (x86)/microchip/xc16/v1.25/bin/bin/../../lib\libc-elf.a(doprnt.eo)
                                                  c:/program files (x86)/microchip/xc16/v1.25/bin/bin/../../lib\libc-elf.a(doprnt_cdnopsuxX.XXeo)
                                                  c:/program files (x86)/microchip/xc16/v1.25/bin/bin/../../lib\libm-elf.a(divsi3.eo)
                                                  build/default/production/_ext/1472/serial.o
                                                  build/default/production/_ext/1472/misc.o
                                                  build/default/production/_ext/1477781822/mbrtu.o
___umoddi3                                        c:/program files (x86)/microchip/xc16/v1.25/bin/bin/../../lib\libm-elf.a(divmoddi3.eo)
                                                  c:/program files (x86)/microchip/xc16/v1.25/bin/bin/../../lib\libc-elf.a(doprnt.eo)
___umuldi3                                        c:/program files (x86)/microchip/xc16/v1.25/bin/bin/../../lib\libm-elf.a(umuldi3.eo)
                                                  c:/program files (x86)/microchip/xc16/v1.25/bin/bin/../../lib\libm-elf.a(muldi3.eo)
__atexitptr                                       c:/program files (x86)/microchip/xc16/v1.25/bin/bin/../../lib\libc-elf.a(stdclean.elo)
__bootconst_psvpage                               dist/default/production/O5DaughterDbg.production.elf
__cleanup                                         c:/program files (x86)/microchip/xc16/v1.25/bin/bin/../../lib\libc-elf.a(stdclean.elo)
                                                  c:/program files (x86)/microchip/xc16/v1.25/bin/bin/../../lib\libc-elf.a(exit.elo)
__const_length                                    dist/default/production/O5DaughterDbg.production.elf
                                                  c:/program files (x86)/microchip/xc16/v1.25/bin/bin/../../lib\libpic30-elf.a(crt0_extended.o)
__const_psvpage                                   dist/default/production/O5DaughterDbg.production.elf
                                                  c:/program files (x86)/microchip/xc16/v1.25/bin/bin/../../lib\libpic30-elf.a(crt0_extended.o)
__dPropagateNaN                                   c:/program files (x86)/microchip/xc16/v1.25/bin/bin/../../lib\libm-elf.a(dpropagateNaN.eo)
                                                  c:/program files (x86)/microchip/xc16/v1.25/bin/bin/../../lib\libm-elf.a(dunpack2.eo)
__data_init                                       c:/program files (x86)/microchip/xc16/v1.25/bin/bin/../../lib\libpic30-elf.a(data_init_extended.o)
__data_init_extended                              c:/program files (x86)/microchip/xc16/v1.25/bin/bin/../../lib\libpic30-elf.a(data_init_extended.o)
                                                  c:/program files (x86)/microchip/xc16/v1.25/bin/bin/../../lib\libpic30-elf.a(crt0_extended.o)
__dcompare                                        c:/program files (x86)/microchip/xc16/v1.25/bin/bin/../../lib\libm-elf.a(dcompare.eo)
                                                  c:/program files (x86)/microchip/xc16/v1.25/bin/bin/../../lib\libm-elf.a(dne.eo)
                                                  c:/program files (x86)/microchip/xc16/v1.25/bin/bin/../../lib\libm-elf.a(dgtge.eo)
                                                  c:/program files (x86)/microchip/xc16/v1.25/bin/bin/../../lib\libm-elf.a(deqltle.eo)
__dinit_tbloffset                                 dist/default/production/O5DaughterDbg.production.elf
                                                  c:/program files (x86)/microchip/xc16/v1.25/bin/bin/../../lib\libpic30-elf.a(crt0_extended.o)
__dinit_tblpage                                   dist/default/production/O5DaughterDbg.production.elf
                                                  c:/program files (x86)/microchip/xc16/v1.25/bin/bin/../../lib\libpic30-elf.a(crt0_extended.o)
__dpack                                           c:/program files (x86)/microchip/xc16/v1.25/bin/bin/../../lib\libm-elf.a(dpack.eo)
                                                  c:/program files (x86)/microchip/xc16/v1.25/bin/bin/../../lib\libm-elf.a(muldf3.eo)
                                                  c:/program files (x86)/microchip/xc16/v1.25/bin/bin/../../lib\libm-elf.a(floatundidf.eo)
                                                  c:/program files (x86)/microchip/xc16/v1.25/bin/bin/../../lib\libm-elf.a(divdf3.eo)
                                                  c:/program files (x86)/microchip/xc16/v1.25/bin/bin/../../lib\libm-elf.a(adddf3.eo)
__dreturnNaN                                      c:/program files (x86)/microchip/xc16/v1.25/bin/bin/../../lib\libm-elf.a(dunpack2.eo)
                                                  c:/program files (x86)/microchip/xc16/v1.25/bin/bin/../../lib\libm-elf.a(muldf3.eo)
                                                  c:/program files (x86)/microchip/xc16/v1.25/bin/bin/../../lib\libm-elf.a(divdf3.eo)
                                                  c:/program files (x86)/microchip/xc16/v1.25/bin/bin/../../lib\libm-elf.a(adddf3.eo)
__dtype                                           c:/program files (x86)/microchip/xc16/v1.25/bin/bin/../../lib\libm-elf.a(dtype.eo)
                                                  c:/program files (x86)/microchip/xc16/v1.25/bin/bin/../../lib\libm-elf.a(dcompare.eo)
__dunpack                                         c:/program files (x86)/microchip/xc16/v1.25/bin/bin/../../lib\libm-elf.a(dunpack.eo)
                                                  c:/program files (x86)/microchip/xc16/v1.25/bin/bin/../../lib\libm-elf.a(frexp.eo)
                                                  c:/program files (x86)/microchip/xc16/v1.25/bin/bin/../../lib\libm-elf.a(fixunsdfsi.eo)
                                                  c:/program files (x86)/microchip/xc16/v1.25/bin/bin/../../lib\libm-elf.a(fixunsdfdi.eo)
                                                  c:/program files (x86)/microchip/xc16/v1.25/bin/bin/../../lib\libm-elf.a(dunpack2.eo)
__dunpack2                                        c:/program files (x86)/microchip/xc16/v1.25/bin/bin/../../lib\libm-elf.a(dunpack2.eo)
                                                  c:/program files (x86)/microchip/xc16/v1.25/bin/bin/../../lib\libm-elf.a(muldf3.eo)
                                                  c:/program files (x86)/microchip/xc16/v1.25/bin/bin/../../lib\libm-elf.a(divdf3.eo)
                                                  c:/program files (x86)/microchip/xc16/v1.25/bin/bin/../../lib\libm-elf.a(adddf3.eo)
__dunpack2exit                                    c:/program files (x86)/microchip/xc16/v1.25/bin/bin/../../lib\libm-elf.a(dunpack2.eo)
                                                  c:/program files (x86)/microchip/xc16/v1.25/bin/bin/../../lib\libm-elf.a(muldf3.eo)
                                                  c:/program files (x86)/microchip/xc16/v1.25/bin/bin/../../lib\libm-elf.a(frexp.eo)
                                                  c:/program files (x86)/microchip/xc16/v1.25/bin/bin/../../lib\libm-elf.a(fixunsdfsi.eo)
                                                  c:/program files (x86)/microchip/xc16/v1.25/bin/bin/../../lib\libm-elf.a(fixunsdfdi.eo)
                                                  c:/program files (x86)/microchip/xc16/v1.25/bin/bin/../../lib\libm-elf.a(divdf3.eo)
                                                  c:/program files (x86)/microchip/xc16/v1.25/bin/bin/../../lib\libm-elf.a(adddf3.eo)
__eheap                                           dist/default/production/O5DaughterDbg.production.elf
__enable_fixed                                    dist/default/production/O5DaughterDbg.production.elf
                                                  c:/program files (x86)/microchip/xc16/v1.25/bin/bin/../../lib\libpic30-elf.a(crt0_extended.o)
__exit                                            c:/program files (x86)/microchip/xc16/v1.25/bin/bin/../../lib\libpic30-elf.a(_exit.eo)
                                                  c:/program files (x86)/microchip/xc16/v1.25/bin/bin/../../lib\libc-elf.a(exit.elo)
__fassert                                         c:/program files (x86)/microchip/xc16/v1.25/bin/bin/../../lib\libc-elf.a(fassert.eo)
                                                  build/default/production/_ext/1477781822/mbrtu.o
                                                  build/default/production/_ext/833655638/mbutils.o
                                                  build/default/production/_ext/1470100448/mbascii.o
__flsbuf                                          c:/program files (x86)/microchip/xc16/v1.25/bin/bin/../../lib\libc-elf.a(flsbuf.eo)
                                                  c:/program files (x86)/microchip/xc16/v1.25/bin/bin/../../lib\libc-elf.a(fputc.eo)
__funpack                                         c:/program files (x86)/microchip/xc16/v1.25/bin/bin/../../lib\libm-elf.a(funpack.eo)
                                                  c:/program files (x86)/microchip/xc16/v1.25/bin/bin/../../lib\libm-elf.a(extendsfdf.eo)
__has_user_init                                   c:/program files (x86)/microchip/xc16/v1.25/bin/bin/../../lib\libpic30-elf.a(crt0_extended.o)
__heap                                            dist/default/production/O5DaughterDbg.production.elf
__iob                                             c:/program files (x86)/microchip/xc16/v1.25/bin/bin/../../lib\libc-elf.a(_iob.eo)
                                                  c:/program files (x86)/microchip/xc16/v1.25/bin/bin/../../lib\libc-elf.a(fassert.eo)
__npowers_                                        c:/program files (x86)/microchip/xc16/v1.25/bin/bin/../../lib\libc-elf.a(powers.eo)
                                                  c:/program files (x86)/microchip/xc16/v1.25/bin/bin/../../lib\libc-elf.a(doprnt.eo)
__outdone                                         c:/program files (x86)/microchip/xc16/v1.25/bin/bin/../../lib\libc-elf.a(_iob.eo)
                                                  c:/program files (x86)/microchip/xc16/v1.25/bin/bin/../../lib\libc-elf.a(fputc.eo)
__powers_                                         c:/program files (x86)/microchip/xc16/v1.25/bin/bin/../../lib\libc-elf.a(powers.eo)
                                                  c:/program files (x86)/microchip/xc16/v1.25/bin/bin/../../lib\libc-elf.a(doprnt.eo)
__psv_init                                        c:/program files (x86)/microchip/xc16/v1.25/bin/bin/../../lib\libpic30-elf.a(crt0_extended.o)
__reset                                           c:/program files (x86)/microchip/xc16/v1.25/bin/bin/../../lib\libpic30-elf.a(crt0_extended.o)
__resetALT                                        dist/default/production/O5DaughterDbg.production.elf
__resetPRI                                        c:/program files (x86)/microchip/xc16/v1.25/bin/bin/../../lib\libpic30-elf.a(crt0_extended.o)
__secureconst_psvpage                             dist/default/production/O5DaughterDbg.production.elf
__sibuf                                           c:/program files (x86)/microchip/xc16/v1.25/bin/bin/../../lib\libc-elf.a(_iob.eo)
__sobuf                                           c:/program files (x86)/microchip/xc16/v1.25/bin/bin/../../lib\libc-elf.a(_iob.eo)
                                                  c:/program files (x86)/microchip/xc16/v1.25/bin/bin/../../lib\libc-elf.a(flsbuf.eo)
__sprintf_cdnopsuxX                               c:/program files (x86)/microchip/xc16/v1.25/bin/bin/../../lib\libc-elf.a(sprintf_cdnopsuxX.XXeo)
                                                  build/default/production/_ext/1472/main.o
__user_init                                       c:/program files (x86)/microchip/xc16/v1.25/bin/bin/../../lib\libpic30-elf.a(crt0_extended.o)
__vfprintf_cdnopsuxX                              c:/program files (x86)/microchip/xc16/v1.25/bin/bin/../../lib\libc-elf.a(doprnt_cdnopsuxX.XXeo)
                                                  c:/program files (x86)/microchip/xc16/v1.25/bin/bin/../../lib\libc-elf.a(sprintf_cdnopsuxX.XXeo)
_abort                                            c:/program files (x86)/microchip/xc16/v1.25/bin/bin/../../lib\libc-elf.a(signal.eo)
                                                  c:/program files (x86)/microchip/xc16/v1.25/bin/bin/../../lib\libc-elf.a(fassert.eo)
_atoi                                             c:/program files (x86)/microchip/xc16/v1.25/bin/bin/../../lib\libc-elf.a(atoi.eo)
                                                  build/default/production/_ext/1472/main.o
_atol                                             c:/program files (x86)/microchip/xc16/v1.25/bin/bin/../../lib\libc-elf.a(atol.eo)
                                                  build/default/production/_ext/1472/main.o
_bitSet                                           build/default/production/_ext/1472/main.o
_blinkyTask                                       build/default/production/_ext/1472/misc.o
                                                  build/default/production/_ext/1472/main.o
_bufClear                                         build/default/production/_ext/1472/buffer.o
                                                  build/default/production/_ext/1472/serial.o
_bufGet                                           build/default/production/_ext/1472/buffer.o
                                                  build/default/production/_ext/1472/inst_port.o
                                                  build/default/production/_ext/1472/serial.o
_bufInit                                          build/default/production/_ext/1472/buffer.o
                                                  build/default/production/_ext/1472/inst_port.o
                                                  build/default/production/_ext/1472/serial.o
_bufPut                                           build/default/production/_ext/1472/buffer.o
                                                  build/default/production/_ext/1472/inst_port.o
_calcCheckSum                                     build/default/production/_ext/1472/config.o
_cfgCheck                                         build/default/production/_ext/1472/config.o
_cfgRead                                          build/default/production/_ext/1472/config.o
                                                  build/default/production/_ext/1472/main.o
_cfgSetBootFlag                                   build/default/production/_ext/1472/config.o
_cfgWrite                                         build/default/production/_ext/1472/config.o
                                                  build/default/production/_ext/1472/main.o
_checkMenuSeq                                     build/default/production/_ext/1472/main.o
_digGetSerEnable                                  build/default/production/_ext/1472/dig_io.o
                                                  build/default/production/_ext/1472/inst_port.o
_digInit                                          build/default/production/_ext/1472/dig_io.o
                                                  build/default/production/_ext/1472/main.o
_digPwrGet                                        build/default/production/_ext/1472/dig_io.o
                                                  build/default/production/_ext/1472/misc.o
_digPwrIsOn                                       build/default/production/_ext/1472/dig_io.o
                                                  build/default/production/_ext/1472/main.o
_digPwrSet                                        build/default/production/_ext/1472/dig_io.o
                                                  build/default/production/_ext/1472/main.o
_digPwrVecSet                                     build/default/production/_ext/1472/dig_io.o
                                                  build/default/production/_ext/1472/main.o
_digSerDisable                                    build/default/production/_ext/1472/dig_io.o
                                                  build/default/production/_ext/1472/inst_port.o
_digSerEnable                                     build/default/production/_ext/1472/dig_io.o
                                                  build/default/production/_ext/1472/inst_port.o
                                                  build/default/production/_ext/1472/main.o
_digSetSerEnable                                  build/default/production/_ext/1472/dig_io.o
                                                  build/default/production/_ext/1472/main.o
_eMBASCIIInit                                     build/default/production/_ext/1470100448/mbascii.o
                                                  build/default/production/_ext/1043210786/mb.o
_eMBASCIIReceive                                  build/default/production/_ext/1470100448/mbascii.o
                                                  jump_table
                                                  build/default/production/_ext/1043210786/mb.o
_eMBASCIISend                                     build/default/production/_ext/1470100448/mbascii.o
                                                  jump_table
                                                  build/default/production/_ext/1043210786/mb.o
_eMBASCIIStart                                    build/default/production/_ext/1470100448/mbascii.o
                                                  jump_table
                                                  build/default/production/_ext/1043210786/mb.o
_eMBASCIIStop                                     build/default/production/_ext/1470100448/mbascii.o
                                                  jump_table
                                                  build/default/production/_ext/1043210786/mb.o
_eMBClose                                         build/default/production/_ext/1043210786/mb.o
_eMBDisable                                       build/default/production/_ext/1043210786/mb.o
_eMBEnable                                        build/default/production/_ext/1043210786/mb.o
                                                  build/default/production/_ext/1472/main.o
_eMBFuncReadCoils                                 build/default/production/_ext/833655638/mbfunccoils.o
                                                  jump_table
                                                  build/default/production/_ext/1043210786/mb.o
_eMBFuncReadDiscreteInputs                        build/default/production/_ext/833655638/mbfuncdisc.o
                                                  jump_table
                                                  build/default/production/_ext/1043210786/mb.o
_eMBFuncReadHoldingRegister                       build/default/production/_ext/833655638/mbfuncholding.o
                                                  jump_table
                                                  build/default/production/_ext/1043210786/mb.o
_eMBFuncReadInputRegister                         build/default/production/_ext/833655638/mbfuncinput.o
                                                  jump_table
                                                  build/default/production/_ext/1043210786/mb.o
_eMBFuncReadWriteMultipleHoldingRegister          build/default/production/_ext/833655638/mbfuncholding.o
                                                  jump_table
                                                  build/default/production/_ext/1043210786/mb.o
_eMBFuncReportSlaveID                             build/default/production/_ext/833655638/mbfuncother.o
                                                  jump_table
                                                  build/default/production/_ext/1043210786/mb.o
_eMBFuncWriteCoil                                 build/default/production/_ext/833655638/mbfunccoils.o
                                                  jump_table
                                                  build/default/production/_ext/1043210786/mb.o
_eMBFuncWriteHoldingRegister                      build/default/production/_ext/833655638/mbfuncholding.o
                                                  jump_table
                                                  build/default/production/_ext/1043210786/mb.o
_eMBFuncWriteMultipleCoils                        build/default/production/_ext/833655638/mbfunccoils.o
                                                  jump_table
                                                  build/default/production/_ext/1043210786/mb.o
_eMBFuncWriteMultipleHoldingRegister              build/default/production/_ext/833655638/mbfuncholding.o
                                                  jump_table
                                                  build/default/production/_ext/1043210786/mb.o
_eMBInit                                          build/default/production/_ext/1043210786/mb.o
                                                  build/default/production/_ext/1472/main.o
_eMBPoll                                          build/default/production/_ext/1043210786/mb.o
                                                  build/default/production/_ext/1472/main.o
_eMBRTUInit                                       build/default/production/_ext/1477781822/mbrtu.o
                                                  build/default/production/_ext/1043210786/mb.o
_eMBRTUReceive                                    build/default/production/_ext/1477781822/mbrtu.o
                                                  jump_table
                                                  build/default/production/_ext/1043210786/mb.o
_eMBRTUSend                                       build/default/production/_ext/1477781822/mbrtu.o
                                                  jump_table
                                                  build/default/production/_ext/1043210786/mb.o
_eMBRTUStart                                      build/default/production/_ext/1477781822/mbrtu.o
                                                  jump_table
                                                  build/default/production/_ext/1043210786/mb.o
_eMBRTUStop                                       build/default/production/_ext/1477781822/mbrtu.o
                                                  jump_table
                                                  build/default/production/_ext/1043210786/mb.o
_eMBRegCoilsCB                                    build/default/production/_ext/1472/main.o
                                                  build/default/production/_ext/833655638/mbfunccoils.o
_eMBRegDiscreteCB                                 build/default/production/_ext/1472/main.o
                                                  build/default/production/_ext/833655638/mbfuncdisc.o
_eMBRegHoldingCB                                  build/default/production/_ext/1472/main.o
                                                  build/default/production/_ext/833655638/mbfuncholding.o
_eMBRegInputCB                                    build/default/production/_ext/1472/main.o
                                                  build/default/production/_ext/833655638/mbfuncinput.o
_eMBRegisterCB                                    build/default/production/_ext/1043210786/mb.o
_eMBSetSlaveID                                    build/default/production/_ext/833655638/mbfuncother.o
_errno                                            c:/program files (x86)/microchip/xc16/v1.25/bin/bin/../../lib\libc-elf.a(errno.elo)
                                                  c:/program files (x86)/microchip/xc16/v1.25/bin/bin/../../lib\libc-elf.a(strtol.eo)
_exit                                             c:/program files (x86)/microchip/xc16/v1.25/bin/bin/../../lib\libc-elf.a(exit.elo)
                                                  c:/program files (x86)/microchip/xc16/v1.25/bin/bin/../../lib\libc-elf.a(signal.eo)
_fprintf                                          c:/program files (x86)/microchip/xc16/v1.25/bin/bin/../../lib\libc-elf.a(fprintf.eo)
                                                  c:/program files (x86)/microchip/xc16/v1.25/bin/bin/../../lib\libc-elf.a(fassert.eo)
_fputc                                            c:/program files (x86)/microchip/xc16/v1.25/bin/bin/../../lib\libc-elf.a(fputc.eo)
                                                  c:/program files (x86)/microchip/xc16/v1.25/bin/bin/../../lib\libc-elf.a(doprnt.eo)
                                                  c:/program files (x86)/microchip/xc16/v1.25/bin/bin/../../lib\libc-elf.a(doprnt_cdnopsuxX.XXeo)
_frexp                                            c:/program files (x86)/microchip/xc16/v1.25/bin/bin/../../lib\libm-elf.a(frexp.eo)
_frexpl                                           c:/program files (x86)/microchip/xc16/v1.25/bin/bin/../../lib\libm-elf.a(frexp.eo)
                                                  c:/program files (x86)/microchip/xc16/v1.25/bin/bin/../../lib\libc-elf.a(doprnt.eo)
_getBlinkyDebug                                   build/default/production/_ext/1472/misc.o
_getLine                                          build/default/production/_ext/1472/main.o
_instPortClearWriteReq                            build/default/production/_ext/1472/inst_port.o
                                                  build/default/production/_ext/1472/main.o
_instPortInit                                     build/default/production/_ext/1472/inst_port.o
                                                  build/default/production/_ext/1472/main.o
_instPortReadReg                                  build/default/production/_ext/1472/inst_port.o
                                                  build/default/production/_ext/1472/main.o
_instPortTxTask                                   build/default/production/_ext/1472/inst_port.o
                                                  build/default/production/_ext/1472/main.o
_instPortWriteReg                                 build/default/production/_ext/1472/inst_port.o
                                                  build/default/production/_ext/1472/main.o
_instSnapshotRxAvail                              build/default/production/_ext/1472/inst_port.o
                                                  build/default/production/_ext/1472/main.o
_isBitSet                                         build/default/production/_ext/1472/main.o
_isalpha                                          c:/program files (x86)/microchip/xc16/v1.25/bin/bin/../../lib\libc-elf.a(isalpha.eso)
                                                  c:/program files (x86)/microchip/xc16/v1.25/bin/bin/../../lib\libc-elf.a(strtol.eo)
_isspace                                          c:/program files (x86)/microchip/xc16/v1.25/bin/bin/../../lib\libc-elf.a(isspace.eso)
                                                  c:/program files (x86)/microchip/xc16/v1.25/bin/bin/../../lib\libc-elf.a(strtol.eo)
_main                                             build/default/production/_ext/1472/main.o
                                                  c:/program files (x86)/microchip/xc16/v1.25/bin/bin/../../lib\libpic30-elf.a(crt0_extended.o)
_mbTimeout                                        build/default/production/_ext/1472/main.o
                                                  build/default/production/_ext/1472/misc.o
_memErase                                         build/default/production/_ext/1472/flash_mem.o
                                                  build/default/production/_ext/1472/config.o
                                                  build/default/production/_ext/1472/main.o
_memRead                                          build/default/production/_ext/1472/flash_mem.o
                                                  build/default/production/_ext/1472/config.o
_memWrite                                         build/default/production/_ext/1472/flash_mem.o
                                                  build/default/production/_ext/1472/config.o
_memcpy                                           c:/program files (x86)/microchip/xc16/v1.25/bin/bin/../../lib\libc-elf.a(memcpy.eo)
                                                  build/default/production/_ext/1472/config.o
                                                  build/default/production/_ext/833655638/mbfuncother.o
_memset                                           c:/program files (x86)/microchip/xc16/v1.25/bin/bin/../../lib\libc-elf.a(memset.eo)
                                                  build/default/production/_ext/1472/config.o
                                                  build/default/production/_ext/1472/main.o
_menuBanner                                       build/default/production/_ext/1472/main.o
_menuConfig                                       build/default/production/_ext/1472/main.o
_menuHelp                                         build/default/production/_ext/1472/main.o
_menuOpt0                                         build/default/production/_ext/1472/main.o
_menuOpt1                                         build/default/production/_ext/1472/main.o
_menuOpt2                                         build/default/production/_ext/1472/main.o
_menuOpt3                                         build/default/production/_ext/1472/main.o
_menuOpt4                                         build/default/production/_ext/1472/main.o
_menuOpt5                                         build/default/production/_ext/1472/main.o
_menuOpt6                                         build/default/production/_ext/1472/main.o
_menuOpt7                                         build/default/production/_ext/1472/main.o
_menuOpt8                                         build/default/production/_ext/1472/main.o
_menuOpt9                                         build/default/production/_ext/1472/main.o
_menuTask                                         build/default/production/_ext/1472/main.o
_miscInit                                         build/default/production/_ext/1472/misc.o
                                                  build/default/production/_ext/1472/main.o
_miscRegRead                                      build/default/production/_ext/1472/misc.o
                                                  build/default/production/_ext/1472/main.o
_miscRegWrite                                     build/default/production/_ext/1472/misc.o
                                                  build/default/production/_ext/1472/main.o
_modBusTask                                       build/default/production/_ext/1472/main.o
_paramBuff                                        build/default/production/_ext/1472/flash_mem.o
_periphInit                                       build/default/production/_ext/1472/periph.o
                                                  build/default/production/_ext/1472/main.o
_prveMBError2Exception                            build/default/production/_ext/833655638/mbutils.o
                                                  build/default/production/_ext/833655638/mbfuncinput.o
                                                  build/default/production/_ext/833655638/mbfuncholding.o
                                                  build/default/production/_ext/833655638/mbfuncdisc.o
                                                  build/default/production/_ext/833655638/mbfunccoils.o
_pwrBits                                          build/default/production/_ext/1472/dig_io.o
_pxMBFrameCBByteReceived                          build/default/production/_ext/1043210786/mb.o
                                                  build/default/production/_ext/1433339410/portserial.o
_pxMBFrameCBReceiveFSMCur                         build/default/production/_ext/1043210786/mb.o
_pxMBFrameCBTransmitFSMCur                        build/default/production/_ext/1043210786/mb.o
_pxMBFrameCBTransmitterEmpty                      build/default/production/_ext/1043210786/mb.o
                                                  build/default/production/_ext/1433339410/portserial.o
_pxMBPortCBTimerExpired                           build/default/production/_ext/1043210786/mb.o
                                                  build/default/production/_ext/1433339410/porttimer.o
_raise                                            c:/program files (x86)/microchip/xc16/v1.25/bin/bin/../../lib\libc-elf.a(signal.eo)
_serClrFERR                                       build/default/production/_ext/1472/serial.o
                                                  build/default/production/_ext/1472/inst_port.o
_serClrOERR                                       build/default/production/_ext/1472/serial.o
                                                  build/default/production/_ext/1472/inst_port.o
_serClrPERR                                       build/default/production/_ext/1472/serial.o
                                                  build/default/production/_ext/1472/inst_port.o
_serClrXERR                                       build/default/production/_ext/1472/serial.o
                                                  build/default/production/_ext/1472/inst_port.o
_serEnblBits                                      build/default/production/_ext/1472/dig_io.o
_serGetBaud                                       build/default/production/_ext/1472/serial.o
                                                  build/default/production/_ext/1472/inst_port.o
_serGetBreak                                      build/default/production/_ext/1472/serial.o
                                                  build/default/production/_ext/1472/inst_port.o
_serGetByte                                       build/default/production/_ext/1472/serial.o
                                                  build/default/production/_ext/1472/inst_port.o
                                                  build/default/production/_ext/1472/main.o
_serGetConfig                                     build/default/production/_ext/1472/serial.o
                                                  build/default/production/_ext/1472/inst_port.o
_serGetErrFlag                                    build/default/production/_ext/1472/serial.o
                                                  build/default/production/_ext/1472/inst_port.o
_serGetFERR                                       build/default/production/_ext/1472/serial.o
                                                  build/default/production/_ext/1472/inst_port.o
_serGetOERR                                       build/default/production/_ext/1472/serial.o
                                                  build/default/production/_ext/1472/inst_port.o
_serGetPERR                                       build/default/production/_ext/1472/serial.o
                                                  build/default/production/_ext/1472/inst_port.o
_serGetXERR                                       build/default/production/_ext/1472/serial.o
                                                  build/default/production/_ext/1472/inst_port.o
_serInit                                          build/default/production/_ext/1472/serial.o
                                                  build/default/production/_ext/1472/main.o
_serIsRxFull                                      build/default/production/_ext/1472/serial.o
_serIsTxEmpty                                     build/default/production/_ext/1472/serial.o
_serIsTxFull                                      build/default/production/_ext/1472/serial.o
                                                  build/default/production/_ext/1472/inst_port.o
_serPutByte                                       build/default/production/_ext/1472/serial.o
                                                  build/default/production/_ext/1472/inst_port.o
                                                  build/default/production/_ext/1472/main.o
_serPutString                                     build/default/production/_ext/1472/serial.o
                                                  build/default/production/_ext/1472/main.o
_serPutStringBool                                 build/default/production/_ext/1472/serial.o
                                                  build/default/production/_ext/1472/main.o
_serRxAvailable                                   build/default/production/_ext/1472/serial.o
                                                  build/default/production/_ext/1472/inst_port.o
_serRxFlush                                       build/default/production/_ext/1472/serial.o
                                                  build/default/production/_ext/1472/inst_port.o
_serSetBaud                                       build/default/production/_ext/1472/serial.o
                                                  build/default/production/_ext/1472/inst_port.o
_serSetBreak                                      build/default/production/_ext/1472/serial.o
                                                  build/default/production/_ext/1472/inst_port.o
_serSetConfig                                     build/default/production/_ext/1472/serial.o
                                                  build/default/production/_ext/1472/inst_port.o
_serTxFlush                                       build/default/production/_ext/1472/serial.o
                                                  build/default/production/_ext/1472/inst_port.o
_setBlinkyDebug                                   build/default/production/_ext/1472/misc.o
                                                  build/default/production/_ext/1472/main.o
_signal                                           c:/program files (x86)/microchip/xc16/v1.25/bin/bin/../../lib\libc-elf.a(signal.eo)
_signon                                           build/default/production/_ext/1472/main.o
_strtol                                           c:/program files (x86)/microchip/xc16/v1.25/bin/bin/../../lib\libc-elf.a(strtol.eo)
                                                  build/default/production/_ext/1472/main.o
_strtoul                                          c:/program files (x86)/microchip/xc16/v1.25/bin/bin/../../lib\libc-elf.a(strtol.eo)
_tmrDelayMs                                       build/default/production/_ext/1472/sys_timer.o
_tmrDelayTicks                                    build/default/production/_ext/1472/sys_timer.o
                                                  build/default/production/_ext/1472/dig_io.o
_tmrDelayUs                                       build/default/production/_ext/1472/sys_timer.o
_tmrGetTicks                                      build/default/production/_ext/1472/sys_timer.o
                                                  build/default/production/_ext/1472/serial.o
                                                  build/default/production/_ext/1472/misc.o
_tmrInit                                          build/default/production/_ext/1472/sys_timer.o
                                                  build/default/production/_ext/1472/main.o
_tmrTask                                          build/default/production/_ext/1472/sys_timer.o
                                                  build/default/production/_ext/1472/main.o
_toupper                                          c:/program files (x86)/microchip/xc16/v1.25/bin/bin/../../lib\libc-elf.a(toupper.eso)
                                                  c:/program files (x86)/microchip/xc16/v1.25/bin/bin/../../lib\libc-elf.a(strtol.eo)
                                                  build/default/production/_ext/1472/main.o
_ucRTUBuf                                         build/default/production/_ext/1477781822/mbrtu.o
                                                  build/default/production/_ext/1470100448/mbascii.o
_usMBCRC16                                        build/default/production/_ext/1477781822/mbcrc.o
                                                  build/default/production/_ext/1477781822/mbrtu.o
_vMBPortSerialEnable                              build/default/production/_ext/1433339410/portserial.o
                                                  build/default/production/_ext/1477781822/mbrtu.o
                                                  build/default/production/_ext/1470100448/mbascii.o
_vMBPortTimersDisable                             build/default/production/_ext/1433339410/porttimer.o
                                                  build/default/production/_ext/1477781822/mbrtu.o
                                                  build/default/production/_ext/1470100448/mbascii.o
_vMBPortTimersEnable                              build/default/production/_ext/1433339410/porttimer.o
                                                  build/default/production/_ext/1477781822/mbrtu.o
                                                  build/default/production/_ext/1470100448/mbascii.o
_vfprintf                                         c:/program files (x86)/microchip/xc16/v1.25/bin/bin/../../lib\libc-elf.a(doprnt.eo)
                                                  c:/program files (x86)/microchip/xc16/v1.25/bin/bin/../../lib\libc-elf.a(fprintf.eo)
_write                                            c:/program files (x86)/microchip/xc16/v1.25/bin/bin/../../lib\libpic30-elf.a(write.eo)
                                                  c:/program files (x86)/microchip/xc16/v1.25/bin/bin/../../lib\libc-elf.a(flsbuf.eo)
                                                  c:/program files (x86)/microchip/xc16/v1.25/bin/bin/../../lib\libc-elf.a(fputc.eo)
_xMBASCIIReceiveFSM                               build/default/production/_ext/1470100448/mbascii.o
                                                  jump_table
                                                  build/default/production/_ext/1043210786/mb.o
_xMBASCIITimerT1SExpired                          build/default/production/_ext/1470100448/mbascii.o
                                                  jump_table
                                                  build/default/production/_ext/1043210786/mb.o
_xMBASCIITransmitFSM                              build/default/production/_ext/1470100448/mbascii.o
                                                  jump_table
                                                  build/default/production/_ext/1043210786/mb.o
_xMBPortEventGet                                  build/default/production/_ext/1433339410/portevent.o
                                                  build/default/production/_ext/1043210786/mb.o
_xMBPortEventInit                                 build/default/production/_ext/1433339410/portevent.o
                                                  build/default/production/_ext/1043210786/mb.o
_xMBPortEventPost                                 build/default/production/_ext/1433339410/portevent.o
                                                  build/default/production/_ext/1043210786/mb.o
                                                  build/default/production/_ext/1477781822/mbrtu.o
                                                  build/default/production/_ext/1470100448/mbascii.o
_xMBPortSerialGetByte                             build/default/production/_ext/1433339410/portserial.o
                                                  build/default/production/_ext/1477781822/mbrtu.o
                                                  build/default/production/_ext/1470100448/mbascii.o
_xMBPortSerialInit                                build/default/production/_ext/1433339410/portserial.o
                                                  build/default/production/_ext/1477781822/mbrtu.o
                                                  build/default/production/_ext/1470100448/mbascii.o
_xMBPortSerialPutByte                             build/default/production/_ext/1433339410/portserial.o
                                                  build/default/production/_ext/1477781822/mbrtu.o
                                                  build/default/production/_ext/1470100448/mbascii.o
_xMBPortTimersInit                                build/default/production/_ext/1433339410/porttimer.o
                                                  build/default/production/_ext/1472/misc.o
                                                  build/default/production/_ext/1472/main.o
                                                  build/default/production/_ext/1477781822/mbrtu.o
                                                  build/default/production/_ext/1470100448/mbascii.o
_xMBRTUReceiveFSM                                 build/default/production/_ext/1477781822/mbrtu.o
                                                  jump_table
                                                  build/default/production/_ext/1043210786/mb.o
_xMBRTUTimerT35Expired                            build/default/production/_ext/1477781822/mbrtu.o
                                                  jump_table
                                                  build/default/production/_ext/1043210786/mb.o
_xMBRTUTransmitFSM                                build/default/production/_ext/1477781822/mbrtu.o
                                                  jump_table
                                                  build/default/production/_ext/1043210786/mb.o
_xMBUtilGetBits                                   build/default/production/_ext/833655638/mbutils.o
_xMBUtilSetBits                                   build/default/production/_ext/833655638/mbutils.o
